Archive member included to satisfy reference by file (symbol)

c:/ac6/systemworkbench/plugins/fr.ac6.mcu.externaltools.arm-none.win32_1.17.0.201812190825/tools/compiler/bin/../lib/gcc/arm-none-eabi/7.3.1/../../../../arm-none-eabi/lib/thumb/v7e-m/fpv4-sp/hard\libstdc++_nano.a(new_op.o)
                              MLKWS/KWS/KWS_DNN/kws_dnn.o (operator new(unsigned int))
c:/ac6/systemworkbench/plugins/fr.ac6.mcu.externaltools.arm-none.win32_1.17.0.201812190825/tools/compiler/bin/../lib/gcc/arm-none-eabi/7.3.1/../../../../arm-none-eabi/lib/thumb/v7e-m/fpv4-sp/hard\libstdc++_nano.a(pure.o)
                              MLKWS/NN/nn.o (__cxa_pure_virtual)
c:/ac6/systemworkbench/plugins/fr.ac6.mcu.externaltools.arm-none.win32_1.17.0.201812190825/tools/compiler/bin/../lib/gcc/arm-none-eabi/7.3.1/../../../../arm-none-eabi/lib/thumb/v7e-m/fpv4-sp/hard\libstdc++_nano.a(del_opv.o)
                              MLKWS/MFCC/mfcc.o (operator delete[](void*))
c:/ac6/systemworkbench/plugins/fr.ac6.mcu.externaltools.arm-none.win32_1.17.0.201812190825/tools/compiler/bin/../lib/gcc/arm-none-eabi/7.3.1/../../../../arm-none-eabi/lib/thumb/v7e-m/fpv4-sp/hard\libstdc++_nano.a(new_handler.o)
                              c:/ac6/systemworkbench/plugins/fr.ac6.mcu.externaltools.arm-none.win32_1.17.0.201812190825/tools/compiler/bin/../lib/gcc/arm-none-eabi/7.3.1/../../../../arm-none-eabi/lib/thumb/v7e-m/fpv4-sp/hard\libstdc++_nano.a(new_op.o) (std::get_new_handler())
c:/ac6/systemworkbench/plugins/fr.ac6.mcu.externaltools.arm-none.win32_1.17.0.201812190825/tools/compiler/bin/../lib/gcc/arm-none-eabi/7.3.1/../../../../arm-none-eabi/lib/thumb/v7e-m/fpv4-sp/hard\libstdc++_nano.a(eh_terminate.o)
                              c:/ac6/systemworkbench/plugins/fr.ac6.mcu.externaltools.arm-none.win32_1.17.0.201812190825/tools/compiler/bin/../lib/gcc/arm-none-eabi/7.3.1/../../../../arm-none-eabi/lib/thumb/v7e-m/fpv4-sp/hard\libstdc++_nano.a(pure.o) (std::terminate())
c:/ac6/systemworkbench/plugins/fr.ac6.mcu.externaltools.arm-none.win32_1.17.0.201812190825/tools/compiler/bin/../lib/gcc/arm-none-eabi/7.3.1/../../../../arm-none-eabi/lib/thumb/v7e-m/fpv4-sp/hard\libstdc++_nano.a(del_ops.o)
                              MLKWS/KWS/kws.o (operator delete(void*, unsigned int))
c:/ac6/systemworkbench/plugins/fr.ac6.mcu.externaltools.arm-none.win32_1.17.0.201812190825/tools/compiler/bin/../lib/gcc/arm-none-eabi/7.3.1/../../../../arm-none-eabi/lib/thumb/v7e-m/fpv4-sp/hard\libstdc++_nano.a(new_opv.o)
                              MLKWS/KWS/kws.o (operator new[](unsigned int))
c:/ac6/systemworkbench/plugins/fr.ac6.mcu.externaltools.arm-none.win32_1.17.0.201812190825/tools/compiler/bin/../lib/gcc/arm-none-eabi/7.3.1/../../../../arm-none-eabi/lib/thumb/v7e-m/fpv4-sp/hard\libstdc++_nano.a(del_op.o)
                              c:/ac6/systemworkbench/plugins/fr.ac6.mcu.externaltools.arm-none.win32_1.17.0.201812190825/tools/compiler/bin/../lib/gcc/arm-none-eabi/7.3.1/../../../../arm-none-eabi/lib/thumb/v7e-m/fpv4-sp/hard\libstdc++_nano.a(del_opv.o) (operator delete(void*))
c:/ac6/systemworkbench/plugins/fr.ac6.mcu.externaltools.arm-none.win32_1.17.0.201812190825/tools/compiler/bin/../lib/gcc/arm-none-eabi/7.3.1/../../../../arm-none-eabi/lib/thumb/v7e-m/fpv4-sp/hard\libstdc++_nano.a(eh_term_handler.o)
                              c:/ac6/systemworkbench/plugins/fr.ac6.mcu.externaltools.arm-none.win32_1.17.0.201812190825/tools/compiler/bin/../lib/gcc/arm-none-eabi/7.3.1/../../../../arm-none-eabi/lib/thumb/v7e-m/fpv4-sp/hard\libstdc++_nano.a(eh_terminate.o) (__cxxabiv1::__terminate_handler)
c:/ac6/systemworkbench/plugins/fr.ac6.mcu.externaltools.arm-none.win32_1.17.0.201812190825/tools/compiler/bin/../lib/gcc/arm-none-eabi/7.3.1/../../../../arm-none-eabi/lib/thumb/v7e-m/fpv4-sp/hard\libstdc++_nano.a(eh_unex_handler.o)
                              c:/ac6/systemworkbench/plugins/fr.ac6.mcu.externaltools.arm-none.win32_1.17.0.201812190825/tools/compiler/bin/../lib/gcc/arm-none-eabi/7.3.1/../../../../arm-none-eabi/lib/thumb/v7e-m/fpv4-sp/hard\libstdc++_nano.a(eh_terminate.o) (__cxxabiv1::__unexpected_handler)
c:/ac6/systemworkbench/plugins/fr.ac6.mcu.externaltools.arm-none.win32_1.17.0.201812190825/tools/compiler/bin/../lib/gcc/arm-none-eabi/7.3.1/../../../../arm-none-eabi/lib/thumb/v7e-m/fpv4-sp/hard\libm.a(lib_a-s_ceil.o)
                              MLKWS/MFCC/mfcc.o (ceil)
c:/ac6/systemworkbench/plugins/fr.ac6.mcu.externaltools.arm-none.win32_1.17.0.201812190825/tools/compiler/bin/../lib/gcc/arm-none-eabi/7.3.1/../../../../arm-none-eabi/lib/thumb/v7e-m/fpv4-sp/hard\libm.a(lib_a-s_cos.o)
                              MLKWS/MFCC/mfcc.o (cos)
c:/ac6/systemworkbench/plugins/fr.ac6.mcu.externaltools.arm-none.win32_1.17.0.201812190825/tools/compiler/bin/../lib/gcc/arm-none-eabi/7.3.1/../../../../arm-none-eabi/lib/thumb/v7e-m/fpv4-sp/hard\libm.a(lib_a-sf_round.o)
                              MLKWS/MFCC/mfcc.o (roundf)
c:/ac6/systemworkbench/plugins/fr.ac6.mcu.externaltools.arm-none.win32_1.17.0.201812190825/tools/compiler/bin/../lib/gcc/arm-none-eabi/7.3.1/../../../../arm-none-eabi/lib/thumb/v7e-m/fpv4-sp/hard\libm.a(lib_a-w_log.o)
                              MLKWS/MFCC/mfcc.o (log)
c:/ac6/systemworkbench/plugins/fr.ac6.mcu.externaltools.arm-none.win32_1.17.0.201812190825/tools/compiler/bin/../lib/gcc/arm-none-eabi/7.3.1/../../../../arm-none-eabi/lib/thumb/v7e-m/fpv4-sp/hard\libm.a(lib_a-w_pow.o)
                              Application/User/datalog_application.o (pow)
c:/ac6/systemworkbench/plugins/fr.ac6.mcu.externaltools.arm-none.win32_1.17.0.201812190825/tools/compiler/bin/../lib/gcc/arm-none-eabi/7.3.1/../../../../arm-none-eabi/lib/thumb/v7e-m/fpv4-sp/hard\libm.a(lib_a-wf_log.o)
                              MLKWS/MFCC/mfcc.o (logf)
c:/ac6/systemworkbench/plugins/fr.ac6.mcu.externaltools.arm-none.win32_1.17.0.201812190825/tools/compiler/bin/../lib/gcc/arm-none-eabi/7.3.1/../../../../arm-none-eabi/lib/thumb/v7e-m/fpv4-sp/hard\libm.a(lib_a-wf_sqrt.o)
                              CMSIS/DSP/ComplexMathFunctions/arm_cmplx_mag_f32.o (sqrtf)
c:/ac6/systemworkbench/plugins/fr.ac6.mcu.externaltools.arm-none.win32_1.17.0.201812190825/tools/compiler/bin/../lib/gcc/arm-none-eabi/7.3.1/../../../../arm-none-eabi/lib/thumb/v7e-m/fpv4-sp/hard\libm.a(lib_a-e_log.o)
                              c:/ac6/systemworkbench/plugins/fr.ac6.mcu.externaltools.arm-none.win32_1.17.0.201812190825/tools/compiler/bin/../lib/gcc/arm-none-eabi/7.3.1/../../../../arm-none-eabi/lib/thumb/v7e-m/fpv4-sp/hard\libm.a(lib_a-w_log.o) (__ieee754_log)
c:/ac6/systemworkbench/plugins/fr.ac6.mcu.externaltools.arm-none.win32_1.17.0.201812190825/tools/compiler/bin/../lib/gcc/arm-none-eabi/7.3.1/../../../../arm-none-eabi/lib/thumb/v7e-m/fpv4-sp/hard\libm.a(lib_a-e_pow.o)
                              c:/ac6/systemworkbench/plugins/fr.ac6.mcu.externaltools.arm-none.win32_1.17.0.201812190825/tools/compiler/bin/../lib/gcc/arm-none-eabi/7.3.1/../../../../arm-none-eabi/lib/thumb/v7e-m/fpv4-sp/hard\libm.a(lib_a-w_pow.o) (__ieee754_pow)
c:/ac6/systemworkbench/plugins/fr.ac6.mcu.externaltools.arm-none.win32_1.17.0.201812190825/tools/compiler/bin/../lib/gcc/arm-none-eabi/7.3.1/../../../../arm-none-eabi/lib/thumb/v7e-m/fpv4-sp/hard\libm.a(lib_a-e_rem_pio2.o)
                              c:/ac6/systemworkbench/plugins/fr.ac6.mcu.externaltools.arm-none.win32_1.17.0.201812190825/tools/compiler/bin/../lib/gcc/arm-none-eabi/7.3.1/../../../../arm-none-eabi/lib/thumb/v7e-m/fpv4-sp/hard\libm.a(lib_a-s_cos.o) (__ieee754_rem_pio2)
c:/ac6/systemworkbench/plugins/fr.ac6.mcu.externaltools.arm-none.win32_1.17.0.201812190825/tools/compiler/bin/../lib/gcc/arm-none-eabi/7.3.1/../../../../arm-none-eabi/lib/thumb/v7e-m/fpv4-sp/hard\libm.a(lib_a-e_sqrt.o)
                              c:/ac6/systemworkbench/plugins/fr.ac6.mcu.externaltools.arm-none.win32_1.17.0.201812190825/tools/compiler/bin/../lib/gcc/arm-none-eabi/7.3.1/../../../../arm-none-eabi/lib/thumb/v7e-m/fpv4-sp/hard\libm.a(lib_a-e_pow.o) (__ieee754_sqrt)
c:/ac6/systemworkbench/plugins/fr.ac6.mcu.externaltools.arm-none.win32_1.17.0.201812190825/tools/compiler/bin/../lib/gcc/arm-none-eabi/7.3.1/../../../../arm-none-eabi/lib/thumb/v7e-m/fpv4-sp/hard\libm.a(lib_a-ef_log.o)
                              c:/ac6/systemworkbench/plugins/fr.ac6.mcu.externaltools.arm-none.win32_1.17.0.201812190825/tools/compiler/bin/../lib/gcc/arm-none-eabi/7.3.1/../../../../arm-none-eabi/lib/thumb/v7e-m/fpv4-sp/hard\libm.a(lib_a-wf_log.o) (__ieee754_logf)
c:/ac6/systemworkbench/plugins/fr.ac6.mcu.externaltools.arm-none.win32_1.17.0.201812190825/tools/compiler/bin/../lib/gcc/arm-none-eabi/7.3.1/../../../../arm-none-eabi/lib/thumb/v7e-m/fpv4-sp/hard\libm.a(lib_a-ef_sqrt.o)
                              c:/ac6/systemworkbench/plugins/fr.ac6.mcu.externaltools.arm-none.win32_1.17.0.201812190825/tools/compiler/bin/../lib/gcc/arm-none-eabi/7.3.1/../../../../arm-none-eabi/lib/thumb/v7e-m/fpv4-sp/hard\libm.a(lib_a-wf_sqrt.o) (__ieee754_sqrtf)
c:/ac6/systemworkbench/plugins/fr.ac6.mcu.externaltools.arm-none.win32_1.17.0.201812190825/tools/compiler/bin/../lib/gcc/arm-none-eabi/7.3.1/../../../../arm-none-eabi/lib/thumb/v7e-m/fpv4-sp/hard\libm.a(lib_a-k_cos.o)
                              c:/ac6/systemworkbench/plugins/fr.ac6.mcu.externaltools.arm-none.win32_1.17.0.201812190825/tools/compiler/bin/../lib/gcc/arm-none-eabi/7.3.1/../../../../arm-none-eabi/lib/thumb/v7e-m/fpv4-sp/hard\libm.a(lib_a-s_cos.o) (__kernel_cos)
c:/ac6/systemworkbench/plugins/fr.ac6.mcu.externaltools.arm-none.win32_1.17.0.201812190825/tools/compiler/bin/../lib/gcc/arm-none-eabi/7.3.1/../../../../arm-none-eabi/lib/thumb/v7e-m/fpv4-sp/hard\libm.a(lib_a-k_rem_pio2.o)
                              c:/ac6/systemworkbench/plugins/fr.ac6.mcu.externaltools.arm-none.win32_1.17.0.201812190825/tools/compiler/bin/../lib/gcc/arm-none-eabi/7.3.1/../../../../arm-none-eabi/lib/thumb/v7e-m/fpv4-sp/hard\libm.a(lib_a-e_rem_pio2.o) (__kernel_rem_pio2)
c:/ac6/systemworkbench/plugins/fr.ac6.mcu.externaltools.arm-none.win32_1.17.0.201812190825/tools/compiler/bin/../lib/gcc/arm-none-eabi/7.3.1/../../../../arm-none-eabi/lib/thumb/v7e-m/fpv4-sp/hard\libm.a(lib_a-k_sin.o)
                              c:/ac6/systemworkbench/plugins/fr.ac6.mcu.externaltools.arm-none.win32_1.17.0.201812190825/tools/compiler/bin/../lib/gcc/arm-none-eabi/7.3.1/../../../../arm-none-eabi/lib/thumb/v7e-m/fpv4-sp/hard\libm.a(lib_a-s_cos.o) (__kernel_sin)
c:/ac6/systemworkbench/plugins/fr.ac6.mcu.externaltools.arm-none.win32_1.17.0.201812190825/tools/compiler/bin/../lib/gcc/arm-none-eabi/7.3.1/../../../../arm-none-eabi/lib/thumb/v7e-m/fpv4-sp/hard\libm.a(lib_a-s_fabs.o)
                              c:/ac6/systemworkbench/plugins/fr.ac6.mcu.externaltools.arm-none.win32_1.17.0.201812190825/tools/compiler/bin/../lib/gcc/arm-none-eabi/7.3.1/../../../../arm-none-eabi/lib/thumb/v7e-m/fpv4-sp/hard\libm.a(lib_a-e_pow.o) (fabs)
c:/ac6/systemworkbench/plugins/fr.ac6.mcu.externaltools.arm-none.win32_1.17.0.201812190825/tools/compiler/bin/../lib/gcc/arm-none-eabi/7.3.1/../../../../arm-none-eabi/lib/thumb/v7e-m/fpv4-sp/hard\libm.a(lib_a-s_finite.o)
                              c:/ac6/systemworkbench/plugins/fr.ac6.mcu.externaltools.arm-none.win32_1.17.0.201812190825/tools/compiler/bin/../lib/gcc/arm-none-eabi/7.3.1/../../../../arm-none-eabi/lib/thumb/v7e-m/fpv4-sp/hard\libm.a(lib_a-w_pow.o) (finite)
c:/ac6/systemworkbench/plugins/fr.ac6.mcu.externaltools.arm-none.win32_1.17.0.201812190825/tools/compiler/bin/../lib/gcc/arm-none-eabi/7.3.1/../../../../arm-none-eabi/lib/thumb/v7e-m/fpv4-sp/hard\libm.a(lib_a-s_floor.o)
                              c:/ac6/systemworkbench/plugins/fr.ac6.mcu.externaltools.arm-none.win32_1.17.0.201812190825/tools/compiler/bin/../lib/gcc/arm-none-eabi/7.3.1/../../../../arm-none-eabi/lib/thumb/v7e-m/fpv4-sp/hard\libm.a(lib_a-k_rem_pio2.o) (floor)
c:/ac6/systemworkbench/plugins/fr.ac6.mcu.externaltools.arm-none.win32_1.17.0.201812190825/tools/compiler/bin/../lib/gcc/arm-none-eabi/7.3.1/../../../../arm-none-eabi/lib/thumb/v7e-m/fpv4-sp/hard\libm.a(lib_a-s_lib_ver.o)
                              c:/ac6/systemworkbench/plugins/fr.ac6.mcu.externaltools.arm-none.win32_1.17.0.201812190825/tools/compiler/bin/../lib/gcc/arm-none-eabi/7.3.1/../../../../arm-none-eabi/lib/thumb/v7e-m/fpv4-sp/hard\libm.a(lib_a-w_log.o) (__fdlib_version)
c:/ac6/systemworkbench/plugins/fr.ac6.mcu.externaltools.arm-none.win32_1.17.0.201812190825/tools/compiler/bin/../lib/gcc/arm-none-eabi/7.3.1/../../../../arm-none-eabi/lib/thumb/v7e-m/fpv4-sp/hard\libm.a(lib_a-s_matherr.o)
                              c:/ac6/systemworkbench/plugins/fr.ac6.mcu.externaltools.arm-none.win32_1.17.0.201812190825/tools/compiler/bin/../lib/gcc/arm-none-eabi/7.3.1/../../../../arm-none-eabi/lib/thumb/v7e-m/fpv4-sp/hard\libm.a(lib_a-w_log.o) (matherr)
c:/ac6/systemworkbench/plugins/fr.ac6.mcu.externaltools.arm-none.win32_1.17.0.201812190825/tools/compiler/bin/../lib/gcc/arm-none-eabi/7.3.1/../../../../arm-none-eabi/lib/thumb/v7e-m/fpv4-sp/hard\libm.a(lib_a-s_nan.o)
                              c:/ac6/systemworkbench/plugins/fr.ac6.mcu.externaltools.arm-none.win32_1.17.0.201812190825/tools/compiler/bin/../lib/gcc/arm-none-eabi/7.3.1/../../../../arm-none-eabi/lib/thumb/v7e-m/fpv4-sp/hard\libm.a(lib_a-w_log.o) (nan)
c:/ac6/systemworkbench/plugins/fr.ac6.mcu.externaltools.arm-none.win32_1.17.0.201812190825/tools/compiler/bin/../lib/gcc/arm-none-eabi/7.3.1/../../../../arm-none-eabi/lib/thumb/v7e-m/fpv4-sp/hard\libm.a(lib_a-s_rint.o)
                              c:/ac6/systemworkbench/plugins/fr.ac6.mcu.externaltools.arm-none.win32_1.17.0.201812190825/tools/compiler/bin/../lib/gcc/arm-none-eabi/7.3.1/../../../../arm-none-eabi/lib/thumb/v7e-m/fpv4-sp/hard\libm.a(lib_a-w_pow.o) (rint)
c:/ac6/systemworkbench/plugins/fr.ac6.mcu.externaltools.arm-none.win32_1.17.0.201812190825/tools/compiler/bin/../lib/gcc/arm-none-eabi/7.3.1/../../../../arm-none-eabi/lib/thumb/v7e-m/fpv4-sp/hard\libm.a(lib_a-s_scalbn.o)
                              c:/ac6/systemworkbench/plugins/fr.ac6.mcu.externaltools.arm-none.win32_1.17.0.201812190825/tools/compiler/bin/../lib/gcc/arm-none-eabi/7.3.1/../../../../arm-none-eabi/lib/thumb/v7e-m/fpv4-sp/hard\libm.a(lib_a-e_pow.o) (scalbn)
c:/ac6/systemworkbench/plugins/fr.ac6.mcu.externaltools.arm-none.win32_1.17.0.201812190825/tools/compiler/bin/../lib/gcc/arm-none-eabi/7.3.1/../../../../arm-none-eabi/lib/thumb/v7e-m/fpv4-sp/hard\libm.a(lib_a-s_copysign.o)
                              c:/ac6/systemworkbench/plugins/fr.ac6.mcu.externaltools.arm-none.win32_1.17.0.201812190825/tools/compiler/bin/../lib/gcc/arm-none-eabi/7.3.1/../../../../arm-none-eabi/lib/thumb/v7e-m/fpv4-sp/hard\libm.a(lib_a-s_scalbn.o) (copysign)
c:/ac6/systemworkbench/plugins/fr.ac6.mcu.externaltools.arm-none.win32_1.17.0.201812190825/tools/compiler/bin/../lib/gcc/arm-none-eabi/7.3.1/thumb/v7e-m/fpv4-sp/hard\libgcc.a(_arm_addsubdf3.o)
                              CMSIS/DSP/MatrixFunctions/arm_mat_inverse_f64.o (__aeabi_dsub)
c:/ac6/systemworkbench/plugins/fr.ac6.mcu.externaltools.arm-none.win32_1.17.0.201812190825/tools/compiler/bin/../lib/gcc/arm-none-eabi/7.3.1/thumb/v7e-m/fpv4-sp/hard\libgcc.a(_arm_muldivdf3.o)
                              Application/User/datalog_application.o (__aeabi_dmul)
c:/ac6/systemworkbench/plugins/fr.ac6.mcu.externaltools.arm-none.win32_1.17.0.201812190825/tools/compiler/bin/../lib/gcc/arm-none-eabi/7.3.1/thumb/v7e-m/fpv4-sp/hard\libgcc.a(_arm_cmpdf2.o)
                              CMSIS/DSP/MatrixFunctions/arm_mat_inverse_f64.o (__aeabi_dcmpeq)
c:/ac6/systemworkbench/plugins/fr.ac6.mcu.externaltools.arm-none.win32_1.17.0.201812190825/tools/compiler/bin/../lib/gcc/arm-none-eabi/7.3.1/thumb/v7e-m/fpv4-sp/hard\libgcc.a(_arm_unorddf2.o)
                              c:/ac6/systemworkbench/plugins/fr.ac6.mcu.externaltools.arm-none.win32_1.17.0.201812190825/tools/compiler/bin/../lib/gcc/arm-none-eabi/7.3.1/../../../../arm-none-eabi/lib/thumb/v7e-m/fpv4-sp/hard\libm.a(lib_a-w_log.o) (__aeabi_dcmpun)
c:/ac6/systemworkbench/plugins/fr.ac6.mcu.externaltools.arm-none.win32_1.17.0.201812190825/tools/compiler/bin/../lib/gcc/arm-none-eabi/7.3.1/thumb/v7e-m/fpv4-sp/hard\libgcc.a(_arm_fixdfsi.o)
                              Application/User/datalog_application.o (__aeabi_d2iz)
c:/ac6/systemworkbench/plugins/fr.ac6.mcu.externaltools.arm-none.win32_1.17.0.201812190825/tools/compiler/bin/../lib/gcc/arm-none-eabi/7.3.1/thumb/v7e-m/fpv4-sp/hard\libgcc.a(_arm_truncdfsf2.o)
                              MLKWS/MFCC/mfcc.o (__aeabi_d2f)
c:/ac6/systemworkbench/plugins/fr.ac6.mcu.externaltools.arm-none.win32_1.17.0.201812190825/tools/compiler/bin/../lib/gcc/arm-none-eabi/7.3.1/thumb/v7e-m/fpv4-sp/hard\libgcc.a(_aeabi_ldivmod.o)
                              CMSIS/DSP/StatisticsFunctions/arm_mean_q31.o (__aeabi_ldivmod)
c:/ac6/systemworkbench/plugins/fr.ac6.mcu.externaltools.arm-none.win32_1.17.0.201812190825/tools/compiler/bin/../lib/gcc/arm-none-eabi/7.3.1/thumb/v7e-m/fpv4-sp/hard\libgcc.a(_aeabi_uldivmod.o)
                              CMSIS/DSP/StatisticsFunctions/arm_std_q15.o (__aeabi_uldivmod)
c:/ac6/systemworkbench/plugins/fr.ac6.mcu.externaltools.arm-none.win32_1.17.0.201812190825/tools/compiler/bin/../lib/gcc/arm-none-eabi/7.3.1/thumb/v7e-m/fpv4-sp/hard\libgcc.a(_fixsfdi.o)
                              CMSIS/DSP/SupportFunctions/arm_float_to_q31.o (__aeabi_f2lz)
c:/ac6/systemworkbench/plugins/fr.ac6.mcu.externaltools.arm-none.win32_1.17.0.201812190825/tools/compiler/bin/../lib/gcc/arm-none-eabi/7.3.1/thumb/v7e-m/fpv4-sp/hard\libgcc.a(_fixunssfdi.o)
                              c:/ac6/systemworkbench/plugins/fr.ac6.mcu.externaltools.arm-none.win32_1.17.0.201812190825/tools/compiler/bin/../lib/gcc/arm-none-eabi/7.3.1/thumb/v7e-m/fpv4-sp/hard\libgcc.a(_fixsfdi.o) (__aeabi_f2ulz)
c:/ac6/systemworkbench/plugins/fr.ac6.mcu.externaltools.arm-none.win32_1.17.0.201812190825/tools/compiler/bin/../lib/gcc/arm-none-eabi/7.3.1/thumb/v7e-m/fpv4-sp/hard\libgcc.a(_udivmoddi4.o)
                              c:/ac6/systemworkbench/plugins/fr.ac6.mcu.externaltools.arm-none.win32_1.17.0.201812190825/tools/compiler/bin/../lib/gcc/arm-none-eabi/7.3.1/thumb/v7e-m/fpv4-sp/hard\libgcc.a(_aeabi_ldivmod.o) (__udivmoddi4)
c:/ac6/systemworkbench/plugins/fr.ac6.mcu.externaltools.arm-none.win32_1.17.0.201812190825/tools/compiler/bin/../lib/gcc/arm-none-eabi/7.3.1/thumb/v7e-m/fpv4-sp/hard\libgcc.a(_dvmd_tls.o)
                              c:/ac6/systemworkbench/plugins/fr.ac6.mcu.externaltools.arm-none.win32_1.17.0.201812190825/tools/compiler/bin/../lib/gcc/arm-none-eabi/7.3.1/thumb/v7e-m/fpv4-sp/hard\libgcc.a(_aeabi_ldivmod.o) (__aeabi_ldiv0)
c:/ac6/systemworkbench/plugins/fr.ac6.mcu.externaltools.arm-none.win32_1.17.0.201812190825/tools/compiler/bin/../lib/gcc/arm-none-eabi/7.3.1/thumb/v7e-m/fpv4-sp/hard\libgcc.a(_arm_fixunsdfsi.o)
                              c:/ac6/systemworkbench/plugins/fr.ac6.mcu.externaltools.arm-none.win32_1.17.0.201812190825/tools/compiler/bin/../lib/gcc/arm-none-eabi/7.3.1/thumb/v7e-m/fpv4-sp/hard\libgcc.a(_fixunssfdi.o) (__aeabi_d2uiz)
c:/ac6/systemworkbench/plugins/fr.ac6.mcu.externaltools.arm-none.win32_1.17.0.201812190825/tools/compiler/bin/../lib/gcc/arm-none-eabi/7.3.1/../../../../arm-none-eabi/lib/thumb/v7e-m/fpv4-sp/hard\libc_nano.a(lib_a-abort.o)
                              c:/ac6/systemworkbench/plugins/fr.ac6.mcu.externaltools.arm-none.win32_1.17.0.201812190825/tools/compiler/bin/../lib/gcc/arm-none-eabi/7.3.1/../../../../arm-none-eabi/lib/thumb/v7e-m/fpv4-sp/hard\libstdc++_nano.a(new_op.o) (abort)
c:/ac6/systemworkbench/plugins/fr.ac6.mcu.externaltools.arm-none.win32_1.17.0.201812190825/tools/compiler/bin/../lib/gcc/arm-none-eabi/7.3.1/../../../../arm-none-eabi/lib/thumb/v7e-m/fpv4-sp/hard\libc_nano.a(lib_a-errno.o)
                              c:/ac6/systemworkbench/plugins/fr.ac6.mcu.externaltools.arm-none.win32_1.17.0.201812190825/tools/compiler/bin/../lib/gcc/arm-none-eabi/7.3.1/../../../../arm-none-eabi/lib/thumb/v7e-m/fpv4-sp/hard\libm.a(lib_a-w_log.o) (__errno)
c:/ac6/systemworkbench/plugins/fr.ac6.mcu.externaltools.arm-none.win32_1.17.0.201812190825/tools/compiler/bin/../lib/gcc/arm-none-eabi/7.3.1/../../../../arm-none-eabi/lib/thumb/v7e-m/fpv4-sp/hard\libc_nano.a(lib_a-exit.o)
                              c:/ac6/systemworkbench/plugins/fr.ac6.mcu.externaltools.arm-none.win32_1.17.0.201812190825/tools/compiler/bin/../lib/gcc/arm-none-eabi/7.3.1/../../../../arm-none-eabi/lib/thumb/v7e-m/fpv4-sp/hard/crt0.o (exit)
c:/ac6/systemworkbench/plugins/fr.ac6.mcu.externaltools.arm-none.win32_1.17.0.201812190825/tools/compiler/bin/../lib/gcc/arm-none-eabi/7.3.1/../../../../arm-none-eabi/lib/thumb/v7e-m/fpv4-sp/hard\libc_nano.a(lib_a-impure.o)
                              c:/ac6/systemworkbench/plugins/fr.ac6.mcu.externaltools.arm-none.win32_1.17.0.201812190825/tools/compiler/bin/../lib/gcc/arm-none-eabi/7.3.1/../../../../arm-none-eabi/lib/thumb/v7e-m/fpv4-sp/hard\libc_nano.a(lib_a-exit.o) (_global_impure_ptr)
c:/ac6/systemworkbench/plugins/fr.ac6.mcu.externaltools.arm-none.win32_1.17.0.201812190825/tools/compiler/bin/../lib/gcc/arm-none-eabi/7.3.1/../../../../arm-none-eabi/lib/thumb/v7e-m/fpv4-sp/hard\libc_nano.a(lib_a-init.o)
                              c:/ac6/systemworkbench/plugins/fr.ac6.mcu.externaltools.arm-none.win32_1.17.0.201812190825/tools/compiler/bin/../lib/gcc/arm-none-eabi/7.3.1/../../../../arm-none-eabi/lib/thumb/v7e-m/fpv4-sp/hard/crt0.o (__libc_init_array)
c:/ac6/systemworkbench/plugins/fr.ac6.mcu.externaltools.arm-none.win32_1.17.0.201812190825/tools/compiler/bin/../lib/gcc/arm-none-eabi/7.3.1/../../../../arm-none-eabi/lib/thumb/v7e-m/fpv4-sp/hard\libc_nano.a(lib_a-malloc.o)
                              Middlewares/FatFs/Options/syscall.o (malloc)
c:/ac6/systemworkbench/plugins/fr.ac6.mcu.externaltools.arm-none.win32_1.17.0.201812190825/tools/compiler/bin/../lib/gcc/arm-none-eabi/7.3.1/../../../../arm-none-eabi/lib/thumb/v7e-m/fpv4-sp/hard\libc_nano.a(lib_a-memcmp.o)
                              Middlewares/STM32_BlueNRG/HCI/Controller/bluenrg_utils.o (memcmp)
c:/ac6/systemworkbench/plugins/fr.ac6.mcu.externaltools.arm-none.win32_1.17.0.201812190825/tools/compiler/bin/../lib/gcc/arm-none-eabi/7.3.1/../../../../arm-none-eabi/lib/thumb/v7e-m/fpv4-sp/hard\libc_nano.a(lib_a-memcpy-stub.o)
                              Application/User/datalog_application.o (memcpy)
c:/ac6/systemworkbench/plugins/fr.ac6.mcu.externaltools.arm-none.win32_1.17.0.201812190825/tools/compiler/bin/../lib/gcc/arm-none-eabi/7.3.1/../../../../arm-none-eabi/lib/thumb/v7e-m/fpv4-sp/hard\libc_nano.a(lib_a-memmove.o)
                              CMSIS/NN/PoolingFunctions/arm_pool_q7_HWC.o (memmove)
c:/ac6/systemworkbench/plugins/fr.ac6.mcu.externaltools.arm-none.win32_1.17.0.201812190825/tools/compiler/bin/../lib/gcc/arm-none-eabi/7.3.1/../../../../arm-none-eabi/lib/thumb/v7e-m/fpv4-sp/hard\libc_nano.a(lib_a-memset.o)
                              c:/ac6/systemworkbench/plugins/fr.ac6.mcu.externaltools.arm-none.win32_1.17.0.201812190825/tools/compiler/bin/../lib/gcc/arm-none-eabi/7.3.1/../../../../arm-none-eabi/lib/thumb/v7e-m/fpv4-sp/hard/crt0.o (memset)
c:/ac6/systemworkbench/plugins/fr.ac6.mcu.externaltools.arm-none.win32_1.17.0.201812190825/tools/compiler/bin/../lib/gcc/arm-none-eabi/7.3.1/../../../../arm-none-eabi/lib/thumb/v7e-m/fpv4-sp/hard\libc_nano.a(lib_a-nano-freer.o)
                              c:/ac6/systemworkbench/plugins/fr.ac6.mcu.externaltools.arm-none.win32_1.17.0.201812190825/tools/compiler/bin/../lib/gcc/arm-none-eabi/7.3.1/../../../../arm-none-eabi/lib/thumb/v7e-m/fpv4-sp/hard\libc_nano.a(lib_a-malloc.o) (_free_r)
c:/ac6/systemworkbench/plugins/fr.ac6.mcu.externaltools.arm-none.win32_1.17.0.201812190825/tools/compiler/bin/../lib/gcc/arm-none-eabi/7.3.1/../../../../arm-none-eabi/lib/thumb/v7e-m/fpv4-sp/hard\libc_nano.a(lib_a-nano-mallocr.o)
                              c:/ac6/systemworkbench/plugins/fr.ac6.mcu.externaltools.arm-none.win32_1.17.0.201812190825/tools/compiler/bin/../lib/gcc/arm-none-eabi/7.3.1/../../../../arm-none-eabi/lib/thumb/v7e-m/fpv4-sp/hard\libc_nano.a(lib_a-malloc.o) (_malloc_r)
c:/ac6/systemworkbench/plugins/fr.ac6.mcu.externaltools.arm-none.win32_1.17.0.201812190825/tools/compiler/bin/../lib/gcc/arm-none-eabi/7.3.1/../../../../arm-none-eabi/lib/thumb/v7e-m/fpv4-sp/hard\libc_nano.a(lib_a-nano-vfprintf_float.o)
                              (_printf_float)
c:/ac6/systemworkbench/plugins/fr.ac6.mcu.externaltools.arm-none.win32_1.17.0.201812190825/tools/compiler/bin/../lib/gcc/arm-none-eabi/7.3.1/../../../../arm-none-eabi/lib/thumb/v7e-m/fpv4-sp/hard\libc_nano.a(lib_a-nano-vfprintf_i.o)
                              c:/ac6/systemworkbench/plugins/fr.ac6.mcu.externaltools.arm-none.win32_1.17.0.201812190825/tools/compiler/bin/../lib/gcc/arm-none-eabi/7.3.1/../../../../arm-none-eabi/lib/thumb/v7e-m/fpv4-sp/hard\libc_nano.a(lib_a-nano-vfprintf_float.o) (_printf_common)
c:/ac6/systemworkbench/plugins/fr.ac6.mcu.externaltools.arm-none.win32_1.17.0.201812190825/tools/compiler/bin/../lib/gcc/arm-none-eabi/7.3.1/../../../../arm-none-eabi/lib/thumb/v7e-m/fpv4-sp/hard\libc_nano.a(lib_a-printf.o)
                              Drivers/BSP/Components/HTS221_Driver.o (printf)
c:/ac6/systemworkbench/plugins/fr.ac6.mcu.externaltools.arm-none.win32_1.17.0.201812190825/tools/compiler/bin/../lib/gcc/arm-none-eabi/7.3.1/../../../../arm-none-eabi/lib/thumb/v7e-m/fpv4-sp/hard\libc_nano.a(lib_a-sbrkr.o)
                              c:/ac6/systemworkbench/plugins/fr.ac6.mcu.externaltools.arm-none.win32_1.17.0.201812190825/tools/compiler/bin/../lib/gcc/arm-none-eabi/7.3.1/../../../../arm-none-eabi/lib/thumb/v7e-m/fpv4-sp/hard\libc_nano.a(lib_a-nano-mallocr.o) (_sbrk_r)
c:/ac6/systemworkbench/plugins/fr.ac6.mcu.externaltools.arm-none.win32_1.17.0.201812190825/tools/compiler/bin/../lib/gcc/arm-none-eabi/7.3.1/../../../../arm-none-eabi/lib/thumb/v7e-m/fpv4-sp/hard\libc_nano.a(lib_a-signal.o)
                              c:/ac6/systemworkbench/plugins/fr.ac6.mcu.externaltools.arm-none.win32_1.17.0.201812190825/tools/compiler/bin/../lib/gcc/arm-none-eabi/7.3.1/../../../../arm-none-eabi/lib/thumb/v7e-m/fpv4-sp/hard\libc_nano.a(lib_a-abort.o) (raise)
c:/ac6/systemworkbench/plugins/fr.ac6.mcu.externaltools.arm-none.win32_1.17.0.201812190825/tools/compiler/bin/../lib/gcc/arm-none-eabi/7.3.1/../../../../arm-none-eabi/lib/thumb/v7e-m/fpv4-sp/hard\libc_nano.a(lib_a-signalr.o)
                              c:/ac6/systemworkbench/plugins/fr.ac6.mcu.externaltools.arm-none.win32_1.17.0.201812190825/tools/compiler/bin/../lib/gcc/arm-none-eabi/7.3.1/../../../../arm-none-eabi/lib/thumb/v7e-m/fpv4-sp/hard\libc_nano.a(lib_a-signal.o) (_kill_r)
c:/ac6/systemworkbench/plugins/fr.ac6.mcu.externaltools.arm-none.win32_1.17.0.201812190825/tools/compiler/bin/../lib/gcc/arm-none-eabi/7.3.1/../../../../arm-none-eabi/lib/thumb/v7e-m/fpv4-sp/hard\libc_nano.a(lib_a-sprintf.o)
                              Application/User/datalog_application.o (sprintf)
c:/ac6/systemworkbench/plugins/fr.ac6.mcu.externaltools.arm-none.win32_1.17.0.201812190825/tools/compiler/bin/../lib/gcc/arm-none-eabi/7.3.1/../../../../arm-none-eabi/lib/thumb/v7e-m/fpv4-sp/hard\libc_nano.a(lib_a-strlen.o)
                              c:/ac6/systemworkbench/plugins/fr.ac6.mcu.externaltools.arm-none.win32_1.17.0.201812190825/tools/compiler/bin/../lib/gcc/arm-none-eabi/7.3.1/../../../../arm-none-eabi/lib/thumb/v7e-m/fpv4-sp/hard\libc_nano.a(lib_a-nano-vfprintf_float.o) (strlen)
c:/ac6/systemworkbench/plugins/fr.ac6.mcu.externaltools.arm-none.win32_1.17.0.201812190825/tools/compiler/bin/../lib/gcc/arm-none-eabi/7.3.1/../../../../arm-none-eabi/lib/thumb/v7e-m/fpv4-sp/hard\libc_nano.a(lib_a-dtoa.o)
                              c:/ac6/systemworkbench/plugins/fr.ac6.mcu.externaltools.arm-none.win32_1.17.0.201812190825/tools/compiler/bin/../lib/gcc/arm-none-eabi/7.3.1/../../../../arm-none-eabi/lib/thumb/v7e-m/fpv4-sp/hard\libc_nano.a(lib_a-nano-vfprintf_float.o) (_dtoa_r)
c:/ac6/systemworkbench/plugins/fr.ac6.mcu.externaltools.arm-none.win32_1.17.0.201812190825/tools/compiler/bin/../lib/gcc/arm-none-eabi/7.3.1/../../../../arm-none-eabi/lib/thumb/v7e-m/fpv4-sp/hard\libc_nano.a(lib_a-findfp.o)
                              c:/ac6/systemworkbench/plugins/fr.ac6.mcu.externaltools.arm-none.win32_1.17.0.201812190825/tools/compiler/bin/../lib/gcc/arm-none-eabi/7.3.1/../../../../arm-none-eabi/lib/thumb/v7e-m/fpv4-sp/hard\libc_nano.a(lib_a-printf.o) (__sinit)
c:/ac6/systemworkbench/plugins/fr.ac6.mcu.externaltools.arm-none.win32_1.17.0.201812190825/tools/compiler/bin/../lib/gcc/arm-none-eabi/7.3.1/../../../../arm-none-eabi/lib/thumb/v7e-m/fpv4-sp/hard\libc_nano.a(lib_a-fwalk.o)
                              c:/ac6/systemworkbench/plugins/fr.ac6.mcu.externaltools.arm-none.win32_1.17.0.201812190825/tools/compiler/bin/../lib/gcc/arm-none-eabi/7.3.1/../../../../arm-none-eabi/lib/thumb/v7e-m/fpv4-sp/hard\libc_nano.a(lib_a-findfp.o) (_fwalk)
c:/ac6/systemworkbench/plugins/fr.ac6.mcu.externaltools.arm-none.win32_1.17.0.201812190825/tools/compiler/bin/../lib/gcc/arm-none-eabi/7.3.1/../../../../arm-none-eabi/lib/thumb/v7e-m/fpv4-sp/hard\libc_nano.a(lib_a-localeconv.o)
                              c:/ac6/systemworkbench/plugins/fr.ac6.mcu.externaltools.arm-none.win32_1.17.0.201812190825/tools/compiler/bin/../lib/gcc/arm-none-eabi/7.3.1/../../../../arm-none-eabi/lib/thumb/v7e-m/fpv4-sp/hard\libc_nano.a(lib_a-nano-vfprintf_float.o) (_localeconv_r)
c:/ac6/systemworkbench/plugins/fr.ac6.mcu.externaltools.arm-none.win32_1.17.0.201812190825/tools/compiler/bin/../lib/gcc/arm-none-eabi/7.3.1/../../../../arm-none-eabi/lib/thumb/v7e-m/fpv4-sp/hard\libc_nano.a(lib_a-memchr.o)
                              c:/ac6/systemworkbench/plugins/fr.ac6.mcu.externaltools.arm-none.win32_1.17.0.201812190825/tools/compiler/bin/../lib/gcc/arm-none-eabi/7.3.1/../../../../arm-none-eabi/lib/thumb/v7e-m/fpv4-sp/hard\libc_nano.a(lib_a-nano-vfprintf_i.o) (memchr)
c:/ac6/systemworkbench/plugins/fr.ac6.mcu.externaltools.arm-none.win32_1.17.0.201812190825/tools/compiler/bin/../lib/gcc/arm-none-eabi/7.3.1/../../../../arm-none-eabi/lib/thumb/v7e-m/fpv4-sp/hard\libc_nano.a(lib_a-mlock.o)
                              c:/ac6/systemworkbench/plugins/fr.ac6.mcu.externaltools.arm-none.win32_1.17.0.201812190825/tools/compiler/bin/../lib/gcc/arm-none-eabi/7.3.1/../../../../arm-none-eabi/lib/thumb/v7e-m/fpv4-sp/hard\libc_nano.a(lib_a-nano-freer.o) (__malloc_lock)
c:/ac6/systemworkbench/plugins/fr.ac6.mcu.externaltools.arm-none.win32_1.17.0.201812190825/tools/compiler/bin/../lib/gcc/arm-none-eabi/7.3.1/../../../../arm-none-eabi/lib/thumb/v7e-m/fpv4-sp/hard\libc_nano.a(lib_a-mprec.o)
                              c:/ac6/systemworkbench/plugins/fr.ac6.mcu.externaltools.arm-none.win32_1.17.0.201812190825/tools/compiler/bin/../lib/gcc/arm-none-eabi/7.3.1/../../../../arm-none-eabi/lib/thumb/v7e-m/fpv4-sp/hard\libc_nano.a(lib_a-dtoa.o) (_Balloc)
c:/ac6/systemworkbench/plugins/fr.ac6.mcu.externaltools.arm-none.win32_1.17.0.201812190825/tools/compiler/bin/../lib/gcc/arm-none-eabi/7.3.1/../../../../arm-none-eabi/lib/thumb/v7e-m/fpv4-sp/hard\libc_nano.a(lib_a-nano-callocr.o)
                              c:/ac6/systemworkbench/plugins/fr.ac6.mcu.externaltools.arm-none.win32_1.17.0.201812190825/tools/compiler/bin/../lib/gcc/arm-none-eabi/7.3.1/../../../../arm-none-eabi/lib/thumb/v7e-m/fpv4-sp/hard\libc_nano.a(lib_a-mprec.o) (_calloc_r)
c:/ac6/systemworkbench/plugins/fr.ac6.mcu.externaltools.arm-none.win32_1.17.0.201812190825/tools/compiler/bin/../lib/gcc/arm-none-eabi/7.3.1/../../../../arm-none-eabi/lib/thumb/v7e-m/fpv4-sp/hard\libc_nano.a(lib_a-nano-svfprintf.o)
                              c:/ac6/systemworkbench/plugins/fr.ac6.mcu.externaltools.arm-none.win32_1.17.0.201812190825/tools/compiler/bin/../lib/gcc/arm-none-eabi/7.3.1/../../../../arm-none-eabi/lib/thumb/v7e-m/fpv4-sp/hard\libc_nano.a(lib_a-sprintf.o) (_svfprintf_r)
c:/ac6/systemworkbench/plugins/fr.ac6.mcu.externaltools.arm-none.win32_1.17.0.201812190825/tools/compiler/bin/../lib/gcc/arm-none-eabi/7.3.1/../../../../arm-none-eabi/lib/thumb/v7e-m/fpv4-sp/hard\libc_nano.a(lib_a-nano-vfprintf.o)
                              c:/ac6/systemworkbench/plugins/fr.ac6.mcu.externaltools.arm-none.win32_1.17.0.201812190825/tools/compiler/bin/../lib/gcc/arm-none-eabi/7.3.1/../../../../arm-none-eabi/lib/thumb/v7e-m/fpv4-sp/hard\libc_nano.a(lib_a-printf.o) (_vfprintf_r)
c:/ac6/systemworkbench/plugins/fr.ac6.mcu.externaltools.arm-none.win32_1.17.0.201812190825/tools/compiler/bin/../lib/gcc/arm-none-eabi/7.3.1/../../../../arm-none-eabi/lib/thumb/v7e-m/fpv4-sp/hard\libc_nano.a(lib_a-reent.o)
                              c:/ac6/systemworkbench/plugins/fr.ac6.mcu.externaltools.arm-none.win32_1.17.0.201812190825/tools/compiler/bin/../lib/gcc/arm-none-eabi/7.3.1/../../../../arm-none-eabi/lib/thumb/v7e-m/fpv4-sp/hard\libc_nano.a(lib_a-sbrkr.o) (errno)
c:/ac6/systemworkbench/plugins/fr.ac6.mcu.externaltools.arm-none.win32_1.17.0.201812190825/tools/compiler/bin/../lib/gcc/arm-none-eabi/7.3.1/../../../../arm-none-eabi/lib/thumb/v7e-m/fpv4-sp/hard\libc_nano.a(lib_a-stdio.o)
                              c:/ac6/systemworkbench/plugins/fr.ac6.mcu.externaltools.arm-none.win32_1.17.0.201812190825/tools/compiler/bin/../lib/gcc/arm-none-eabi/7.3.1/../../../../arm-none-eabi/lib/thumb/v7e-m/fpv4-sp/hard\libc_nano.a(lib_a-findfp.o) (__sread)
c:/ac6/systemworkbench/plugins/fr.ac6.mcu.externaltools.arm-none.win32_1.17.0.201812190825/tools/compiler/bin/../lib/gcc/arm-none-eabi/7.3.1/../../../../arm-none-eabi/lib/thumb/v7e-m/fpv4-sp/hard\libc_nano.a(lib_a-wbuf.o)
                              c:/ac6/systemworkbench/plugins/fr.ac6.mcu.externaltools.arm-none.win32_1.17.0.201812190825/tools/compiler/bin/../lib/gcc/arm-none-eabi/7.3.1/../../../../arm-none-eabi/lib/thumb/v7e-m/fpv4-sp/hard\libc_nano.a(lib_a-nano-vfprintf.o) (__swbuf_r)
c:/ac6/systemworkbench/plugins/fr.ac6.mcu.externaltools.arm-none.win32_1.17.0.201812190825/tools/compiler/bin/../lib/gcc/arm-none-eabi/7.3.1/../../../../arm-none-eabi/lib/thumb/v7e-m/fpv4-sp/hard\libc_nano.a(lib_a-writer.o)
                              c:/ac6/systemworkbench/plugins/fr.ac6.mcu.externaltools.arm-none.win32_1.17.0.201812190825/tools/compiler/bin/../lib/gcc/arm-none-eabi/7.3.1/../../../../arm-none-eabi/lib/thumb/v7e-m/fpv4-sp/hard\libc_nano.a(lib_a-stdio.o) (_write_r)
c:/ac6/systemworkbench/plugins/fr.ac6.mcu.externaltools.arm-none.win32_1.17.0.201812190825/tools/compiler/bin/../lib/gcc/arm-none-eabi/7.3.1/../../../../arm-none-eabi/lib/thumb/v7e-m/fpv4-sp/hard\libc_nano.a(lib_a-wsetup.o)
                              c:/ac6/systemworkbench/plugins/fr.ac6.mcu.externaltools.arm-none.win32_1.17.0.201812190825/tools/compiler/bin/../lib/gcc/arm-none-eabi/7.3.1/../../../../arm-none-eabi/lib/thumb/v7e-m/fpv4-sp/hard\libc_nano.a(lib_a-nano-vfprintf.o) (__swsetup_r)
c:/ac6/systemworkbench/plugins/fr.ac6.mcu.externaltools.arm-none.win32_1.17.0.201812190825/tools/compiler/bin/../lib/gcc/arm-none-eabi/7.3.1/../../../../arm-none-eabi/lib/thumb/v7e-m/fpv4-sp/hard\libc_nano.a(lib_a-closer.o)
                              c:/ac6/systemworkbench/plugins/fr.ac6.mcu.externaltools.arm-none.win32_1.17.0.201812190825/tools/compiler/bin/../lib/gcc/arm-none-eabi/7.3.1/../../../../arm-none-eabi/lib/thumb/v7e-m/fpv4-sp/hard\libc_nano.a(lib_a-stdio.o) (_close_r)
c:/ac6/systemworkbench/plugins/fr.ac6.mcu.externaltools.arm-none.win32_1.17.0.201812190825/tools/compiler/bin/../lib/gcc/arm-none-eabi/7.3.1/../../../../arm-none-eabi/lib/thumb/v7e-m/fpv4-sp/hard\libc_nano.a(lib_a-fflush.o)
                              c:/ac6/systemworkbench/plugins/fr.ac6.mcu.externaltools.arm-none.win32_1.17.0.201812190825/tools/compiler/bin/../lib/gcc/arm-none-eabi/7.3.1/../../../../arm-none-eabi/lib/thumb/v7e-m/fpv4-sp/hard\libc_nano.a(lib_a-findfp.o) (_fflush_r)
c:/ac6/systemworkbench/plugins/fr.ac6.mcu.externaltools.arm-none.win32_1.17.0.201812190825/tools/compiler/bin/../lib/gcc/arm-none-eabi/7.3.1/../../../../arm-none-eabi/lib/thumb/v7e-m/fpv4-sp/hard\libc_nano.a(lib_a-fvwrite.o)
                              c:/ac6/systemworkbench/plugins/fr.ac6.mcu.externaltools.arm-none.win32_1.17.0.201812190825/tools/compiler/bin/../lib/gcc/arm-none-eabi/7.3.1/../../../../arm-none-eabi/lib/thumb/v7e-m/fpv4-sp/hard\libc_nano.a(lib_a-nano-vfprintf.o) (__sfvwrite_r)
c:/ac6/systemworkbench/plugins/fr.ac6.mcu.externaltools.arm-none.win32_1.17.0.201812190825/tools/compiler/bin/../lib/gcc/arm-none-eabi/7.3.1/../../../../arm-none-eabi/lib/thumb/v7e-m/fpv4-sp/hard\libc_nano.a(lib_a-locale.o)
                              c:/ac6/systemworkbench/plugins/fr.ac6.mcu.externaltools.arm-none.win32_1.17.0.201812190825/tools/compiler/bin/../lib/gcc/arm-none-eabi/7.3.1/../../../../arm-none-eabi/lib/thumb/v7e-m/fpv4-sp/hard\libc_nano.a(lib_a-localeconv.o) (__global_locale)
c:/ac6/systemworkbench/plugins/fr.ac6.mcu.externaltools.arm-none.win32_1.17.0.201812190825/tools/compiler/bin/../lib/gcc/arm-none-eabi/7.3.1/../../../../arm-none-eabi/lib/thumb/v7e-m/fpv4-sp/hard\libc_nano.a(lib_a-lseekr.o)
                              c:/ac6/systemworkbench/plugins/fr.ac6.mcu.externaltools.arm-none.win32_1.17.0.201812190825/tools/compiler/bin/../lib/gcc/arm-none-eabi/7.3.1/../../../../arm-none-eabi/lib/thumb/v7e-m/fpv4-sp/hard\libc_nano.a(lib_a-stdio.o) (_lseek_r)
c:/ac6/systemworkbench/plugins/fr.ac6.mcu.externaltools.arm-none.win32_1.17.0.201812190825/tools/compiler/bin/../lib/gcc/arm-none-eabi/7.3.1/../../../../arm-none-eabi/lib/thumb/v7e-m/fpv4-sp/hard\libc_nano.a(lib_a-makebuf.o)
                              c:/ac6/systemworkbench/plugins/fr.ac6.mcu.externaltools.arm-none.win32_1.17.0.201812190825/tools/compiler/bin/../lib/gcc/arm-none-eabi/7.3.1/../../../../arm-none-eabi/lib/thumb/v7e-m/fpv4-sp/hard\libc_nano.a(lib_a-wsetup.o) (__smakebuf_r)
c:/ac6/systemworkbench/plugins/fr.ac6.mcu.externaltools.arm-none.win32_1.17.0.201812190825/tools/compiler/bin/../lib/gcc/arm-none-eabi/7.3.1/../../../../arm-none-eabi/lib/thumb/v7e-m/fpv4-sp/hard\libc_nano.a(lib_a-mbtowc_r.o)
                              c:/ac6/systemworkbench/plugins/fr.ac6.mcu.externaltools.arm-none.win32_1.17.0.201812190825/tools/compiler/bin/../lib/gcc/arm-none-eabi/7.3.1/../../../../arm-none-eabi/lib/thumb/v7e-m/fpv4-sp/hard\libc_nano.a(lib_a-locale.o) (__ascii_mbtowc)
c:/ac6/systemworkbench/plugins/fr.ac6.mcu.externaltools.arm-none.win32_1.17.0.201812190825/tools/compiler/bin/../lib/gcc/arm-none-eabi/7.3.1/../../../../arm-none-eabi/lib/thumb/v7e-m/fpv4-sp/hard\libc_nano.a(lib_a-nano-reallocr.o)
                              c:/ac6/systemworkbench/plugins/fr.ac6.mcu.externaltools.arm-none.win32_1.17.0.201812190825/tools/compiler/bin/../lib/gcc/arm-none-eabi/7.3.1/../../../../arm-none-eabi/lib/thumb/v7e-m/fpv4-sp/hard\libc_nano.a(lib_a-nano-svfprintf.o) (_realloc_r)
c:/ac6/systemworkbench/plugins/fr.ac6.mcu.externaltools.arm-none.win32_1.17.0.201812190825/tools/compiler/bin/../lib/gcc/arm-none-eabi/7.3.1/../../../../arm-none-eabi/lib/thumb/v7e-m/fpv4-sp/hard\libc_nano.a(lib_a-readr.o)
                              c:/ac6/systemworkbench/plugins/fr.ac6.mcu.externaltools.arm-none.win32_1.17.0.201812190825/tools/compiler/bin/../lib/gcc/arm-none-eabi/7.3.1/../../../../arm-none-eabi/lib/thumb/v7e-m/fpv4-sp/hard\libc_nano.a(lib_a-stdio.o) (_read_r)
c:/ac6/systemworkbench/plugins/fr.ac6.mcu.externaltools.arm-none.win32_1.17.0.201812190825/tools/compiler/bin/../lib/gcc/arm-none-eabi/7.3.1/../../../../arm-none-eabi/lib/thumb/v7e-m/fpv4-sp/hard\libc_nano.a(lib_a-strcmp.o)
                              c:/ac6/systemworkbench/plugins/fr.ac6.mcu.externaltools.arm-none.win32_1.17.0.201812190825/tools/compiler/bin/../lib/gcc/arm-none-eabi/7.3.1/../../../../arm-none-eabi/lib/thumb/v7e-m/fpv4-sp/hard\libc_nano.a(lib_a-locale.o) (strcmp)
c:/ac6/systemworkbench/plugins/fr.ac6.mcu.externaltools.arm-none.win32_1.17.0.201812190825/tools/compiler/bin/../lib/gcc/arm-none-eabi/7.3.1/../../../../arm-none-eabi/lib/thumb/v7e-m/fpv4-sp/hard\libc_nano.a(lib_a-wctomb_r.o)
                              c:/ac6/systemworkbench/plugins/fr.ac6.mcu.externaltools.arm-none.win32_1.17.0.201812190825/tools/compiler/bin/../lib/gcc/arm-none-eabi/7.3.1/../../../../arm-none-eabi/lib/thumb/v7e-m/fpv4-sp/hard\libc_nano.a(lib_a-locale.o) (__ascii_wctomb)
c:/ac6/systemworkbench/plugins/fr.ac6.mcu.externaltools.arm-none.win32_1.17.0.201812190825/tools/compiler/bin/../lib/gcc/arm-none-eabi/7.3.1/../../../../arm-none-eabi/lib/thumb/v7e-m/fpv4-sp/hard\libc_nano.a(lib_a-ctype_.o)
                              c:/ac6/systemworkbench/plugins/fr.ac6.mcu.externaltools.arm-none.win32_1.17.0.201812190825/tools/compiler/bin/../lib/gcc/arm-none-eabi/7.3.1/../../../../arm-none-eabi/lib/thumb/v7e-m/fpv4-sp/hard\libc_nano.a(lib_a-locale.o) (_ctype_)
c:/ac6/systemworkbench/plugins/fr.ac6.mcu.externaltools.arm-none.win32_1.17.0.201812190825/tools/compiler/bin/../lib/gcc/arm-none-eabi/7.3.1/../../../../arm-none-eabi/lib/thumb/v7e-m/fpv4-sp/hard\libc_nano.a(lib_a-fstatr.o)
                              c:/ac6/systemworkbench/plugins/fr.ac6.mcu.externaltools.arm-none.win32_1.17.0.201812190825/tools/compiler/bin/../lib/gcc/arm-none-eabi/7.3.1/../../../../arm-none-eabi/lib/thumb/v7e-m/fpv4-sp/hard\libc_nano.a(lib_a-makebuf.o) (_fstat_r)
c:/ac6/systemworkbench/plugins/fr.ac6.mcu.externaltools.arm-none.win32_1.17.0.201812190825/tools/compiler/bin/../lib/gcc/arm-none-eabi/7.3.1/../../../../arm-none-eabi/lib/thumb/v7e-m/fpv4-sp/hard\libc_nano.a(lib_a-isattyr.o)
                              c:/ac6/systemworkbench/plugins/fr.ac6.mcu.externaltools.arm-none.win32_1.17.0.201812190825/tools/compiler/bin/../lib/gcc/arm-none-eabi/7.3.1/../../../../arm-none-eabi/lib/thumb/v7e-m/fpv4-sp/hard\libc_nano.a(lib_a-makebuf.o) (_isatty_r)
c:/ac6/systemworkbench/plugins/fr.ac6.mcu.externaltools.arm-none.win32_1.17.0.201812190825/tools/compiler/bin/../lib/gcc/arm-none-eabi/7.3.1/../../../../arm-none-eabi/lib/thumb/v7e-m/fpv4-sp/hard\libc_nano.a(lib_a-nano-msizer.o)
                              c:/ac6/systemworkbench/plugins/fr.ac6.mcu.externaltools.arm-none.win32_1.17.0.201812190825/tools/compiler/bin/../lib/gcc/arm-none-eabi/7.3.1/../../../../arm-none-eabi/lib/thumb/v7e-m/fpv4-sp/hard\libc_nano.a(lib_a-nano-reallocr.o) (_malloc_usable_size_r)
c:/ac6/systemworkbench/plugins/fr.ac6.mcu.externaltools.arm-none.win32_1.17.0.201812190825/tools/compiler/bin/../lib/gcc/arm-none-eabi/7.3.1/../../../../arm-none-eabi/lib/thumb/v7e-m/fpv4-sp/hard\libnosys.a(close.o)
                              c:/ac6/systemworkbench/plugins/fr.ac6.mcu.externaltools.arm-none.win32_1.17.0.201812190825/tools/compiler/bin/../lib/gcc/arm-none-eabi/7.3.1/../../../../arm-none-eabi/lib/thumb/v7e-m/fpv4-sp/hard\libc_nano.a(lib_a-closer.o) (_close)
c:/ac6/systemworkbench/plugins/fr.ac6.mcu.externaltools.arm-none.win32_1.17.0.201812190825/tools/compiler/bin/../lib/gcc/arm-none-eabi/7.3.1/../../../../arm-none-eabi/lib/thumb/v7e-m/fpv4-sp/hard\libnosys.a(fstat.o)
                              c:/ac6/systemworkbench/plugins/fr.ac6.mcu.externaltools.arm-none.win32_1.17.0.201812190825/tools/compiler/bin/../lib/gcc/arm-none-eabi/7.3.1/../../../../arm-none-eabi/lib/thumb/v7e-m/fpv4-sp/hard\libc_nano.a(lib_a-fstatr.o) (_fstat)
c:/ac6/systemworkbench/plugins/fr.ac6.mcu.externaltools.arm-none.win32_1.17.0.201812190825/tools/compiler/bin/../lib/gcc/arm-none-eabi/7.3.1/../../../../arm-none-eabi/lib/thumb/v7e-m/fpv4-sp/hard\libnosys.a(getpid.o)
                              c:/ac6/systemworkbench/plugins/fr.ac6.mcu.externaltools.arm-none.win32_1.17.0.201812190825/tools/compiler/bin/../lib/gcc/arm-none-eabi/7.3.1/../../../../arm-none-eabi/lib/thumb/v7e-m/fpv4-sp/hard\libc_nano.a(lib_a-signalr.o) (_getpid)
c:/ac6/systemworkbench/plugins/fr.ac6.mcu.externaltools.arm-none.win32_1.17.0.201812190825/tools/compiler/bin/../lib/gcc/arm-none-eabi/7.3.1/../../../../arm-none-eabi/lib/thumb/v7e-m/fpv4-sp/hard\libnosys.a(isatty.o)
                              c:/ac6/systemworkbench/plugins/fr.ac6.mcu.externaltools.arm-none.win32_1.17.0.201812190825/tools/compiler/bin/../lib/gcc/arm-none-eabi/7.3.1/../../../../arm-none-eabi/lib/thumb/v7e-m/fpv4-sp/hard\libc_nano.a(lib_a-isattyr.o) (_isatty)
c:/ac6/systemworkbench/plugins/fr.ac6.mcu.externaltools.arm-none.win32_1.17.0.201812190825/tools/compiler/bin/../lib/gcc/arm-none-eabi/7.3.1/../../../../arm-none-eabi/lib/thumb/v7e-m/fpv4-sp/hard\libnosys.a(kill.o)
                              c:/ac6/systemworkbench/plugins/fr.ac6.mcu.externaltools.arm-none.win32_1.17.0.201812190825/tools/compiler/bin/../lib/gcc/arm-none-eabi/7.3.1/../../../../arm-none-eabi/lib/thumb/v7e-m/fpv4-sp/hard\libc_nano.a(lib_a-signalr.o) (_kill)
c:/ac6/systemworkbench/plugins/fr.ac6.mcu.externaltools.arm-none.win32_1.17.0.201812190825/tools/compiler/bin/../lib/gcc/arm-none-eabi/7.3.1/../../../../arm-none-eabi/lib/thumb/v7e-m/fpv4-sp/hard\libnosys.a(lseek.o)
                              c:/ac6/systemworkbench/plugins/fr.ac6.mcu.externaltools.arm-none.win32_1.17.0.201812190825/tools/compiler/bin/../lib/gcc/arm-none-eabi/7.3.1/../../../../arm-none-eabi/lib/thumb/v7e-m/fpv4-sp/hard\libc_nano.a(lib_a-lseekr.o) (_lseek)
c:/ac6/systemworkbench/plugins/fr.ac6.mcu.externaltools.arm-none.win32_1.17.0.201812190825/tools/compiler/bin/../lib/gcc/arm-none-eabi/7.3.1/../../../../arm-none-eabi/lib/thumb/v7e-m/fpv4-sp/hard\libnosys.a(read.o)
                              c:/ac6/systemworkbench/plugins/fr.ac6.mcu.externaltools.arm-none.win32_1.17.0.201812190825/tools/compiler/bin/../lib/gcc/arm-none-eabi/7.3.1/../../../../arm-none-eabi/lib/thumb/v7e-m/fpv4-sp/hard\libc_nano.a(lib_a-readr.o) (_read)
c:/ac6/systemworkbench/plugins/fr.ac6.mcu.externaltools.arm-none.win32_1.17.0.201812190825/tools/compiler/bin/../lib/gcc/arm-none-eabi/7.3.1/../../../../arm-none-eabi/lib/thumb/v7e-m/fpv4-sp/hard\libnosys.a(sbrk.o)
                              c:/ac6/systemworkbench/plugins/fr.ac6.mcu.externaltools.arm-none.win32_1.17.0.201812190825/tools/compiler/bin/../lib/gcc/arm-none-eabi/7.3.1/../../../../arm-none-eabi/lib/thumb/v7e-m/fpv4-sp/hard\libc_nano.a(lib_a-sbrkr.o) (_sbrk)
c:/ac6/systemworkbench/plugins/fr.ac6.mcu.externaltools.arm-none.win32_1.17.0.201812190825/tools/compiler/bin/../lib/gcc/arm-none-eabi/7.3.1/../../../../arm-none-eabi/lib/thumb/v7e-m/fpv4-sp/hard\libnosys.a(write.o)
                              c:/ac6/systemworkbench/plugins/fr.ac6.mcu.externaltools.arm-none.win32_1.17.0.201812190825/tools/compiler/bin/../lib/gcc/arm-none-eabi/7.3.1/../../../../arm-none-eabi/lib/thumb/v7e-m/fpv4-sp/hard\libc_nano.a(lib_a-writer.o) (_write)
c:/ac6/systemworkbench/plugins/fr.ac6.mcu.externaltools.arm-none.win32_1.17.0.201812190825/tools/compiler/bin/../lib/gcc/arm-none-eabi/7.3.1/../../../../arm-none-eabi/lib/thumb/v7e-m/fpv4-sp/hard\libnosys.a(_exit.o)
                              c:/ac6/systemworkbench/plugins/fr.ac6.mcu.externaltools.arm-none.win32_1.17.0.201812190825/tools/compiler/bin/../lib/gcc/arm-none-eabi/7.3.1/../../../../arm-none-eabi/lib/thumb/v7e-m/fpv4-sp/hard\libc_nano.a(lib_a-abort.o) (_exit)

Allocating common symbols
Common symbol       size              file

errno               0x4               c:/ac6/systemworkbench/plugins/fr.ac6.mcu.externaltools.arm-none.win32_1.17.0.201812190825/tools/compiler/bin/../lib/gcc/arm-none-eabi/7.3.1/../../../../arm-none-eabi/lib/thumb/v7e-m/fpv4-sp/hard\libc_nano.a(lib_a-reent.o)
USB_RxBuffer        0x800             Application/User/usbd_cdc_interface.o
byteswritten        0x4               Application/User/datalog_application.o
hciReadPktPool      0x8               Middlewares/STM32_BlueNRG/HCI/hci.o
BuffLength          0x4               Application/User/usbd_cdc_interface.o
hpcd                0x3cc             Application/User/usbd_conf.o
uwTick              0x4               Drivers/STM32L4xx_HAL_Driver/stm32l4xx_hal.o
xQueueRegistry      0x320             Middlewares/FreeRTOS/queue.o
pFlash              0x20              Drivers/STM32L4xx_HAL_Driver/stm32l4xx_hal_flash.o
bytesread           0x4               Application/User/datalog_application.o
TimCCHandle         0x3c              Application/User/sensor_service.o
TargetBoardFeatures
                    0x34              Application/User/TargetPlatform.o
UserTxBuffer        0x800             Application/User/usbd_cdc_interface.o
SPI_SD_Handle       0x64              Drivers/BSP/SensorTile/SensorTile.o
allCharHandle       0x200             Application/User/sensor_service.o
SDPath              0x4               Application/User/datalog_application.o
SpiHandle           0x64              Drivers/BSP/SensorTile/SensorTile_BlueNRG.o
hdma_tx             0x48              Drivers/BSP/SensorTile/SensorTile.o
SDFatFs             0x230             Application/User/datalog_application.o
HTS221_Combo_Data   0x4               Drivers/BSP/Components/HTS221_Driver_HL.o
LSM6DSM_Combo_Data  0x2               Drivers/BSP/Components/LSM6DSM_ACC_GYRO_driver_HL.o
UserRxBuffer        0x800             Application/User/usbd_cdc_interface.o
MyFile              0x22c             Application/User/datalog_application.o
LSM303AGR_Combo_Data
                    0x2               Drivers/BSP/Components/LSM303AGR_ACC_driver_HL.o
res                 0x1               Application/User/datalog_application.o
USBD_StrDesc        0x100             Application/User/usbd_desc.o
TimHandle           0x3c              Application/User/usbd_cdc_interface.o
hciReadPktRxQueue   0x8               Middlewares/STM32_BlueNRG/HCI/hci.o
LPS22HB_Combo_Data  0x8               Drivers/BSP/Components/LPS22HB_Driver_HL.o

Discarded input sections

 .text          0x00000000        0x0 c:/ac6/systemworkbench/plugins/fr.ac6.mcu.externaltools.arm-none.win32_1.17.0.201812190825/tools/compiler/bin/../lib/gcc/arm-none-eabi/7.3.1/thumb/v7e-m/fpv4-sp/hard/crti.o
 .data          0x00000000        0x0 c:/ac6/systemworkbench/plugins/fr.ac6.mcu.externaltools.arm-none.win32_1.17.0.201812190825/tools/compiler/bin/../lib/gcc/arm-none-eabi/7.3.1/thumb/v7e-m/fpv4-sp/hard/crti.o
 .bss           0x00000000        0x0 c:/ac6/systemworkbench/plugins/fr.ac6.mcu.externaltools.arm-none.win32_1.17.0.201812190825/tools/compiler/bin/../lib/gcc/arm-none-eabi/7.3.1/thumb/v7e-m/fpv4-sp/hard/crti.o
 .data          0x00000000        0x4 c:/ac6/systemworkbench/plugins/fr.ac6.mcu.externaltools.arm-none.win32_1.17.0.201812190825/tools/compiler/bin/../lib/gcc/arm-none-eabi/7.3.1/thumb/v7e-m/fpv4-sp/hard/crtbegin.o
 .text          0x00000000       0x74 c:/ac6/systemworkbench/plugins/fr.ac6.mcu.externaltools.arm-none.win32_1.17.0.201812190825/tools/compiler/bin/../lib/gcc/arm-none-eabi/7.3.1/../../../../arm-none-eabi/lib/thumb/v7e-m/fpv4-sp/hard/crt0.o
 .data          0x00000000        0x0 c:/ac6/systemworkbench/plugins/fr.ac6.mcu.externaltools.arm-none.win32_1.17.0.201812190825/tools/compiler/bin/../lib/gcc/arm-none-eabi/7.3.1/../../../../arm-none-eabi/lib/thumb/v7e-m/fpv4-sp/hard/crt0.o
 .bss           0x00000000        0x0 c:/ac6/systemworkbench/plugins/fr.ac6.mcu.externaltools.arm-none.win32_1.17.0.201812190825/tools/compiler/bin/../lib/gcc/arm-none-eabi/7.3.1/../../../../arm-none-eabi/lib/thumb/v7e-m/fpv4-sp/hard/crt0.o
 .ARM.extab     0x00000000        0x0 c:/ac6/systemworkbench/plugins/fr.ac6.mcu.externaltools.arm-none.win32_1.17.0.201812190825/tools/compiler/bin/../lib/gcc/arm-none-eabi/7.3.1/../../../../arm-none-eabi/lib/thumb/v7e-m/fpv4-sp/hard/crt0.o
 .ARM.exidx     0x00000000        0x8 c:/ac6/systemworkbench/plugins/fr.ac6.mcu.externaltools.arm-none.win32_1.17.0.201812190825/tools/compiler/bin/../lib/gcc/arm-none-eabi/7.3.1/../../../../arm-none-eabi/lib/thumb/v7e-m/fpv4-sp/hard/crt0.o
 .ARM.attributes
                0x00000000       0x20 c:/ac6/systemworkbench/plugins/fr.ac6.mcu.externaltools.arm-none.win32_1.17.0.201812190825/tools/compiler/bin/../lib/gcc/arm-none-eabi/7.3.1/../../../../arm-none-eabi/lib/thumb/v7e-m/fpv4-sp/hard/crt0.o
 .group         0x00000000        0xc Application/User/TargetPlatform.o
 .group         0x00000000        0xc Application/User/TargetPlatform.o
 .group         0x00000000        0xc Application/User/TargetPlatform.o
 .group         0x00000000        0xc Application/User/TargetPlatform.o
 .group         0x00000000        0xc Application/User/TargetPlatform.o
 .group         0x00000000        0xc Application/User/TargetPlatform.o
 .group         0x00000000        0xc Application/User/TargetPlatform.o
Memory Configuration

Name             Origin             Length             Attributes
FLASH            0x08000000         0x00100000         xr
RAM              0x20000000         0x00018000         xrw
*default*        0x00000000         0xffffffff

Linker script and memory map

LOAD c:/ac6/systemworkbench/plugins/fr.ac6.mcu.externaltools.arm-none.win32_1.17.0.201812190825/tools/compiler/bin/../lib/gcc/arm-none-eabi/7.3.1/thumb/v7e-m/fpv4-sp/hard/crti.o
LOAD c:/ac6/systemworkbench/plugins/fr.ac6.mcu.externaltools.arm-none.win32_1.17.0.201812190825/tools/compiler/bin/../lib/gcc/arm-none-eabi/7.3.1/thumb/v7e-m/fpv4-sp/hard/crtbegin.o
LOAD c:/ac6/systemworkbench/plugins/fr.ac6.mcu.externaltools.arm-none.win32_1.17.0.201812190825/tools/compiler/bin/../lib/gcc/arm-none-eabi/7.3.1/../../../../arm-none-eabi/lib/thumb/v7e-m/fpv4-sp/hard/crt0.o
LOAD Application/User/TargetPlatform.o
LOAD Application/User/cube_hal_l4.o
LOAD Application/User/datalog_application.o
LOAD Application/User/main.o
LOAD Application/User/sensor_service.o
LOAD Application/User/stm32l4xx_hal_msp.o
LOAD Application/User/stm32l4xx_it.o
LOAD Application/User/usbd_cdc_interface.o
LOAD Application/User/usbd_conf.o
LOAD Application/User/usbd_desc.o
LOAD CMSIS/DSP/BasicMathFunctions/arm_abs_f32.o
LOAD CMSIS/DSP/BasicMathFunctions/arm_abs_q15.o
LOAD CMSIS/DSP/BasicMathFunctions/arm_abs_q31.o
LOAD CMSIS/DSP/BasicMathFunctions/arm_abs_q7.o
LOAD CMSIS/DSP/BasicMathFunctions/arm_add_f32.o
LOAD CMSIS/DSP/BasicMathFunctions/arm_add_q15.o
LOAD CMSIS/DSP/BasicMathFunctions/arm_add_q31.o
LOAD CMSIS/DSP/BasicMathFunctions/arm_add_q7.o
LOAD CMSIS/DSP/BasicMathFunctions/arm_dot_prod_f32.o
LOAD CMSIS/DSP/BasicMathFunctions/arm_dot_prod_q15.o
LOAD CMSIS/DSP/BasicMathFunctions/arm_dot_prod_q31.o
LOAD CMSIS/DSP/BasicMathFunctions/arm_dot_prod_q7.o
LOAD CMSIS/DSP/BasicMathFunctions/arm_mult_f32.o
LOAD CMSIS/DSP/BasicMathFunctions/arm_mult_q15.o
LOAD CMSIS/DSP/BasicMathFunctions/arm_mult_q31.o
LOAD CMSIS/DSP/BasicMathFunctions/arm_mult_q7.o
LOAD CMSIS/DSP/BasicMathFunctions/arm_negate_f32.o
LOAD CMSIS/DSP/BasicMathFunctions/arm_negate_q15.o
LOAD CMSIS/DSP/BasicMathFunctions/arm_negate_q31.o
LOAD CMSIS/DSP/BasicMathFunctions/arm_negate_q7.o
LOAD CMSIS/DSP/BasicMathFunctions/arm_offset_f32.o
LOAD CMSIS/DSP/BasicMathFunctions/arm_offset_q15.o
LOAD CMSIS/DSP/BasicMathFunctions/arm_offset_q31.o
LOAD CMSIS/DSP/BasicMathFunctions/arm_offset_q7.o
LOAD CMSIS/DSP/BasicMathFunctions/arm_scale_f32.o
LOAD CMSIS/DSP/BasicMathFunctions/arm_scale_q15.o
LOAD CMSIS/DSP/BasicMathFunctions/arm_scale_q31.o
LOAD CMSIS/DSP/BasicMathFunctions/arm_scale_q7.o
LOAD CMSIS/DSP/BasicMathFunctions/arm_shift_q15.o
LOAD CMSIS/DSP/BasicMathFunctions/arm_shift_q31.o
LOAD CMSIS/DSP/BasicMathFunctions/arm_shift_q7.o
LOAD CMSIS/DSP/BasicMathFunctions/arm_sub_f32.o
LOAD CMSIS/DSP/BasicMathFunctions/arm_sub_q15.o
LOAD CMSIS/DSP/BasicMathFunctions/arm_sub_q31.o
LOAD CMSIS/DSP/BasicMathFunctions/arm_sub_q7.o
LOAD CMSIS/DSP/CommonTables/arm_common_tables.o
LOAD CMSIS/DSP/CommonTables/arm_const_structs.o
LOAD CMSIS/DSP/ComplexMathFunctions/arm_cmplx_conj_f32.o
LOAD CMSIS/DSP/ComplexMathFunctions/arm_cmplx_conj_q15.o
LOAD CMSIS/DSP/ComplexMathFunctions/arm_cmplx_conj_q31.o
LOAD CMSIS/DSP/ComplexMathFunctions/arm_cmplx_dot_prod_f32.o
LOAD CMSIS/DSP/ComplexMathFunctions/arm_cmplx_dot_prod_q15.o
LOAD CMSIS/DSP/ComplexMathFunctions/arm_cmplx_dot_prod_q31.o
LOAD CMSIS/DSP/ComplexMathFunctions/arm_cmplx_mag_f32.o
LOAD CMSIS/DSP/ComplexMathFunctions/arm_cmplx_mag_q15.o
LOAD CMSIS/DSP/ComplexMathFunctions/arm_cmplx_mag_q31.o
LOAD CMSIS/DSP/ComplexMathFunctions/arm_cmplx_mag_squared_f32.o
LOAD CMSIS/DSP/ComplexMathFunctions/arm_cmplx_mag_squared_q15.o
LOAD CMSIS/DSP/ComplexMathFunctions/arm_cmplx_mag_squared_q31.o
LOAD CMSIS/DSP/ComplexMathFunctions/arm_cmplx_mult_cmplx_f32.o
LOAD CMSIS/DSP/ComplexMathFunctions/arm_cmplx_mult_cmplx_q15.o
LOAD CMSIS/DSP/ComplexMathFunctions/arm_cmplx_mult_cmplx_q31.o
LOAD CMSIS/DSP/ComplexMathFunctions/arm_cmplx_mult_real_f32.o
LOAD CMSIS/DSP/ComplexMathFunctions/arm_cmplx_mult_real_q15.o
LOAD CMSIS/DSP/ComplexMathFunctions/arm_cmplx_mult_real_q31.o
LOAD CMSIS/DSP/ControllerFunctions/arm_pid_init_f32.o
LOAD CMSIS/DSP/ControllerFunctions/arm_pid_init_q15.o
LOAD CMSIS/DSP/ControllerFunctions/arm_pid_init_q31.o
LOAD CMSIS/DSP/ControllerFunctions/arm_pid_reset_f32.o
LOAD CMSIS/DSP/ControllerFunctions/arm_pid_reset_q15.o
LOAD CMSIS/DSP/ControllerFunctions/arm_pid_reset_q31.o
LOAD CMSIS/DSP/ControllerFunctions/arm_sin_cos_f32.o
LOAD CMSIS/DSP/ControllerFunctions/arm_sin_cos_q31.o
LOAD CMSIS/DSP/FastMathFunctions/arm_cos_f32.o
LOAD CMSIS/DSP/FastMathFunctions/arm_cos_q15.o
LOAD CMSIS/DSP/FastMathFunctions/arm_cos_q31.o
LOAD CMSIS/DSP/FastMathFunctions/arm_sin_f32.o
LOAD CMSIS/DSP/FastMathFunctions/arm_sin_q15.o
LOAD CMSIS/DSP/FastMathFunctions/arm_sin_q31.o
LOAD CMSIS/DSP/FastMathFunctions/arm_sqrt_q15.o
LOAD CMSIS/DSP/FastMathFunctions/arm_sqrt_q31.o
LOAD CMSIS/DSP/FilteringFunctions/arm_biquad_cascade_df1_32x64_init_q31.o
LOAD CMSIS/DSP/FilteringFunctions/arm_biquad_cascade_df1_32x64_q31.o
LOAD CMSIS/DSP/FilteringFunctions/arm_biquad_cascade_df1_f32.o
LOAD CMSIS/DSP/FilteringFunctions/arm_biquad_cascade_df1_fast_q15.o
LOAD CMSIS/DSP/FilteringFunctions/arm_biquad_cascade_df1_fast_q31.o
LOAD CMSIS/DSP/FilteringFunctions/arm_biquad_cascade_df1_init_f32.o
LOAD CMSIS/DSP/FilteringFunctions/arm_biquad_cascade_df1_init_q15.o
LOAD CMSIS/DSP/FilteringFunctions/arm_biquad_cascade_df1_init_q31.o
LOAD CMSIS/DSP/FilteringFunctions/arm_biquad_cascade_df1_q15.o
LOAD CMSIS/DSP/FilteringFunctions/arm_biquad_cascade_df1_q31.o
LOAD CMSIS/DSP/FilteringFunctions/arm_biquad_cascade_df2T_f32.o
LOAD CMSIS/DSP/FilteringFunctions/arm_biquad_cascade_df2T_f64.o
LOAD CMSIS/DSP/FilteringFunctions/arm_biquad_cascade_df2T_init_f32.o
LOAD CMSIS/DSP/FilteringFunctions/arm_biquad_cascade_df2T_init_f64.o
LOAD CMSIS/DSP/FilteringFunctions/arm_biquad_cascade_stereo_df2T_f32.o
LOAD CMSIS/DSP/FilteringFunctions/arm_biquad_cascade_stereo_df2T_init_f32.o
LOAD CMSIS/DSP/FilteringFunctions/arm_conv_f32.o
LOAD CMSIS/DSP/FilteringFunctions/arm_conv_fast_opt_q15.o
LOAD CMSIS/DSP/FilteringFunctions/arm_conv_fast_q15.o
LOAD CMSIS/DSP/FilteringFunctions/arm_conv_fast_q31.o
LOAD CMSIS/DSP/FilteringFunctions/arm_conv_opt_q15.o
LOAD CMSIS/DSP/FilteringFunctions/arm_conv_opt_q7.o
LOAD CMSIS/DSP/FilteringFunctions/arm_conv_partial_f32.o
LOAD CMSIS/DSP/FilteringFunctions/arm_conv_partial_fast_opt_q15.o
LOAD CMSIS/DSP/FilteringFunctions/arm_conv_partial_fast_q15.o
LOAD CMSIS/DSP/FilteringFunctions/arm_conv_partial_fast_q31.o
LOAD CMSIS/DSP/FilteringFunctions/arm_conv_partial_opt_q15.o
LOAD CMSIS/DSP/FilteringFunctions/arm_conv_partial_opt_q7.o
LOAD CMSIS/DSP/FilteringFunctions/arm_conv_partial_q15.o
LOAD CMSIS/DSP/FilteringFunctions/arm_conv_partial_q31.o
LOAD CMSIS/DSP/FilteringFunctions/arm_conv_partial_q7.o
LOAD CMSIS/DSP/FilteringFunctions/arm_conv_q15.o
LOAD CMSIS/DSP/FilteringFunctions/arm_conv_q31.o
LOAD CMSIS/DSP/FilteringFunctions/arm_conv_q7.o
LOAD CMSIS/DSP/FilteringFunctions/arm_correlate_f32.o
LOAD CMSIS/DSP/FilteringFunctions/arm_correlate_fast_opt_q15.o
LOAD CMSIS/DSP/FilteringFunctions/arm_correlate_fast_q15.o
LOAD CMSIS/DSP/FilteringFunctions/arm_correlate_fast_q31.o
LOAD CMSIS/DSP/FilteringFunctions/arm_correlate_opt_q15.o
LOAD CMSIS/DSP/FilteringFunctions/arm_correlate_opt_q7.o
LOAD CMSIS/DSP/FilteringFunctions/arm_correlate_q15.o
LOAD CMSIS/DSP/FilteringFunctions/arm_correlate_q31.o
LOAD CMSIS/DSP/FilteringFunctions/arm_correlate_q7.o
LOAD CMSIS/DSP/FilteringFunctions/arm_fir_decimate_f32.o
LOAD CMSIS/DSP/FilteringFunctions/arm_fir_decimate_fast_q15.o
LOAD CMSIS/DSP/FilteringFunctions/arm_fir_decimate_fast_q31.o
LOAD CMSIS/DSP/FilteringFunctions/arm_fir_decimate_init_f32.o
LOAD CMSIS/DSP/FilteringFunctions/arm_fir_decimate_init_q15.o
LOAD CMSIS/DSP/FilteringFunctions/arm_fir_decimate_init_q31.o
LOAD CMSIS/DSP/FilteringFunctions/arm_fir_decimate_q15.o
LOAD CMSIS/DSP/FilteringFunctions/arm_fir_decimate_q31.o
LOAD CMSIS/DSP/FilteringFunctions/arm_fir_f32.o
LOAD CMSIS/DSP/FilteringFunctions/arm_fir_fast_q15.o
LOAD CMSIS/DSP/FilteringFunctions/arm_fir_fast_q31.o
LOAD CMSIS/DSP/FilteringFunctions/arm_fir_init_f32.o
LOAD CMSIS/DSP/FilteringFunctions/arm_fir_init_q15.o
LOAD CMSIS/DSP/FilteringFunctions/arm_fir_init_q31.o
LOAD CMSIS/DSP/FilteringFunctions/arm_fir_init_q7.o
LOAD CMSIS/DSP/FilteringFunctions/arm_fir_interpolate_f32.o
LOAD CMSIS/DSP/FilteringFunctions/arm_fir_interpolate_init_f32.o
LOAD CMSIS/DSP/FilteringFunctions/arm_fir_interpolate_init_q15.o
LOAD CMSIS/DSP/FilteringFunctions/arm_fir_interpolate_init_q31.o
LOAD CMSIS/DSP/FilteringFunctions/arm_fir_interpolate_q15.o
LOAD CMSIS/DSP/FilteringFunctions/arm_fir_interpolate_q31.o
LOAD CMSIS/DSP/FilteringFunctions/arm_fir_lattice_f32.o
LOAD CMSIS/DSP/FilteringFunctions/arm_fir_lattice_init_f32.o
LOAD CMSIS/DSP/FilteringFunctions/arm_fir_lattice_init_q15.o
LOAD CMSIS/DSP/FilteringFunctions/arm_fir_lattice_init_q31.o
LOAD CMSIS/DSP/FilteringFunctions/arm_fir_lattice_q15.o
LOAD CMSIS/DSP/FilteringFunctions/arm_fir_lattice_q31.o
LOAD CMSIS/DSP/FilteringFunctions/arm_fir_q15.o
LOAD CMSIS/DSP/FilteringFunctions/arm_fir_q31.o
LOAD CMSIS/DSP/FilteringFunctions/arm_fir_q7.o
LOAD CMSIS/DSP/FilteringFunctions/arm_fir_sparse_f32.o
LOAD CMSIS/DSP/FilteringFunctions/arm_fir_sparse_init_f32.o
LOAD CMSIS/DSP/FilteringFunctions/arm_fir_sparse_init_q15.o
LOAD CMSIS/DSP/FilteringFunctions/arm_fir_sparse_init_q31.o
LOAD CMSIS/DSP/FilteringFunctions/arm_fir_sparse_init_q7.o
LOAD CMSIS/DSP/FilteringFunctions/arm_fir_sparse_q15.o
LOAD CMSIS/DSP/FilteringFunctions/arm_fir_sparse_q31.o
LOAD CMSIS/DSP/FilteringFunctions/arm_fir_sparse_q7.o
LOAD CMSIS/DSP/FilteringFunctions/arm_iir_lattice_f32.o
LOAD CMSIS/DSP/FilteringFunctions/arm_iir_lattice_init_f32.o
LOAD CMSIS/DSP/FilteringFunctions/arm_iir_lattice_init_q15.o
LOAD CMSIS/DSP/FilteringFunctions/arm_iir_lattice_init_q31.o
LOAD CMSIS/DSP/FilteringFunctions/arm_iir_lattice_q15.o
LOAD CMSIS/DSP/FilteringFunctions/arm_iir_lattice_q31.o
LOAD CMSIS/DSP/FilteringFunctions/arm_lms_f32.o
LOAD CMSIS/DSP/FilteringFunctions/arm_lms_init_f32.o
LOAD CMSIS/DSP/FilteringFunctions/arm_lms_init_q15.o
LOAD CMSIS/DSP/FilteringFunctions/arm_lms_init_q31.o
LOAD CMSIS/DSP/FilteringFunctions/arm_lms_norm_f32.o
LOAD CMSIS/DSP/FilteringFunctions/arm_lms_norm_init_f32.o
LOAD CMSIS/DSP/FilteringFunctions/arm_lms_norm_init_q15.o
LOAD CMSIS/DSP/FilteringFunctions/arm_lms_norm_init_q31.o
LOAD CMSIS/DSP/FilteringFunctions/arm_lms_norm_q15.o
LOAD CMSIS/DSP/FilteringFunctions/arm_lms_norm_q31.o
LOAD CMSIS/DSP/FilteringFunctions/arm_lms_q15.o
LOAD CMSIS/DSP/FilteringFunctions/arm_lms_q31.o
LOAD CMSIS/DSP/MatrixFunctions/arm_mat_add_f32.o
LOAD CMSIS/DSP/MatrixFunctions/arm_mat_add_q15.o
LOAD CMSIS/DSP/MatrixFunctions/arm_mat_add_q31.o
LOAD CMSIS/DSP/MatrixFunctions/arm_mat_cmplx_mult_f32.o
LOAD CMSIS/DSP/MatrixFunctions/arm_mat_cmplx_mult_q15.o
LOAD CMSIS/DSP/MatrixFunctions/arm_mat_cmplx_mult_q31.o
LOAD CMSIS/DSP/MatrixFunctions/arm_mat_init_f32.o
LOAD CMSIS/DSP/MatrixFunctions/arm_mat_init_q15.o
LOAD CMSIS/DSP/MatrixFunctions/arm_mat_init_q31.o
LOAD CMSIS/DSP/MatrixFunctions/arm_mat_inverse_f32.o
LOAD CMSIS/DSP/MatrixFunctions/arm_mat_inverse_f64.o
LOAD CMSIS/DSP/MatrixFunctions/arm_mat_mult_f32.o
LOAD CMSIS/DSP/MatrixFunctions/arm_mat_mult_fast_q15.o
LOAD CMSIS/DSP/MatrixFunctions/arm_mat_mult_fast_q31.o
LOAD CMSIS/DSP/MatrixFunctions/arm_mat_mult_q15.o
LOAD CMSIS/DSP/MatrixFunctions/arm_mat_mult_q31.o
LOAD CMSIS/DSP/MatrixFunctions/arm_mat_scale_f32.o
LOAD CMSIS/DSP/MatrixFunctions/arm_mat_scale_q15.o
LOAD CMSIS/DSP/MatrixFunctions/arm_mat_scale_q31.o
LOAD CMSIS/DSP/MatrixFunctions/arm_mat_sub_f32.o
LOAD CMSIS/DSP/MatrixFunctions/arm_mat_sub_q15.o
LOAD CMSIS/DSP/MatrixFunctions/arm_mat_sub_q31.o
LOAD CMSIS/DSP/MatrixFunctions/arm_mat_trans_f32.o
LOAD CMSIS/DSP/MatrixFunctions/arm_mat_trans_q15.o
LOAD CMSIS/DSP/MatrixFunctions/arm_mat_trans_q31.o
LOAD CMSIS/DSP/StatisticsFunctions/arm_max_f32.o
LOAD CMSIS/DSP/StatisticsFunctions/arm_max_q15.o
LOAD CMSIS/DSP/StatisticsFunctions/arm_max_q31.o
LOAD CMSIS/DSP/StatisticsFunctions/arm_max_q7.o
LOAD CMSIS/DSP/StatisticsFunctions/arm_mean_f32.o
LOAD CMSIS/DSP/StatisticsFunctions/arm_mean_q15.o
LOAD CMSIS/DSP/StatisticsFunctions/arm_mean_q31.o
LOAD CMSIS/DSP/StatisticsFunctions/arm_mean_q7.o
LOAD CMSIS/DSP/StatisticsFunctions/arm_min_f32.o
LOAD CMSIS/DSP/StatisticsFunctions/arm_min_q15.o
LOAD CMSIS/DSP/StatisticsFunctions/arm_min_q31.o
LOAD CMSIS/DSP/StatisticsFunctions/arm_min_q7.o
LOAD CMSIS/DSP/StatisticsFunctions/arm_power_f32.o
LOAD CMSIS/DSP/StatisticsFunctions/arm_power_q15.o
LOAD CMSIS/DSP/StatisticsFunctions/arm_power_q31.o
LOAD CMSIS/DSP/StatisticsFunctions/arm_power_q7.o
LOAD CMSIS/DSP/StatisticsFunctions/arm_rms_f32.o
LOAD CMSIS/DSP/StatisticsFunctions/arm_rms_q15.o
LOAD CMSIS/DSP/StatisticsFunctions/arm_rms_q31.o
LOAD CMSIS/DSP/StatisticsFunctions/arm_std_f32.o
LOAD CMSIS/DSP/StatisticsFunctions/arm_std_q15.o
LOAD CMSIS/DSP/StatisticsFunctions/arm_std_q31.o
LOAD CMSIS/DSP/StatisticsFunctions/arm_var_f32.o
LOAD CMSIS/DSP/StatisticsFunctions/arm_var_q15.o
LOAD CMSIS/DSP/StatisticsFunctions/arm_var_q31.o
LOAD CMSIS/DSP/SupportFunctions/arm_copy_f32.o
LOAD CMSIS/DSP/SupportFunctions/arm_copy_q15.o
LOAD CMSIS/DSP/SupportFunctions/arm_copy_q31.o
LOAD CMSIS/DSP/SupportFunctions/arm_copy_q7.o
LOAD CMSIS/DSP/SupportFunctions/arm_fill_f32.o
LOAD CMSIS/DSP/SupportFunctions/arm_fill_q15.o
LOAD CMSIS/DSP/SupportFunctions/arm_fill_q31.o
LOAD CMSIS/DSP/SupportFunctions/arm_fill_q7.o
LOAD CMSIS/DSP/SupportFunctions/arm_float_to_q15.o
LOAD CMSIS/DSP/SupportFunctions/arm_float_to_q31.o
LOAD CMSIS/DSP/SupportFunctions/arm_float_to_q7.o
LOAD CMSIS/DSP/SupportFunctions/arm_q15_to_float.o
LOAD CMSIS/DSP/SupportFunctions/arm_q15_to_q31.o
LOAD CMSIS/DSP/SupportFunctions/arm_q15_to_q7.o
LOAD CMSIS/DSP/SupportFunctions/arm_q31_to_float.o
LOAD CMSIS/DSP/SupportFunctions/arm_q31_to_q15.o
LOAD CMSIS/DSP/SupportFunctions/arm_q31_to_q7.o
LOAD CMSIS/DSP/SupportFunctions/arm_q7_to_float.o
LOAD CMSIS/DSP/SupportFunctions/arm_q7_to_q15.o
LOAD CMSIS/DSP/SupportFunctions/arm_q7_to_q31.o
LOAD CMSIS/DSP/TransformFunctions/arm_bitreversal.o
LOAD CMSIS/DSP/TransformFunctions/arm_bitreversal2.o
LOAD CMSIS/DSP/TransformFunctions/arm_cfft_f32.o
LOAD CMSIS/DSP/TransformFunctions/arm_cfft_q15.o
LOAD CMSIS/DSP/TransformFunctions/arm_cfft_q31.o
LOAD CMSIS/DSP/TransformFunctions/arm_cfft_radix2_f32.o
LOAD CMSIS/DSP/TransformFunctions/arm_cfft_radix2_init_f32.o
LOAD CMSIS/DSP/TransformFunctions/arm_cfft_radix2_init_q15.o
LOAD CMSIS/DSP/TransformFunctions/arm_cfft_radix2_init_q31.o
LOAD CMSIS/DSP/TransformFunctions/arm_cfft_radix2_q15.o
LOAD CMSIS/DSP/TransformFunctions/arm_cfft_radix2_q31.o
LOAD CMSIS/DSP/TransformFunctions/arm_cfft_radix4_f32.o
LOAD CMSIS/DSP/TransformFunctions/arm_cfft_radix4_init_f32.o
LOAD CMSIS/DSP/TransformFunctions/arm_cfft_radix4_init_q15.o
LOAD CMSIS/DSP/TransformFunctions/arm_cfft_radix4_init_q31.o
LOAD CMSIS/DSP/TransformFunctions/arm_cfft_radix4_q15.o
LOAD CMSIS/DSP/TransformFunctions/arm_cfft_radix4_q31.o
LOAD CMSIS/DSP/TransformFunctions/arm_cfft_radix8_f32.o
LOAD CMSIS/DSP/TransformFunctions/arm_dct4_f32.o
LOAD CMSIS/DSP/TransformFunctions/arm_dct4_init_f32.o
LOAD CMSIS/DSP/TransformFunctions/arm_dct4_init_q15.o
LOAD CMSIS/DSP/TransformFunctions/arm_dct4_init_q31.o
LOAD CMSIS/DSP/TransformFunctions/arm_dct4_q15.o
LOAD CMSIS/DSP/TransformFunctions/arm_dct4_q31.o
LOAD CMSIS/DSP/TransformFunctions/arm_rfft_f32.o
LOAD CMSIS/DSP/TransformFunctions/arm_rfft_fast_f32.o
LOAD CMSIS/DSP/TransformFunctions/arm_rfft_fast_init_f32.o
LOAD CMSIS/DSP/TransformFunctions/arm_rfft_init_f32.o
LOAD CMSIS/DSP/TransformFunctions/arm_rfft_init_q15.o
LOAD CMSIS/DSP/TransformFunctions/arm_rfft_init_q31.o
LOAD CMSIS/DSP/TransformFunctions/arm_rfft_q15.o
LOAD CMSIS/DSP/TransformFunctions/arm_rfft_q31.o
LOAD CMSIS/NN/ActivationFunctions/arm_nn_activations_q15.o
LOAD CMSIS/NN/ActivationFunctions/arm_nn_activations_q7.o
LOAD CMSIS/NN/ActivationFunctions/arm_relu_q15.o
LOAD CMSIS/NN/ActivationFunctions/arm_relu_q7.o
LOAD CMSIS/NN/ConvolutionFunctions/arm_convolve_1x1_HWC_q7_fast_nonsquare.o
LOAD CMSIS/NN/ConvolutionFunctions/arm_convolve_HWC_q15_basic.o
LOAD CMSIS/NN/ConvolutionFunctions/arm_convolve_HWC_q15_fast.o
LOAD CMSIS/NN/ConvolutionFunctions/arm_convolve_HWC_q15_fast_nonsquare.o
LOAD CMSIS/NN/ConvolutionFunctions/arm_convolve_HWC_q7_RGB.o
LOAD CMSIS/NN/ConvolutionFunctions/arm_convolve_HWC_q7_basic.o
LOAD CMSIS/NN/ConvolutionFunctions/arm_convolve_HWC_q7_basic_nonsquare.o
LOAD CMSIS/NN/ConvolutionFunctions/arm_convolve_HWC_q7_fast.o
LOAD CMSIS/NN/ConvolutionFunctions/arm_convolve_HWC_q7_fast_nonsquare.o
LOAD CMSIS/NN/ConvolutionFunctions/arm_depthwise_separable_conv_HWC_q7.o
LOAD CMSIS/NN/ConvolutionFunctions/arm_depthwise_separable_conv_HWC_q7_nonsquare.o
LOAD CMSIS/NN/ConvolutionFunctions/arm_nn_mat_mult_kernel_q7_q15.o
LOAD CMSIS/NN/ConvolutionFunctions/arm_nn_mat_mult_kernel_q7_q15_reordered.o
LOAD CMSIS/NN/FullyConnectedFunctions/arm_fully_connected_mat_q7_vec_q15.o
LOAD CMSIS/NN/FullyConnectedFunctions/arm_fully_connected_mat_q7_vec_q15_opt.o
LOAD CMSIS/NN/FullyConnectedFunctions/arm_fully_connected_q15.o
LOAD CMSIS/NN/FullyConnectedFunctions/arm_fully_connected_q15_opt.o
LOAD CMSIS/NN/FullyConnectedFunctions/arm_fully_connected_q7.o
LOAD CMSIS/NN/FullyConnectedFunctions/arm_fully_connected_q7_opt.o
LOAD CMSIS/NN/NNSupportFunctions/arm_nn_mult_q15.o
LOAD CMSIS/NN/NNSupportFunctions/arm_nn_mult_q7.o
LOAD CMSIS/NN/NNSupportFunctions/arm_nntables.o
LOAD CMSIS/NN/NNSupportFunctions/arm_q7_to_q15_no_shift.o
LOAD CMSIS/NN/NNSupportFunctions/arm_q7_to_q15_reordered_no_shift.o
LOAD CMSIS/NN/PoolingFunctions/arm_pool_q7_HWC.o
LOAD CMSIS/NN/SoftmaxFunctions/arm_softmax_q15.o
LOAD CMSIS/NN/SoftmaxFunctions/arm_softmax_q7.o
LOAD Drivers/BSP/Components/HTS221_Driver.o
LOAD Drivers/BSP/Components/HTS221_Driver_HL.o
LOAD Drivers/BSP/Components/LPS22HB_Driver.o
LOAD Drivers/BSP/Components/LPS22HB_Driver_HL.o
LOAD Drivers/BSP/Components/LSM303AGR_ACC_driver.o
LOAD Drivers/BSP/Components/LSM303AGR_ACC_driver_HL.o
LOAD Drivers/BSP/Components/LSM303AGR_MAG_driver.o
LOAD Drivers/BSP/Components/LSM303AGR_MAG_driver_HL.o
LOAD Drivers/BSP/Components/LSM6DSM_ACC_GYRO_driver.o
LOAD Drivers/BSP/Components/LSM6DSM_ACC_GYRO_driver_HL.o
LOAD Drivers/BSP/Components/STC3115_Driver.o
LOAD Drivers/BSP/SensorTile/SensorTile.o
LOAD Drivers/BSP/SensorTile/SensorTile_BlueNRG.o
LOAD Drivers/BSP/SensorTile/SensorTile_accelero.o
LOAD Drivers/BSP/SensorTile/SensorTile_gg.o
LOAD Drivers/BSP/SensorTile/SensorTile_gyro.o
LOAD Drivers/BSP/SensorTile/SensorTile_humidity.o
LOAD Drivers/BSP/SensorTile/SensorTile_magneto.o
LOAD Drivers/BSP/SensorTile/SensorTile_pressure.o
LOAD Drivers/BSP/SensorTile/SensorTile_sd.o
LOAD Drivers/BSP/SensorTile/SensorTile_temperature.o
LOAD Drivers/CMSIS/system_stm32l4xx.o
LOAD Drivers/STM32L4xx_HAL_Driver/stm32l4xx_hal.o
LOAD Drivers/STM32L4xx_HAL_Driver/stm32l4xx_hal_adc.o
LOAD Drivers/STM32L4xx_HAL_Driver/stm32l4xx_hal_adc_ex.o
LOAD Drivers/STM32L4xx_HAL_Driver/stm32l4xx_hal_cortex.o
LOAD Drivers/STM32L4xx_HAL_Driver/stm32l4xx_hal_crc.o
LOAD Drivers/STM32L4xx_HAL_Driver/stm32l4xx_hal_crc_ex.o
LOAD Drivers/STM32L4xx_HAL_Driver/stm32l4xx_hal_dma.o
LOAD Drivers/STM32L4xx_HAL_Driver/stm32l4xx_hal_flash.o
LOAD Drivers/STM32L4xx_HAL_Driver/stm32l4xx_hal_flash_ex.o
LOAD Drivers/STM32L4xx_HAL_Driver/stm32l4xx_hal_gpio.o
LOAD Drivers/STM32L4xx_HAL_Driver/stm32l4xx_hal_i2c.o
LOAD Drivers/STM32L4xx_HAL_Driver/stm32l4xx_hal_i2c_ex.o
LOAD Drivers/STM32L4xx_HAL_Driver/stm32l4xx_hal_pcd.o
LOAD Drivers/STM32L4xx_HAL_Driver/stm32l4xx_hal_pcd_ex.o
LOAD Drivers/STM32L4xx_HAL_Driver/stm32l4xx_hal_pwr.o
LOAD Drivers/STM32L4xx_HAL_Driver/stm32l4xx_hal_pwr_ex.o
LOAD Drivers/STM32L4xx_HAL_Driver/stm32l4xx_hal_rcc.o
LOAD Drivers/STM32L4xx_HAL_Driver/stm32l4xx_hal_rcc_ex.o
LOAD Drivers/STM32L4xx_HAL_Driver/stm32l4xx_hal_rtc.o
LOAD Drivers/STM32L4xx_HAL_Driver/stm32l4xx_hal_rtc_ex.o
LOAD Drivers/STM32L4xx_HAL_Driver/stm32l4xx_hal_spi.o
LOAD Drivers/STM32L4xx_HAL_Driver/stm32l4xx_hal_spi_ex.o
LOAD Drivers/STM32L4xx_HAL_Driver/stm32l4xx_hal_tim.o
LOAD Drivers/STM32L4xx_HAL_Driver/stm32l4xx_hal_tim_ex.o
LOAD Drivers/STM32L4xx_HAL_Driver/stm32l4xx_hal_uart.o
LOAD Drivers/STM32L4xx_HAL_Driver/stm32l4xx_hal_uart_ex.o
LOAD Drivers/STM32L4xx_HAL_Driver/stm32l4xx_ll_usb.o
LOAD Example/SW4STM32/startup_stm32l476xx.o
LOAD MLKWS/KWS/KWS_DNN/kws_dnn.o
LOAD MLKWS/KWS/KWS_DS_CNN/kws_ds_cnn.o
LOAD MLKWS/KWS/kws.o
LOAD MLKWS/KWS_F746NG/kws_f746ng.o
LOAD MLKWS/MFCC/mfcc.o
LOAD MLKWS/NN/DNN/dnn.o
LOAD MLKWS/NN/DS_CNN/ds_cnn.o
LOAD MLKWS/NN/nn.o
LOAD MLKWS/local_NN/arm_avepool_q7_HWC_nonsquare.o
LOAD Middlewares/FatFs/Core/diskio.o
LOAD Middlewares/FatFs/Core/ff.o
LOAD Middlewares/FatFs/Core/ff_gen_drv.o
LOAD Middlewares/FatFs/Drivers/sd_diskio.o
LOAD Middlewares/FatFs/Options/syscall.o
LOAD Middlewares/FatFs/Options/unicode.o
LOAD Middlewares/FreeRTOS/CMSIS_RTOS/cmsis_os.o
LOAD Middlewares/FreeRTOS/list.o
LOAD Middlewares/FreeRTOS/queue.o
LOAD Middlewares/FreeRTOS/tasks.o
LOAD Middlewares/FreeRTOS/timers.o
LOAD Middlewares/FreeRTOS/portable/heap_4.o
LOAD Middlewares/FreeRTOS/portable/port.o
LOAD Middlewares/STM32_BlueNRG/HCI/Controller/bluenrg_gap_aci.o
LOAD Middlewares/STM32_BlueNRG/HCI/Controller/bluenrg_gatt_aci.o
LOAD Middlewares/STM32_BlueNRG/HCI/Controller/bluenrg_hal_aci.o
LOAD Middlewares/STM32_BlueNRG/HCI/Controller/bluenrg_l2cap_aci.o
LOAD Middlewares/STM32_BlueNRG/HCI/Controller/bluenrg_utils.o
LOAD Middlewares/STM32_BlueNRG/HCI/hci.o
LOAD Middlewares/STM32_BlueNRG/HCI/hci_le.o
LOAD Middlewares/STM32_BlueNRG/Interface/bluenrg_itf.o
LOAD Middlewares/STM32_BlueNRG/Utils/ble_list.o
LOAD Middlewares/STM32_BlueNRG/Utils/gp_timer.o
LOAD Middlewares/STM32_BlueNRG/Utils/osal.o
LOAD Middlewares/STM32_USBD_Library/Class/CDC/usbd_cdc.o
LOAD Middlewares/STM32_USBD_Library/Core/usbd_core.o
LOAD Middlewares/STM32_USBD_Library/Core/usbd_ctlreq.o
LOAD Middlewares/STM32_USBD_Library/Core/usbd_ioreq.o
LOAD c:/ac6/systemworkbench/plugins/fr.ac6.mcu.externaltools.arm-none.win32_1.17.0.201812190825/tools/compiler/bin/../lib/gcc/arm-none-eabi/7.3.1/../../../../arm-none-eabi/lib/thumb/v7e-m/fpv4-sp/hard\libstdc++_nano.a
LOAD c:/ac6/systemworkbench/plugins/fr.ac6.mcu.externaltools.arm-none.win32_1.17.0.201812190825/tools/compiler/bin/../lib/gcc/arm-none-eabi/7.3.1/../../../../arm-none-eabi/lib/thumb/v7e-m/fpv4-sp/hard\libm.a
START GROUP
LOAD c:/ac6/systemworkbench/plugins/fr.ac6.mcu.externaltools.arm-none.win32_1.17.0.201812190825/tools/compiler/bin/../lib/gcc/arm-none-eabi/7.3.1/thumb/v7e-m/fpv4-sp/hard\libgcc.a
LOAD c:/ac6/systemworkbench/plugins/fr.ac6.mcu.externaltools.arm-none.win32_1.17.0.201812190825/tools/compiler/bin/../lib/gcc/arm-none-eabi/7.3.1/../../../../arm-none-eabi/lib/thumb/v7e-m/fpv4-sp/hard\libc_nano.a
END GROUP
START GROUP
LOAD c:/ac6/systemworkbench/plugins/fr.ac6.mcu.externaltools.arm-none.win32_1.17.0.201812190825/tools/compiler/bin/../lib/gcc/arm-none-eabi/7.3.1/thumb/v7e-m/fpv4-sp/hard\libgcc.a
LOAD c:/ac6/systemworkbench/plugins/fr.ac6.mcu.externaltools.arm-none.win32_1.17.0.201812190825/tools/compiler/bin/../lib/gcc/arm-none-eabi/7.3.1/../../../../arm-none-eabi/lib/thumb/v7e-m/fpv4-sp/hard\libc_nano.a
LOAD c:/ac6/systemworkbench/plugins/fr.ac6.mcu.externaltools.arm-none.win32_1.17.0.201812190825/tools/compiler/bin/../lib/gcc/arm-none-eabi/7.3.1/../../../../arm-none-eabi/lib/thumb/v7e-m/fpv4-sp/hard\libnosys.a
END GROUP
START GROUP
LOAD c:/ac6/systemworkbench/plugins/fr.ac6.mcu.externaltools.arm-none.win32_1.17.0.201812190825/tools/compiler/bin/../lib/gcc/arm-none-eabi/7.3.1/thumb/v7e-m/fpv4-sp/hard\libgcc.a
LOAD c:/ac6/systemworkbench/plugins/fr.ac6.mcu.externaltools.arm-none.win32_1.17.0.201812190825/tools/compiler/bin/../lib/gcc/arm-none-eabi/7.3.1/../../../../arm-none-eabi/lib/thumb/v7e-m/fpv4-sp/hard\libc_nano.a
LOAD c:/ac6/systemworkbench/plugins/fr.ac6.mcu.externaltools.arm-none.win32_1.17.0.201812190825/tools/compiler/bin/../lib/gcc/arm-none-eabi/7.3.1/../../../../arm-none-eabi/lib/thumb/v7e-m/fpv4-sp/hard\libnosys.a
END GROUP
LOAD c:/ac6/systemworkbench/plugins/fr.ac6.mcu.externaltools.arm-none.win32_1.17.0.201812190825/tools/compiler/bin/../lib/gcc/arm-none-eabi/7.3.1/thumb/v7e-m/fpv4-sp/hard/crtend.o
LOAD c:/ac6/systemworkbench/plugins/fr.ac6.mcu.externaltools.arm-none.win32_1.17.0.201812190825/tools/compiler/bin/../lib/gcc/arm-none-eabi/7.3.1/thumb/v7e-m/fpv4-sp/hard/crtn.o
                0x20018000                _estack = 0x20018000
                0x00000200                _Min_Heap_Size = 0x200
                0x00000400                _Min_Stack_Size = 0x400

.isr_vector     0x08000000      0x188
                0x08000000                . = ALIGN (0x8)
 *(.isr_vector)
 .isr_vector    0x08000000      0x188 Example/SW4STM32/startup_stm32l476xx.o
                0x08000000                g_pfnVectors
                0x08000188                . = ALIGN (0x8)

.text           0x08000190    0x11110
                0x08000190                . = ALIGN (0x8)
 *(.text)
 .text          0x08000190       0x40 c:/ac6/systemworkbench/plugins/fr.ac6.mcu.externaltools.arm-none.win32_1.17.0.201812190825/tools/compiler/bin/../lib/gcc/arm-none-eabi/7.3.1/thumb/v7e-m/fpv4-sp/hard/crtbegin.o
 .text          0x080001d0      0x378 c:/ac6/systemworkbench/plugins/fr.ac6.mcu.externaltools.arm-none.win32_1.17.0.201812190825/tools/compiler/bin/../lib/gcc/arm-none-eabi/7.3.1/thumb/v7e-m/fpv4-sp/hard\libgcc.a(_arm_addsubdf3.o)
                0x080001d0                __aeabi_drsub
                0x080001d8                __aeabi_dsub
                0x080001d8                __subdf3
                0x080001dc                __aeabi_dadd
                0x080001dc                __adddf3
                0x08000454                __floatunsidf
                0x08000454                __aeabi_ui2d
                0x08000474                __floatsidf
                0x08000474                __aeabi_i2d
                0x08000498                __aeabi_f2d
                0x08000498                __extendsfdf2
                0x080004dc                __floatundidf
                0x080004dc                __aeabi_ul2d
                0x080004ec                __floatdidf
                0x080004ec                __aeabi_l2d
 .text          0x08000548      0x424 c:/ac6/systemworkbench/plugins/fr.ac6.mcu.externaltools.arm-none.win32_1.17.0.201812190825/tools/compiler/bin/../lib/gcc/arm-none-eabi/7.3.1/thumb/v7e-m/fpv4-sp/hard\libgcc.a(_arm_muldivdf3.o)
                0x08000548                __aeabi_dmul
                0x08000548                __muldf3
                0x0800079c                __divdf3
                0x0800079c                __aeabi_ddiv
 .text          0x0800096c      0x110 c:/ac6/systemworkbench/plugins/fr.ac6.mcu.externaltools.arm-none.win32_1.17.0.201812190825/tools/compiler/bin/../lib/gcc/arm-none-eabi/7.3.1/thumb/v7e-m/fpv4-sp/hard\libgcc.a(_arm_cmpdf2.o)
                0x0800096c                __gtdf2
                0x0800096c                __gedf2
                0x08000974                __ltdf2
                0x08000974                __ledf2
                0x0800097c                __nedf2
                0x0800097c                __eqdf2
                0x0800097c                __cmpdf2
                0x080009f8                __aeabi_cdrcmple
                0x08000a08                __aeabi_cdcmpeq
                0x08000a08                __aeabi_cdcmple
                0x08000a18                __aeabi_dcmpeq
                0x08000a2c                __aeabi_dcmplt
                0x08000a40                __aeabi_dcmple
                0x08000a54                __aeabi_dcmpge
                0x08000a68                __aeabi_dcmpgt
 .text          0x08000a7c       0x2c c:/ac6/systemworkbench/plugins/fr.ac6.mcu.externaltools.arm-none.win32_1.17.0.201812190825/tools/compiler/bin/../lib/gcc/arm-none-eabi/7.3.1/thumb/v7e-m/fpv4-sp/hard\libgcc.a(_arm_unorddf2.o)
                0x08000a7c                __unorddf2
                0x08000a7c                __aeabi_dcmpun
 .text          0x08000aa8       0x50 c:/ac6/systemworkbench/plugins/fr.ac6.mcu.externaltools.arm-none.win32_1.17.0.201812190825/tools/compiler/bin/../lib/gcc/arm-none-eabi/7.3.1/thumb/v7e-m/fpv4-sp/hard\libgcc.a(_arm_fixdfsi.o)
                0x08000aa8                __aeabi_d2iz
                0x08000aa8                __fixdfsi
 .text          0x08000af8       0xa0 c:/ac6/systemworkbench/plugins/fr.ac6.mcu.externaltools.arm-none.win32_1.17.0.201812190825/tools/compiler/bin/../lib/gcc/arm-none-eabi/7.3.1/thumb/v7e-m/fpv4-sp/hard\libgcc.a(_aeabi_ldivmod.o)
                0x08000af8                __aeabi_ldivmod
 .text          0x08000b98      0x2cc c:/ac6/systemworkbench/plugins/fr.ac6.mcu.externaltools.arm-none.win32_1.17.0.201812190825/tools/compiler/bin/../lib/gcc/arm-none-eabi/7.3.1/thumb/v7e-m/fpv4-sp/hard\libgcc.a(_udivmoddi4.o)
                0x08000b98                __udivmoddi4
 .text          0x08000e64        0x4 c:/ac6/systemworkbench/plugins/fr.ac6.mcu.externaltools.arm-none.win32_1.17.0.201812190825/tools/compiler/bin/../lib/gcc/arm-none-eabi/7.3.1/thumb/v7e-m/fpv4-sp/hard\libgcc.a(_dvmd_tls.o)
                0x08000e64                __aeabi_idiv0
                0x08000e64                __aeabi_ldiv0
 .text          0x08000e68       0x10 c:/ac6/systemworkbench/plugins/fr.ac6.mcu.externaltools.arm-none.win32_1.17.0.201812190825/tools/compiler/bin/../lib/gcc/arm-none-eabi/7.3.1/../../../../arm-none-eabi/lib/thumb/v7e-m/fpv4-sp/hard\libc_nano.a(lib_a-strlen.o)
                0x08000e68                strlen
 *fill*         0x08000e78        0x8 
 .text          0x08000e80       0xa0 c:/ac6/systemworkbench/plugins/fr.ac6.mcu.externaltools.arm-none.win32_1.17.0.201812190825/tools/compiler/bin/../lib/gcc/arm-none-eabi/7.3.1/../../../../arm-none-eabi/lib/thumb/v7e-m/fpv4-sp/hard\libc_nano.a(lib_a-memchr.o)
                0x08000e80                memchr
 *(.text*)
 .text.InitTargetPlatform
                0x08000f20       0x10 Application/User/TargetPlatform.o
                0x08000f20                InitTargetPlatform
 .text.SystemClock_Config
                0x08000f30       0xd0 Application/User/cube_hal_l4.o
                0x08000f30                SystemClock_Config
 .text._Z20get_timer_0_CallbackPKv
                0x08001000        0xc Application/User/main.o
                0x08001000                get_timer_0_Callback(void const*)
 .text._ZL15send_to_gatewayi
                0x0800100c      0x1b0 Application/User/main.o
 .text._ZL13send_thread_2PKv
                0x080011bc        0x8 Application/User/main.o
 .text._ZL13send_thread_1PKv
                0x080011c4        0x8 Application/User/main.o
 .text._ZL13send_thread_0PKv
                0x080011cc        0x8 Application/User/main.o
 .text._Z21master_timer_CallbackPKv
                0x080011d4       0x28 Application/User/main.o
                0x080011d4                master_timer_Callback(void const*)
 .text._ZL14temp_thresholdi
                0x080011fc       0x50 Application/User/main.o
 .text._ZL14thrsh_thread_2PKv
                0x0800124c        0x8 Application/User/main.o
 .text._ZL14thrsh_thread_1PKv
                0x08001254        0x8 Application/User/main.o
 .text._ZL16read_from_sensori
                0x0800125c       0xa4 Application/User/main.o
 .text._ZL12get_thread_2PKv
                0x08001300        0x8 Application/User/main.o
 .text._ZL12get_thread_1PKv
                0x08001308        0x8 Application/User/main.o
 .text._ZL12get_thread_0PKv
                0x08001310        0x8 Application/User/main.o
 .text._ZL10ble_threadPKv
                0x08001318       0xc0 Application/User/main.o
 .text._ZL16InitBlueNRGStackv
                0x080013d8      0x290 Application/User/main.o
 .text._Z17get_timer_0_Startv
                0x08001668       0x40 Application/User/main.o
                0x08001668                get_timer_0_Start()
 .text._Z17get_timer_1_Startv
                0x080016a8       0x40 Application/User/main.o
                0x080016a8                get_timer_1_Start()
 .text._Z17get_timer_2_Startv
                0x080016e8       0x40 Application/User/main.o
                0x080016e8                get_timer_2_Start()
 .text._Z16get_timer_1_Stopv
                0x08001728       0x10 Application/User/main.o
                0x08001728                get_timer_1_Stop()
 .text._Z16get_timer_2_Stopv
                0x08001738       0x10 Application/User/main.o
                0x08001738                get_timer_2_Stop()
 .text._Z18ble_timer_CallbackPKv
                0x08001748       0x10 Application/User/main.o
                0x08001748                ble_timer_Callback(void const*)
 .text._Z25get_samp_timer_0_CallbackPKv
                0x08001758        0xc Application/User/main.o
                0x08001758                get_samp_timer_0_Callback(void const*)
 .text._Z20get_timer_1_CallbackPKv
                0x08001764       0x10 Application/User/main.o
                0x08001764                get_timer_1_Callback(void const*)
 .text._Z20get_timer_2_CallbackPKv
                0x08001774       0x10 Application/User/main.o
                0x08001774                get_timer_2_Callback(void const*)
 .text._ZL14thrsh_thread_0PKv
                0x08001784       0xb4 Application/User/main.o
 .text._ZL14pros1_thread_0PKv
                0x08001838       0xd8 Application/User/main.o
 .text._Z16get_timer_0_Stopv
                0x08001910       0x10 Application/User/main.o
                0x08001910                get_timer_0_Stop()
 .text.startup.main
                0x08001920      0x354 Application/User/main.o
                0x08001920                main
 .text._Z11initAllTaskv
                0x08001c74       0x2c Application/User/main.o
                0x08001c74                initAllTask()
 .text._Z18master_timer_Startv
                0x08001ca0       0x44 Application/User/main.o
                0x08001ca0                master_timer_Start()
 .text._Z15ble_timer_Startv
                0x08001ce4       0x34 Application/User/main.o
                0x08001ce4                ble_timer_Start()
 .text._Z22get_samp_timer_0_Startv
                0x08001d18       0x30 Application/User/main.o
                0x08001d18                get_samp_timer_0_Start()
 .text._ZL13master_threadPKv
                0x08001d48      0x258 Application/User/main.o
 .text.HAL_GPIO_EXTI_Callback
                0x08001fa0       0x1c Application/User/main.o
                0x08001fa0                HAL_GPIO_EXTI_Callback
 .text.startup._GLOBAL__sub_I_StartTime
                0x08001fbc       0x24 Application/User/main.o
 .text.sclkUpdate.part.0
                0x08001fe0       0xe4 Application/User/sensor_service.o
 .text.Add_ConfigW2ST_Service
                0x080020c4       0xe4 Application/User/sensor_service.o
                0x080020c4                Add_ConfigW2ST_Service
 .text.Add_HWServW2ST_Service
                0x080021a8       0x60 Application/User/sensor_service.o
                0x080021a8                Add_HWServW2ST_Service
 .text.addSensorCharacteristc
                0x08002208       0x98 Application/User/sensor_service.o
                0x08002208                addSensorCharacteristc
 .text.charUpdate
                0x080022a0      0x280 Application/User/sensor_service.o
                0x080022a0                charUpdate
 .text.cycleUpdate
                0x08002520      0x114 Application/User/sensor_service.o
                0x08002520                cycleUpdate
 .text.setConnectable
                0x08002634       0xe8 Application/User/sensor_service.o
                0x08002634                setConnectable
 .text.Read_Request_CB
                0x0800271c       0xac Application/User/sensor_service.o
                0x0800271c                Read_Request_CB
 .text.Attribute_Modified_CB
                0x080027c8      0x27c Application/User/sensor_service.o
                0x080027c8                Attribute_Modified_CB
 .text.HCI_Event_CB
                0x08002a44      0x108 Application/User/sensor_service.o
                0x08002a44                HCI_Event_CB
 .text.HAL_TIM_Base_MspInit
                0x08002b4c       0x78 Application/User/stm32l4xx_hal_msp.o
                0x08002b4c                HAL_TIM_Base_MspInit
 .text.NMI_Handler
                0x08002bc4        0x4 Application/User/stm32l4xx_it.o
                0x08002bc4                NMI_Handler
 .text.HardFault_Handler
                0x08002bc8        0x4 Application/User/stm32l4xx_it.o
                0x08002bc8                HardFault_Handler
 .text.MemManage_Handler
                0x08002bcc        0x4 Application/User/stm32l4xx_it.o
                0x08002bcc                MemManage_Handler
 .text.BusFault_Handler
                0x08002bd0        0x4 Application/User/stm32l4xx_it.o
                0x08002bd0                BusFault_Handler
 .text.UsageFault_Handler
                0x08002bd4        0x4 Application/User/stm32l4xx_it.o
                0x08002bd4                UsageFault_Handler
 .text.DebugMon_Handler
                0x08002bd8        0x4 Application/User/stm32l4xx_it.o
                0x08002bd8                DebugMon_Handler
 .text.SysTick_Handler
                0x08002bdc       0x10 Application/User/stm32l4xx_it.o
                0x08002bdc                SysTick_Handler
 .text.TIM1_CC_IRQHandler
                0x08002bec        0xc Application/User/stm32l4xx_it.o
                0x08002bec                TIM1_CC_IRQHandler
 .text.EXTI9_5_IRQHandler
                0x08002bf8        0x8 Application/User/stm32l4xx_it.o
                0x08002bf8                EXTI9_5_IRQHandler
 .text.OTG_FS_IRQHandler
                0x08002c00        0xc Application/User/stm32l4xx_it.o
                0x08002c00                OTG_FS_IRQHandler
 .text.DMA2_Channel2_IRQHandler
                0x08002c0c        0xc Application/User/stm32l4xx_it.o
                0x08002c0c                DMA2_Channel2_IRQHandler
 .text.TIM3_IRQHandler
                0x08002c18        0xc Application/User/stm32l4xx_it.o
                0x08002c18                TIM3_IRQHandler
 .text.EXTI2_IRQHandler
                0x08002c24        0x8 Application/User/stm32l4xx_it.o
                0x08002c24                EXTI2_IRQHandler
 .text.CDC_Itf_DeInit
                0x08002c2c        0x4 Application/User/usbd_cdc_interface.o
 .text.CDC_Itf_Receive
                0x08002c30        0x4 Application/User/usbd_cdc_interface.o
 .text.CDC_Itf_Init
                0x08002c34       0x7c Application/User/usbd_cdc_interface.o
 .text.CDC_Itf_Control
                0x08002cb0       0x4c Application/User/usbd_cdc_interface.o
 .text.CDC_Fill_Buffer
                0x08002cfc       0x38 Application/User/usbd_cdc_interface.o
                0x08002cfc                CDC_Fill_Buffer
 .text.HAL_TIM_PeriodElapsedCallback
                0x08002d34       0x44 Application/User/usbd_cdc_interface.o
                0x08002d34                HAL_TIM_PeriodElapsedCallback
 .text.HAL_PCD_MspInit
                0x08002d78       0x64 Application/User/usbd_conf.o
                0x08002d78                HAL_PCD_MspInit
 .text.HAL_PCD_SetupStageCallback
                0x08002ddc        0xc Application/User/usbd_conf.o
                0x08002ddc                HAL_PCD_SetupStageCallback
 .text.HAL_PCD_DataOutStageCallback
                0x08002de8       0x14 Application/User/usbd_conf.o
                0x08002de8                HAL_PCD_DataOutStageCallback
 .text.HAL_PCD_DataInStageCallback
                0x08002dfc       0x14 Application/User/usbd_conf.o
                0x08002dfc                HAL_PCD_DataInStageCallback
 .text.HAL_PCD_SOFCallback
                0x08002e10        0x8 Application/User/usbd_conf.o
                0x08002e10                HAL_PCD_SOFCallback
 .text.HAL_PCD_ResetCallback
                0x08002e18       0x1c Application/User/usbd_conf.o
                0x08002e18                HAL_PCD_ResetCallback
 .text.HAL_PCD_SuspendCallback
                0x08002e34        0x8 Application/User/usbd_conf.o
                0x08002e34                HAL_PCD_SuspendCallback
 .text.HAL_PCD_ResumeCallback
                0x08002e3c        0x8 Application/User/usbd_conf.o
                0x08002e3c                HAL_PCD_ResumeCallback
 .text.HAL_PCD_ISOOUTIncompleteCallback
                0x08002e44        0x8 Application/User/usbd_conf.o
                0x08002e44                HAL_PCD_ISOOUTIncompleteCallback
 .text.HAL_PCD_ISOINIncompleteCallback
                0x08002e4c        0x8 Application/User/usbd_conf.o
                0x08002e4c                HAL_PCD_ISOINIncompleteCallback
 .text.HAL_PCD_ConnectCallback
                0x08002e54        0x8 Application/User/usbd_conf.o
                0x08002e54                HAL_PCD_ConnectCallback
 .text.HAL_PCD_DisconnectCallback
                0x08002e5c        0x8 Application/User/usbd_conf.o
                0x08002e5c                HAL_PCD_DisconnectCallback
 .text.USBD_LL_Init
                0x08002e64       0x5c Application/User/usbd_conf.o
                0x08002e64                USBD_LL_Init
 .text.USBD_LL_Start
                0x08002ec0       0x10 Application/User/usbd_conf.o
                0x08002ec0                USBD_LL_Start
 .text.USBD_LL_OpenEP
                0x08002ed0       0x14 Application/User/usbd_conf.o
                0x08002ed0                USBD_LL_OpenEP
 .text.USBD_LL_CloseEP
                0x08002ee4       0x10 Application/User/usbd_conf.o
                0x08002ee4                USBD_LL_CloseEP
 .text.USBD_LL_StallEP
                0x08002ef4       0x10 Application/User/usbd_conf.o
                0x08002ef4                USBD_LL_StallEP
 .text.USBD_LL_ClearStallEP
                0x08002f04       0x10 Application/User/usbd_conf.o
                0x08002f04                USBD_LL_ClearStallEP
 .text.USBD_LL_IsStallEP
                0x08002f14       0x28 Application/User/usbd_conf.o
                0x08002f14                USBD_LL_IsStallEP
 .text.USBD_LL_SetUSBAddress
                0x08002f3c       0x10 Application/User/usbd_conf.o
                0x08002f3c                USBD_LL_SetUSBAddress
 .text.USBD_LL_Transmit
                0x08002f4c       0x10 Application/User/usbd_conf.o
                0x08002f4c                USBD_LL_Transmit
 .text.USBD_LL_PrepareReceive
                0x08002f5c       0x10 Application/User/usbd_conf.o
                0x08002f5c                USBD_LL_PrepareReceive
 .text.USBD_LL_GetRxDataSize
                0x08002f6c        0xc Application/User/usbd_conf.o
                0x08002f6c                USBD_LL_GetRxDataSize
 .text.USBD_VCP_DeviceDescriptor
                0x08002f78        0xc Application/User/usbd_desc.o
                0x08002f78                USBD_VCP_DeviceDescriptor
 .text.USBD_VCP_LangIDStrDescriptor
                0x08002f84        0xc Application/User/usbd_desc.o
                0x08002f84                USBD_VCP_LangIDStrDescriptor
 .text.USBD_VCP_ProductStrDescriptor
                0x08002f90       0x1c Application/User/usbd_desc.o
                0x08002f90                USBD_VCP_ProductStrDescriptor
 .text.USBD_VCP_ManufacturerStrDescriptor
                0x08002fac       0x1c Application/User/usbd_desc.o
                0x08002fac                USBD_VCP_ManufacturerStrDescriptor
 .text.USBD_VCP_ConfigStrDescriptor
                0x08002fc8       0x1c Application/User/usbd_desc.o
                0x08002fc8                USBD_VCP_ConfigStrDescriptor
 .text.USBD_VCP_InterfaceStrDescriptor
                0x08002fe4       0x1c Application/User/usbd_desc.o
                0x08002fe4                USBD_VCP_InterfaceStrDescriptor
 .text.USBD_VCP_SerialStrDescriptor
                0x08003000      0x14c Application/User/usbd_desc.o
                0x08003000                USBD_VCP_SerialStrDescriptor
 .text.LSM303AGR_ACC_WriteReg
                0x0800314c       0x10 Drivers/BSP/Components/LSM303AGR_ACC_driver.o
                0x0800314c                LSM303AGR_ACC_WriteReg
 .text.LSM303AGR_ACC_ReadReg
                0x0800315c       0x10 Drivers/BSP/Components/LSM303AGR_ACC_driver.o
                0x0800315c                LSM303AGR_ACC_ReadReg
 .text.LSM303AGR_ACC_R_WHO_AM_I
                0x0800316c       0x14 Drivers/BSP/Components/LSM303AGR_ACC_driver.o
                0x0800316c                LSM303AGR_ACC_R_WHO_AM_I
 .text.LSM303AGR_ACC_W_BlockDataUpdate
                0x08003180       0x44 Drivers/BSP/Components/LSM303AGR_ACC_driver.o
                0x08003180                LSM303AGR_ACC_W_BlockDataUpdate
 .text.LSM303AGR_ACC_W_FullScale
                0x080031c4       0x44 Drivers/BSP/Components/LSM303AGR_ACC_driver.o
                0x080031c4                LSM303AGR_ACC_W_FullScale
 .text.LSM303AGR_ACC_R_FullScale
                0x08003208       0x20 Drivers/BSP/Components/LSM303AGR_ACC_driver.o
                0x08003208                LSM303AGR_ACC_R_FullScale
 .text.LSM303AGR_ACC_Get_Raw_Acceleration
                0x08003228       0x14 Drivers/BSP/Components/LSM303AGR_ACC_driver.o
                0x08003228                LSM303AGR_ACC_Get_Raw_Acceleration
 .text.LSM303AGR_ACC_Get_Acceleration
                0x0800323c      0x170 Drivers/BSP/Components/LSM303AGR_ACC_driver.o
                0x0800323c                LSM303AGR_ACC_Get_Acceleration
 .text.LSM303AGR_ACC_W_ODR
                0x080033ac       0x44 Drivers/BSP/Components/LSM303AGR_ACC_driver.o
                0x080033ac                LSM303AGR_ACC_W_ODR
 .text.LSM303AGR_ACC_R_ODR
                0x080033f0       0x20 Drivers/BSP/Components/LSM303AGR_ACC_driver.o
                0x080033f0                LSM303AGR_ACC_R_ODR
 .text.LSM303AGR_ACC_W_XEN
                0x08003410       0x44 Drivers/BSP/Components/LSM303AGR_ACC_driver.o
                0x08003410                LSM303AGR_ACC_W_XEN
 .text.LSM303AGR_ACC_R_XEN
                0x08003454       0x20 Drivers/BSP/Components/LSM303AGR_ACC_driver.o
                0x08003454                LSM303AGR_ACC_R_XEN
 .text.LSM303AGR_ACC_W_YEN
                0x08003474       0x44 Drivers/BSP/Components/LSM303AGR_ACC_driver.o
                0x08003474                LSM303AGR_ACC_W_YEN
 .text.LSM303AGR_ACC_R_YEN
                0x080034b8       0x20 Drivers/BSP/Components/LSM303AGR_ACC_driver.o
                0x080034b8                LSM303AGR_ACC_R_YEN
 .text.LSM303AGR_ACC_W_ZEN
                0x080034d8       0x44 Drivers/BSP/Components/LSM303AGR_ACC_driver.o
                0x080034d8                LSM303AGR_ACC_W_ZEN
 .text.LSM303AGR_ACC_R_ZEN
                0x0800351c       0x20 Drivers/BSP/Components/LSM303AGR_ACC_driver.o
                0x0800351c                LSM303AGR_ACC_R_ZEN
 .text.LSM303AGR_ACC_R_LOWPWR_EN
                0x0800353c       0x20 Drivers/BSP/Components/LSM303AGR_ACC_driver.o
                0x0800353c                LSM303AGR_ACC_R_LOWPWR_EN
 .text.LSM303AGR_ACC_R_HiRes
                0x0800355c       0x20 Drivers/BSP/Components/LSM303AGR_ACC_driver.o
                0x0800355c                LSM303AGR_ACC_R_HiRes
 .text.LSM303AGR_ACC_R_XDataAvail
                0x0800357c       0x20 Drivers/BSP/Components/LSM303AGR_ACC_driver.o
                0x0800357c                LSM303AGR_ACC_R_XDataAvail
 .text.LSM303AGR_ACC_W_FifoMode
                0x0800359c       0x44 Drivers/BSP/Components/LSM303AGR_ACC_driver.o
                0x0800359c                LSM303AGR_ACC_W_FifoMode
 .text.LSM303AGR_X_Get_DRDY_Status
                0x080035e0       0x30 Drivers/BSP/Components/LSM303AGR_ACC_driver_HL.o
 .text.LSM303AGR_X_Write_Reg
                0x08003610       0x1c Drivers/BSP/Components/LSM303AGR_ACC_driver_HL.o
 .text.LSM303AGR_X_Read_Reg
                0x0800362c       0x10 Drivers/BSP/Components/LSM303AGR_ACC_driver_HL.o
 .text.LSM303AGR_X_Get_Axes_Status
                0x0800363c       0x68 Drivers/BSP/Components/LSM303AGR_ACC_driver_HL.o
 .text.LSM303AGR_X_Set_FS_Value
                0x080036a4       0x58 Drivers/BSP/Components/LSM303AGR_ACC_driver_HL.o
 .text.LSM303AGR_X_Set_FS
                0x080036fc       0x30 Drivers/BSP/Components/LSM303AGR_ACC_driver_HL.o
 .text.LSM303AGR_X_Get_FS
                0x0800372c       0x68 Drivers/BSP/Components/LSM303AGR_ACC_driver_HL.o
 .text.LSM303AGR_X_Get_ODR
                0x08003794       0xa0 Drivers/BSP/Components/LSM303AGR_ACC_driver_HL.o
 .text.LSM303AGR_X_Get_Sensitivity
                0x08003834      0x13c Drivers/BSP/Components/LSM303AGR_ACC_driver_HL.o
 .text.LSM303AGR_X_Get_AxesRaw
                0x08003970       0x78 Drivers/BSP/Components/LSM303AGR_ACC_driver_HL.o
 .text.LSM303AGR_X_Get_Axes
                0x080039e8       0x28 Drivers/BSP/Components/LSM303AGR_ACC_driver_HL.o
 .text.LSM303AGR_X_Get_WhoAmI
                0x08003a10       0x10 Drivers/BSP/Components/LSM303AGR_ACC_driver_HL.o
 .text.LSM303AGR_X_Check_WhoAmI
                0x08003a20       0x2c Drivers/BSP/Components/LSM303AGR_ACC_driver_HL.o
 .text.LSM303AGR_X_Set_Axes_Status
                0x08003a4c       0x48 Drivers/BSP/Components/LSM303AGR_ACC_driver_HL.o
 .text.LSM303AGR_X_Set_ODR_Value
                0x08003a94       0xfc Drivers/BSP/Components/LSM303AGR_ACC_driver_HL.o
 .text.LSM303AGR_X_Set_ODR
                0x08003b90       0x84 Drivers/BSP/Components/LSM303AGR_ACC_driver_HL.o
 .text.LSM303AGR_X_Sensor_Enable
                0x08003c14       0xa8 Drivers/BSP/Components/LSM303AGR_ACC_driver_HL.o
 .text.LSM303AGR_X_Sensor_Disable
                0x08003cbc       0xb0 Drivers/BSP/Components/LSM303AGR_ACC_driver_HL.o
 .text.LSM303AGR_X_DeInit
                0x08003d6c       0xdc Drivers/BSP/Components/LSM303AGR_ACC_driver_HL.o
 .text.LSM303AGR_X_Init
                0x08003e48       0x90 Drivers/BSP/Components/LSM303AGR_ACC_driver_HL.o
 .text.LSM6DSM_ACC_GYRO_ReadReg
                0x08003ed8       0x10 Drivers/BSP/Components/LSM6DSM_ACC_GYRO_driver.o
                0x08003ed8                LSM6DSM_ACC_GYRO_ReadReg
 .text.LSM6DSM_ACC_GYRO_WriteReg
                0x08003ee8       0x1c Drivers/BSP/Components/LSM6DSM_ACC_GYRO_driver.o
                0x08003ee8                LSM6DSM_ACC_GYRO_WriteReg
 .text.LSM6DSM_ACC_GYRO_W_FIFO_MODE
                0x08003f04       0x44 Drivers/BSP/Components/LSM6DSM_ACC_GYRO_driver.o
                0x08003f04                LSM6DSM_ACC_GYRO_W_FIFO_MODE
 .text.LSM6DSM_ACC_GYRO_W_STEP_DELTA_on_INT2
                0x08003f48       0x44 Drivers/BSP/Components/LSM6DSM_ACC_GYRO_driver.o
                0x08003f48                LSM6DSM_ACC_GYRO_W_STEP_DELTA_on_INT2
 .text.LSM6DSM_ACC_GYRO_R_WHO_AM_I
                0x08003f8c       0x14 Drivers/BSP/Components/LSM6DSM_ACC_GYRO_driver.o
                0x08003f8c                LSM6DSM_ACC_GYRO_R_WHO_AM_I
 .text.LSM6DSM_ACC_GYRO_W_FS_XL
                0x08003fa0       0x44 Drivers/BSP/Components/LSM6DSM_ACC_GYRO_driver.o
                0x08003fa0                LSM6DSM_ACC_GYRO_W_FS_XL
 .text.LSM6DSM_ACC_GYRO_R_FS_XL
                0x08003fe4       0x20 Drivers/BSP/Components/LSM6DSM_ACC_GYRO_driver.o
                0x08003fe4                LSM6DSM_ACC_GYRO_R_FS_XL
 .text.LSM6DSM_ACC_GYRO_W_ODR_XL
                0x08004004       0x44 Drivers/BSP/Components/LSM6DSM_ACC_GYRO_driver.o
                0x08004004                LSM6DSM_ACC_GYRO_W_ODR_XL
 .text.LSM6DSM_ACC_GYRO_R_ODR_XL
                0x08004048       0x20 Drivers/BSP/Components/LSM6DSM_ACC_GYRO_driver.o
                0x08004048                LSM6DSM_ACC_GYRO_R_ODR_XL
 .text.LSM6DSM_ACC_GYRO_W_FS_125
                0x08004068       0x44 Drivers/BSP/Components/LSM6DSM_ACC_GYRO_driver.o
                0x08004068                LSM6DSM_ACC_GYRO_W_FS_125
 .text.LSM6DSM_ACC_GYRO_R_FS_125
                0x080040ac       0x20 Drivers/BSP/Components/LSM6DSM_ACC_GYRO_driver.o
                0x080040ac                LSM6DSM_ACC_GYRO_R_FS_125
 .text.LSM6DSM_ACC_GYRO_W_FS_G
                0x080040cc       0x44 Drivers/BSP/Components/LSM6DSM_ACC_GYRO_driver.o
                0x080040cc                LSM6DSM_ACC_GYRO_W_FS_G
 .text.LSM6DSM_ACC_GYRO_R_FS_G
                0x08004110       0x20 Drivers/BSP/Components/LSM6DSM_ACC_GYRO_driver.o
                0x08004110                LSM6DSM_ACC_GYRO_R_FS_G
 .text.LSM6DSM_ACC_GYRO_W_ODR_G
                0x08004130       0x44 Drivers/BSP/Components/LSM6DSM_ACC_GYRO_driver.o
                0x08004130                LSM6DSM_ACC_GYRO_W_ODR_G
 .text.LSM6DSM_ACC_GYRO_R_ODR_G
                0x08004174       0x20 Drivers/BSP/Components/LSM6DSM_ACC_GYRO_driver.o
                0x08004174                LSM6DSM_ACC_GYRO_R_ODR_G
 .text.LSM6DSM_ACC_GYRO_W_IF_Addr_Incr
                0x08004194       0x44 Drivers/BSP/Components/LSM6DSM_ACC_GYRO_driver.o
                0x08004194                LSM6DSM_ACC_GYRO_W_IF_Addr_Incr
 .text.LSM6DSM_ACC_GYRO_W_BDU
                0x080041d8       0x44 Drivers/BSP/Components/LSM6DSM_ACC_GYRO_driver.o
                0x080041d8                LSM6DSM_ACC_GYRO_W_BDU
 .text.LSM6DSM_ACC_GYRO_W_I2C_DISABLE
                0x0800421c       0x44 Drivers/BSP/Components/LSM6DSM_ACC_GYRO_driver.o
                0x0800421c                LSM6DSM_ACC_GYRO_W_I2C_DISABLE
 .text.LSM6DSM_ACC_GYRO_W_PedoStepReset
                0x08004260       0x44 Drivers/BSP/Components/LSM6DSM_ACC_GYRO_driver.o
                0x08004260                LSM6DSM_ACC_GYRO_W_PedoStepReset
 .text.LSM6DSM_ACC_GYRO_W_TILT
                0x080042a4       0x44 Drivers/BSP/Components/LSM6DSM_ACC_GYRO_driver.o
                0x080042a4                LSM6DSM_ACC_GYRO_W_TILT
 .text.LSM6DSM_ACC_GYRO_W_PEDO
                0x080042e8       0x44 Drivers/BSP/Components/LSM6DSM_ACC_GYRO_driver.o
                0x080042e8                LSM6DSM_ACC_GYRO_W_PEDO
 .text.LSM6DSM_ACC_GYRO_W_FUNC_EN
                0x0800432c       0x44 Drivers/BSP/Components/LSM6DSM_ACC_GYRO_driver.o
                0x0800432c                LSM6DSM_ACC_GYRO_W_FUNC_EN
 .text.LSM6DSM_ACC_GYRO_R_WU_EV_STATUS
                0x08004370       0x20 Drivers/BSP/Components/LSM6DSM_ACC_GYRO_driver.o
                0x08004370                LSM6DSM_ACC_GYRO_R_WU_EV_STATUS
 .text.LSM6DSM_ACC_GYRO_R_FF_EV_STATUS
                0x08004390       0x20 Drivers/BSP/Components/LSM6DSM_ACC_GYRO_driver.o
                0x08004390                LSM6DSM_ACC_GYRO_R_FF_EV_STATUS
 .text.LSM6DSM_ACC_GYRO_R_DOUBLE_TAP_EV_STATUS
                0x080043b0       0x20 Drivers/BSP/Components/LSM6DSM_ACC_GYRO_driver.o
                0x080043b0                LSM6DSM_ACC_GYRO_R_DOUBLE_TAP_EV_STATUS
 .text.LSM6DSM_ACC_GYRO_R_SINGLE_TAP_EV_STATUS
                0x080043d0       0x20 Drivers/BSP/Components/LSM6DSM_ACC_GYRO_driver.o
                0x080043d0                LSM6DSM_ACC_GYRO_R_SINGLE_TAP_EV_STATUS
 .text.LSM6DSM_ACC_GYRO_R_DSD_XL
                0x080043f0       0x20 Drivers/BSP/Components/LSM6DSM_ACC_GYRO_driver.o
                0x080043f0                LSM6DSM_ACC_GYRO_R_DSD_XL
 .text.LSM6DSM_ACC_GYRO_R_DSD_XH
                0x08004410       0x20 Drivers/BSP/Components/LSM6DSM_ACC_GYRO_driver.o
                0x08004410                LSM6DSM_ACC_GYRO_R_DSD_XH
 .text.LSM6DSM_ACC_GYRO_R_DSD_YL
                0x08004430       0x20 Drivers/BSP/Components/LSM6DSM_ACC_GYRO_driver.o
                0x08004430                LSM6DSM_ACC_GYRO_R_DSD_YL
 .text.LSM6DSM_ACC_GYRO_R_DSD_YH
                0x08004450       0x20 Drivers/BSP/Components/LSM6DSM_ACC_GYRO_driver.o
                0x08004450                LSM6DSM_ACC_GYRO_R_DSD_YH
 .text.LSM6DSM_ACC_GYRO_R_DSD_ZL
                0x08004470       0x20 Drivers/BSP/Components/LSM6DSM_ACC_GYRO_driver.o
                0x08004470                LSM6DSM_ACC_GYRO_R_DSD_ZL
 .text.LSM6DSM_ACC_GYRO_R_DSD_ZH
                0x08004490       0x20 Drivers/BSP/Components/LSM6DSM_ACC_GYRO_driver.o
                0x08004490                LSM6DSM_ACC_GYRO_R_DSD_ZH
 .text.LSM6DSM_ACC_GYRO_R_D6D_EV_STATUS
                0x080044b0       0x20 Drivers/BSP/Components/LSM6DSM_ACC_GYRO_driver.o
                0x080044b0                LSM6DSM_ACC_GYRO_R_D6D_EV_STATUS
 .text.LSM6DSM_ACC_GYRO_R_XLDA
                0x080044d0       0x20 Drivers/BSP/Components/LSM6DSM_ACC_GYRO_driver.o
                0x080044d0                LSM6DSM_ACC_GYRO_R_XLDA
 .text.LSM6DSM_ACC_GYRO_R_GDA
                0x080044f0       0x20 Drivers/BSP/Components/LSM6DSM_ACC_GYRO_driver.o
                0x080044f0                LSM6DSM_ACC_GYRO_R_GDA
 .text.LSM6DSM_ACC_GYRO_R_PEDO_EV_STATUS
                0x08004510       0x20 Drivers/BSP/Components/LSM6DSM_ACC_GYRO_driver.o
                0x08004510                LSM6DSM_ACC_GYRO_R_PEDO_EV_STATUS
 .text.LSM6DSM_ACC_GYRO_R_TILT_EV_STATUS
                0x08004530       0x20 Drivers/BSP/Components/LSM6DSM_ACC_GYRO_driver.o
                0x08004530                LSM6DSM_ACC_GYRO_R_TILT_EV_STATUS
 .text.LSM6DSM_ACC_GYRO_W_TAP_Z_EN
                0x08004550       0x44 Drivers/BSP/Components/LSM6DSM_ACC_GYRO_driver.o
                0x08004550                LSM6DSM_ACC_GYRO_W_TAP_Z_EN
 .text.LSM6DSM_ACC_GYRO_W_TAP_Y_EN
                0x08004594       0x44 Drivers/BSP/Components/LSM6DSM_ACC_GYRO_driver.o
                0x08004594                LSM6DSM_ACC_GYRO_W_TAP_Y_EN
 .text.LSM6DSM_ACC_GYRO_W_TAP_X_EN
                0x080045d8       0x44 Drivers/BSP/Components/LSM6DSM_ACC_GYRO_driver.o
                0x080045d8                LSM6DSM_ACC_GYRO_W_TAP_X_EN
 .text.LSM6DSM_ACC_GYRO_W_BASIC_INT
                0x0800461c       0x44 Drivers/BSP/Components/LSM6DSM_ACC_GYRO_driver.o
                0x0800461c                LSM6DSM_ACC_GYRO_W_BASIC_INT
 .text.LSM6DSM_ACC_GYRO_W_TAP_THS
                0x08004660       0x48 Drivers/BSP/Components/LSM6DSM_ACC_GYRO_driver.o
                0x08004660                LSM6DSM_ACC_GYRO_W_TAP_THS
 .text.LSM6DSM_ACC_GYRO_W_SIXD_THS
                0x080046a8       0x44 Drivers/BSP/Components/LSM6DSM_ACC_GYRO_driver.o
                0x080046a8                LSM6DSM_ACC_GYRO_W_SIXD_THS
 .text.LSM6DSM_ACC_GYRO_W_SHOCK_Duration
                0x080046ec       0x48 Drivers/BSP/Components/LSM6DSM_ACC_GYRO_driver.o
                0x080046ec                LSM6DSM_ACC_GYRO_W_SHOCK_Duration
 .text.LSM6DSM_ACC_GYRO_W_QUIET_Duration
                0x08004734       0x4c Drivers/BSP/Components/LSM6DSM_ACC_GYRO_driver.o
                0x08004734                LSM6DSM_ACC_GYRO_W_QUIET_Duration
 .text.LSM6DSM_ACC_GYRO_W_DUR
                0x08004780       0x48 Drivers/BSP/Components/LSM6DSM_ACC_GYRO_driver.o
                0x08004780                LSM6DSM_ACC_GYRO_W_DUR
 .text.LSM6DSM_ACC_GYRO_W_WK_THS
                0x080047c8       0x48 Drivers/BSP/Components/LSM6DSM_ACC_GYRO_driver.o
                0x080047c8                LSM6DSM_ACC_GYRO_W_WK_THS
 .text.LSM6DSM_ACC_GYRO_W_SINGLE_DOUBLE_TAP_EV
                0x08004810       0x44 Drivers/BSP/Components/LSM6DSM_ACC_GYRO_driver.o
                0x08004810                LSM6DSM_ACC_GYRO_W_SINGLE_DOUBLE_TAP_EV
 .text.LSM6DSM_ACC_GYRO_W_SLEEP_DUR
                0x08004854       0x48 Drivers/BSP/Components/LSM6DSM_ACC_GYRO_driver.o
                0x08004854                LSM6DSM_ACC_GYRO_W_SLEEP_DUR
 .text.LSM6DSM_ACC_GYRO_W_TIMER_HR
                0x0800489c       0x44 Drivers/BSP/Components/LSM6DSM_ACC_GYRO_driver.o
                0x0800489c                LSM6DSM_ACC_GYRO_W_TIMER_HR
 .text.LSM6DSM_ACC_GYRO_W_WAKE_DUR
                0x080048e0       0x4c Drivers/BSP/Components/LSM6DSM_ACC_GYRO_driver.o
                0x080048e0                LSM6DSM_ACC_GYRO_W_WAKE_DUR
 .text.LSM6DSM_ACC_GYRO_W_FF_THS
                0x0800492c       0x44 Drivers/BSP/Components/LSM6DSM_ACC_GYRO_driver.o
                0x0800492c                LSM6DSM_ACC_GYRO_W_FF_THS
 .text.LSM6DSM_ACC_GYRO_W_FF_Duration
                0x08004970       0x80 Drivers/BSP/Components/LSM6DSM_ACC_GYRO_driver.o
                0x08004970                LSM6DSM_ACC_GYRO_W_FF_Duration
 .text.LSM6DSM_ACC_GYRO_W_TiltEvOnInt1
                0x080049f0       0x44 Drivers/BSP/Components/LSM6DSM_ACC_GYRO_driver.o
                0x080049f0                LSM6DSM_ACC_GYRO_W_TiltEvOnInt1
 .text.LSM6DSM_ACC_GYRO_W_6DEvOnInt1
                0x08004a34       0x44 Drivers/BSP/Components/LSM6DSM_ACC_GYRO_driver.o
                0x08004a34                LSM6DSM_ACC_GYRO_W_6DEvOnInt1
 .text.LSM6DSM_ACC_GYRO_W_TapEvOnInt1
                0x08004a78       0x44 Drivers/BSP/Components/LSM6DSM_ACC_GYRO_driver.o
                0x08004a78                LSM6DSM_ACC_GYRO_W_TapEvOnInt1
 .text.LSM6DSM_ACC_GYRO_W_FFEvOnInt1
                0x08004abc       0x44 Drivers/BSP/Components/LSM6DSM_ACC_GYRO_driver.o
                0x08004abc                LSM6DSM_ACC_GYRO_W_FFEvOnInt1
 .text.LSM6DSM_ACC_GYRO_W_WUEvOnInt1
                0x08004b00       0x44 Drivers/BSP/Components/LSM6DSM_ACC_GYRO_driver.o
                0x08004b00                LSM6DSM_ACC_GYRO_W_WUEvOnInt1
 .text.LSM6DSM_ACC_GYRO_W_SingleTapOnInt1
                0x08004b44       0x44 Drivers/BSP/Components/LSM6DSM_ACC_GYRO_driver.o
                0x08004b44                LSM6DSM_ACC_GYRO_W_SingleTapOnInt1
 .text.LSM6DSM_ACC_GYRO_W_TiltEvOnInt2
                0x08004b88       0x44 Drivers/BSP/Components/LSM6DSM_ACC_GYRO_driver.o
                0x08004b88                LSM6DSM_ACC_GYRO_W_TiltEvOnInt2
 .text.LSM6DSM_ACC_GYRO_W_6DEvOnInt2
                0x08004bcc       0x44 Drivers/BSP/Components/LSM6DSM_ACC_GYRO_driver.o
                0x08004bcc                LSM6DSM_ACC_GYRO_W_6DEvOnInt2
 .text.LSM6DSM_ACC_GYRO_W_TapEvOnInt2
                0x08004c10       0x44 Drivers/BSP/Components/LSM6DSM_ACC_GYRO_driver.o
                0x08004c10                LSM6DSM_ACC_GYRO_W_TapEvOnInt2
 .text.LSM6DSM_ACC_GYRO_W_FFEvOnInt2
                0x08004c54       0x44 Drivers/BSP/Components/LSM6DSM_ACC_GYRO_driver.o
                0x08004c54                LSM6DSM_ACC_GYRO_W_FFEvOnInt2
 .text.LSM6DSM_ACC_GYRO_W_WUEvOnInt2
                0x08004c98       0x44 Drivers/BSP/Components/LSM6DSM_ACC_GYRO_driver.o
                0x08004c98                LSM6DSM_ACC_GYRO_W_WUEvOnInt2
 .text.LSM6DSM_ACC_GYRO_W_SingleTapOnInt2
                0x08004cdc       0x44 Drivers/BSP/Components/LSM6DSM_ACC_GYRO_driver.o
                0x08004cdc                LSM6DSM_ACC_GYRO_W_SingleTapOnInt2
 .text.LSM6DSM_ACC_GYRO_GetRawGyroData
                0x08004d20       0x38 Drivers/BSP/Components/LSM6DSM_ACC_GYRO_driver.o
                0x08004d20                LSM6DSM_ACC_GYRO_GetRawGyroData
 .text.LSM6DSM_ACC_GYRO_GetRawAccData
                0x08004d58       0x38 Drivers/BSP/Components/LSM6DSM_ACC_GYRO_driver.o
                0x08004d58                LSM6DSM_ACC_GYRO_GetRawAccData
 .text.LSM6DSM_ACC_GYRO_Get_GetStepCounter
                0x08004d90       0x2c Drivers/BSP/Components/LSM6DSM_ACC_GYRO_driver.o
                0x08004d90                LSM6DSM_ACC_GYRO_Get_GetStepCounter
 .text.LSM6DSM_ACC_GYRO_W_PedoThreshold
                0x08004dbc       0xac Drivers/BSP/Components/LSM6DSM_ACC_GYRO_driver.o
                0x08004dbc                LSM6DSM_ACC_GYRO_W_PedoThreshold
 .text.LSM6DSM_X_Get_6D_Orientation_ZH
                0x08004e68       0x30 Drivers/BSP/Components/LSM6DSM_ACC_GYRO_driver_HL.o
 .text.LSM6DSM_X_Get_6D_Orientation_ZL
                0x08004e98       0x30 Drivers/BSP/Components/LSM6DSM_ACC_GYRO_driver_HL.o
 .text.LSM6DSM_X_Get_6D_Orientation_YH
                0x08004ec8       0x30 Drivers/BSP/Components/LSM6DSM_ACC_GYRO_driver_HL.o
 .text.LSM6DSM_X_Get_6D_Orientation_YL
                0x08004ef8       0x30 Drivers/BSP/Components/LSM6DSM_ACC_GYRO_driver_HL.o
 .text.LSM6DSM_X_Get_6D_Orientation_XH
                0x08004f28       0x30 Drivers/BSP/Components/LSM6DSM_ACC_GYRO_driver_HL.o
 .text.LSM6DSM_X_Get_6D_Orientation_XL
                0x08004f58       0x30 Drivers/BSP/Components/LSM6DSM_ACC_GYRO_driver_HL.o
 .text.LSM6DSM_X_Get_6D_Orientation_Status
                0x08004f88       0x30 Drivers/BSP/Components/LSM6DSM_ACC_GYRO_driver_HL.o
 .text.LSM6DSM_X_Set_FS_Value
                0x08004fb8       0x58 Drivers/BSP/Components/LSM6DSM_ACC_GYRO_driver_HL.o
 .text.LSM6DSM_X_Set_FS
                0x08005010       0x30 Drivers/BSP/Components/LSM6DSM_ACC_GYRO_driver_HL.o
 .text.LSM6DSM_X_Set_Tap_Duration_Time
                0x08005040       0x10 Drivers/BSP/Components/LSM6DSM_ACC_GYRO_driver_HL.o
 .text.LSM6DSM_X_Set_Tap_Quiet_Time
                0x08005050       0x10 Drivers/BSP/Components/LSM6DSM_ACC_GYRO_driver_HL.o
 .text.LSM6DSM_X_Set_Tap_Shock_Time
                0x08005060       0x10 Drivers/BSP/Components/LSM6DSM_ACC_GYRO_driver_HL.o
 .text.LSM6DSM_X_Set_Tap_Threshold
                0x08005070       0x10 Drivers/BSP/Components/LSM6DSM_ACC_GYRO_driver_HL.o
 .text.LSM6DSM_X_Get_Double_Tap_Detection_Status
                0x08005080       0x30 Drivers/BSP/Components/LSM6DSM_ACC_GYRO_driver_HL.o
 .text.LSM6DSM_X_Get_Single_Tap_Detection_Status
                0x080050b0       0x30 Drivers/BSP/Components/LSM6DSM_ACC_GYRO_driver_HL.o
 .text.LSM6DSM_X_Set_Wake_Up_Threshold
                0x080050e0       0x10 Drivers/BSP/Components/LSM6DSM_ACC_GYRO_driver_HL.o
 .text.LSM6DSM_X_Get_Wake_Up_Detection_Status
                0x080050f0       0x30 Drivers/BSP/Components/LSM6DSM_ACC_GYRO_driver_HL.o
 .text.LSM6DSM_X_Get_Tilt_Detection_Status
                0x08005120       0x30 Drivers/BSP/Components/LSM6DSM_ACC_GYRO_driver_HL.o
 .text.LSM6DSM_X_Set_Pedometer_Threshold
                0x08005150       0x10 Drivers/BSP/Components/LSM6DSM_ACC_GYRO_driver_HL.o
 .text.LSM6DSM_X_Disable_Step_Counter_Reset
                0x08005160       0x10 Drivers/BSP/Components/LSM6DSM_ACC_GYRO_driver_HL.o
 .text.LSM6DSM_X_Enable_Step_Counter_Reset
                0x08005170       0x10 Drivers/BSP/Components/LSM6DSM_ACC_GYRO_driver_HL.o
 .text.LSM6DSM_X_Get_Step_Count
                0x08005180       0x10 Drivers/BSP/Components/LSM6DSM_ACC_GYRO_driver_HL.o
 .text.LSM6DSM_X_Get_Pedometer_Status
                0x08005190       0x30 Drivers/BSP/Components/LSM6DSM_ACC_GYRO_driver_HL.o
 .text.LSM6DSM_X_Set_Free_Fall_Threshold
                0x080051c0       0x10 Drivers/BSP/Components/LSM6DSM_ACC_GYRO_driver_HL.o
 .text.LSM6DSM_X_Get_Free_Fall_Detection_Status
                0x080051d0       0x30 Drivers/BSP/Components/LSM6DSM_ACC_GYRO_driver_HL.o
 .text.LSM6DSM_X_Get_DRDY_Status
                0x08005200       0x30 Drivers/BSP/Components/LSM6DSM_ACC_GYRO_driver_HL.o
 .text.LSM6DSM_G_Write_Reg
                0x08005230       0x10 Drivers/BSP/Components/LSM6DSM_ACC_GYRO_driver_HL.o
 .text.LSM6DSM_G_Read_Reg
                0x08005240       0x10 Drivers/BSP/Components/LSM6DSM_ACC_GYRO_driver_HL.o
 .text.LSM6DSM_X_Get_FS
                0x08005250       0x70 Drivers/BSP/Components/LSM6DSM_ACC_GYRO_driver_HL.o
 .text.LSM6DSM_X_Get_Sensitivity
                0x080052c0       0x78 Drivers/BSP/Components/LSM6DSM_ACC_GYRO_driver_HL.o
 .text.LSM6DSM_X_Get_ODR
                0x08005338       0xd4 Drivers/BSP/Components/LSM6DSM_ACC_GYRO_driver_HL.o
 .text.LSM6DSM_X_Get_WhoAmI
                0x0800540c       0x10 Drivers/BSP/Components/LSM6DSM_ACC_GYRO_driver_HL.o
 .text.LSM6DSM_G_Get_DRDY_Status
                0x0800541c       0x30 Drivers/BSP/Components/LSM6DSM_ACC_GYRO_driver_HL.o
 .text.LSM6DSM_G_Set_FS
                0x0800544c       0x30 Drivers/BSP/Components/LSM6DSM_ACC_GYRO_driver_HL.o
 .text.LSM6DSM_G_Get_FS
                0x0800547c       0x90 Drivers/BSP/Components/LSM6DSM_ACC_GYRO_driver_HL.o
 .text.LSM6DSM_G_Get_ODR
                0x0800550c       0xd4 Drivers/BSP/Components/LSM6DSM_ACC_GYRO_driver_HL.o
 .text.LSM6DSM_X_Disable_6D_Orientation
                0x080055e0       0x38 Drivers/BSP/Components/LSM6DSM_ACC_GYRO_driver_HL.o
 .text.LSM6DSM_X_Set_ODR
                0x08005618       0x78 Drivers/BSP/Components/LSM6DSM_ACC_GYRO_driver_HL.o
 .text.LSM6DSM_X_Disable_Double_Tap_Detection
                0x08005690       0x8c Drivers/BSP/Components/LSM6DSM_ACC_GYRO_driver_HL.o
 .text.LSM6DSM_X_Disable_Single_Tap_Detection
                0x0800571c       0x74 Drivers/BSP/Components/LSM6DSM_ACC_GYRO_driver_HL.o
 .text.LSM6DSM_X_Disable_Wake_Up_Detection
                0x08005790       0x44 Drivers/BSP/Components/LSM6DSM_ACC_GYRO_driver_HL.o
 .text.LSM6DSM_X_Disable_Tilt_Detection
                0x080057d4       0x38 Drivers/BSP/Components/LSM6DSM_ACC_GYRO_driver_HL.o
 .text.LSM6DSM_X_Disable_Pedometer
                0x0800580c       0x38 Drivers/BSP/Components/LSM6DSM_ACC_GYRO_driver_HL.o
 .text.LSM6DSM_X_Disable_Free_Fall_Detection
                0x08005844       0x44 Drivers/BSP/Components/LSM6DSM_ACC_GYRO_driver_HL.o
 .text.LSM6DSM_G_Set_FS_Value
                0x08005888       0x90 Drivers/BSP/Components/LSM6DSM_ACC_GYRO_driver_HL.o
 .text.LSM6DSM_G_Get_Sensitivity
                0x08005918       0x90 Drivers/BSP/Components/LSM6DSM_ACC_GYRO_driver_HL.o
 .text.LSM6DSM_G_Set_ODR_Value
                0x080059a8      0x168 Drivers/BSP/Components/LSM6DSM_ACC_GYRO_driver_HL.o
 .text.LSM6DSM_G_Set_ODR
                0x08005b10       0x78 Drivers/BSP/Components/LSM6DSM_ACC_GYRO_driver_HL.o
 .text.LSM6DSM_G_Get_WhoAmI
                0x08005b88       0x10 Drivers/BSP/Components/LSM6DSM_ACC_GYRO_driver_HL.o
 .text.LSM6DSM_X_Read_Reg
                0x08005b98       0x10 Drivers/BSP/Components/LSM6DSM_ACC_GYRO_driver_HL.o
 .text.LSM6DSM_X_Write_Reg
                0x08005ba8       0x10 Drivers/BSP/Components/LSM6DSM_ACC_GYRO_driver_HL.o
 .text.LSM6DSM_X_Set_ODR_Value
                0x08005bb8      0x168 Drivers/BSP/Components/LSM6DSM_ACC_GYRO_driver_HL.o
 .text.LSM6DSM_X_Enable_Double_Tap_Detection
                0x08005d20       0xd0 Drivers/BSP/Components/LSM6DSM_ACC_GYRO_driver_HL.o
 .text.LSM6DSM_X_Enable_Tilt_Detection
                0x08005df0       0x7c Drivers/BSP/Components/LSM6DSM_ACC_GYRO_driver_HL.o
 .text.LSM6DSM_X_Enable_Pedometer
                0x08005e6c       0x70 Drivers/BSP/Components/LSM6DSM_ACC_GYRO_driver_HL.o
 .text.LSM6DSM_G_Get_AxesRaw
                0x08005edc       0x4c Drivers/BSP/Components/LSM6DSM_ACC_GYRO_driver_HL.o
 .text.LSM6DSM_X_Get_AxesRaw
                0x08005f28       0x4c Drivers/BSP/Components/LSM6DSM_ACC_GYRO_driver_HL.o
 .text.LSM6DSM_G_Check_WhoAmI
                0x08005f74       0x2c Drivers/BSP/Components/LSM6DSM_ACC_GYRO_driver_HL.o
 .text.LSM6DSM_X_Check_WhoAmI
                0x08005fa0       0x2c Drivers/BSP/Components/LSM6DSM_ACC_GYRO_driver_HL.o
 .text.LSM6DSM_G_Sensor_Enable
                0x08005fcc       0xe8 Drivers/BSP/Components/LSM6DSM_ACC_GYRO_driver_HL.o
 .text.LSM6DSM_X_Sensor_Enable
                0x080060b4       0xe8 Drivers/BSP/Components/LSM6DSM_ACC_GYRO_driver_HL.o
 .text.LSM6DSM_G_Get_Axes
                0x0800619c       0xf8 Drivers/BSP/Components/LSM6DSM_ACC_GYRO_driver_HL.o
 .text.LSM6DSM_X_Init
                0x08006294       0x78 Drivers/BSP/Components/LSM6DSM_ACC_GYRO_driver_HL.o
 .text.LSM6DSM_G_Init
                0x0800630c       0x78 Drivers/BSP/Components/LSM6DSM_ACC_GYRO_driver_HL.o
 .text.LSM6DSM_X_Enable_6D_Orientation
                0x08006384       0x7c Drivers/BSP/Components/LSM6DSM_ACC_GYRO_driver_HL.o
 .text.LSM6DSM_X_Get_Axes
                0x08006400       0xdc Drivers/BSP/Components/LSM6DSM_ACC_GYRO_driver_HL.o
 .text.LSM6DSM_X_Enable_Free_Fall_Detection
                0x080064dc       0xac Drivers/BSP/Components/LSM6DSM_ACC_GYRO_driver_HL.o
 .text.LSM6DSM_X_Enable_Wake_Up_Detection
                0x08006588       0x88 Drivers/BSP/Components/LSM6DSM_ACC_GYRO_driver_HL.o
 .text.LSM6DSM_X_Enable_Single_Tap_Detection
                0x08006610       0xb8 Drivers/BSP/Components/LSM6DSM_ACC_GYRO_driver_HL.o
 .text.LSM6DSM_G_Sensor_Disable
                0x080066c8       0xe0 Drivers/BSP/Components/LSM6DSM_ACC_GYRO_driver_HL.o
 .text.LSM6DSM_X_Sensor_Disable
                0x080067a8       0xe0 Drivers/BSP/Components/LSM6DSM_ACC_GYRO_driver_HL.o
 .text.LSM6DSM_G_DeInit
                0x08006888      0x10c Drivers/BSP/Components/LSM6DSM_ACC_GYRO_driver_HL.o
 .text.LSM6DSM_X_DeInit
                0x08006994      0x168 Drivers/BSP/Components/LSM6DSM_ACC_GYRO_driver_HL.o
 .text.I2C_SENSORTILE_Init
                0x08006afc       0xd0 Drivers/BSP/SensorTile/SensorTile.o
 .text.BSP_LED_Init
                0x08006bcc       0x7c Drivers/BSP/SensorTile/SensorTile.o
                0x08006bcc                BSP_LED_Init
 .text.Sensor_IO_SPI_Init
                0x08006c48       0xd0 Drivers/BSP/SensorTile/SensorTile.o
                0x08006c48                Sensor_IO_SPI_Init
 .text.Sensor_IO_SPI_CS_Init_All
                0x08006d18      0x10c Drivers/BSP/SensorTile/SensorTile.o
                0x08006d18                Sensor_IO_SPI_CS_Init_All
 .text.Sensor_IO_SPI_CS_Init
                0x08006e24       0xec Drivers/BSP/SensorTile/SensorTile.o
                0x08006e24                Sensor_IO_SPI_CS_Init
 .text.Sensor_IO_SPI_Write
                0x08006f10       0xe0 Drivers/BSP/SensorTile/SensorTile.o
                0x08006f10                Sensor_IO_SPI_Write
 .text.Sensor_IO_Write
                0x08006ff0       0x74 Drivers/BSP/SensorTile/SensorTile.o
                0x08006ff0                Sensor_IO_Write
 .text.Sensor_IO_SPI_Read
                0x08007064      0x174 Drivers/BSP/SensorTile/SensorTile.o
                0x08007064                Sensor_IO_SPI_Read
 .text.Sensor_IO_Read
                0x080071d8       0x74 Drivers/BSP/SensorTile/SensorTile.o
                0x080071d8                Sensor_IO_Read
 .text.LSM6DSM_Sensor_IO_ITConfig
                0x0800724c       0x54 Drivers/BSP/SensorTile/SensorTile.o
                0x0800724c                LSM6DSM_Sensor_IO_ITConfig
 .text.HAL_SPI_MspInit
                0x080072a0      0x158 Drivers/BSP/SensorTile/SensorTile_BlueNRG.o
                0x080072a0                HAL_SPI_MspInit
 .text.BNRG_SPI_Init
                0x080073f8       0x40 Drivers/BSP/SensorTile/SensorTile_BlueNRG.o
                0x080073f8                BNRG_SPI_Init
 .text.BlueNRG_RST
                0x08007438       0x2c Drivers/BSP/SensorTile/SensorTile_BlueNRG.o
                0x08007438                BlueNRG_RST
 .text.BlueNRG_DataPresent
                0x08007464       0x1c Drivers/BSP/SensorTile/SensorTile_BlueNRG.o
                0x08007464                BlueNRG_DataPresent
 .text.BlueNRG_SPI_Read_All
                0x08007480       0xb8 Drivers/BSP/SensorTile/SensorTile_BlueNRG.o
                0x08007480                BlueNRG_SPI_Read_All
 .text.BlueNRG_SPI_Write
                0x08007538       0xb4 Drivers/BSP/SensorTile/SensorTile_BlueNRG.o
                0x08007538                BlueNRG_SPI_Write
 .text.Hal_Write_Serial
                0x080075ec       0x44 Drivers/BSP/SensorTile/SensorTile_BlueNRG.o
                0x080075ec                Hal_Write_Serial
 .text.Enable_SPI_IRQ
                0x08007630        0x8 Drivers/BSP/SensorTile/SensorTile_BlueNRG.o
                0x08007630                Enable_SPI_IRQ
 .text.Disable_SPI_IRQ
                0x08007638        0x8 Drivers/BSP/SensorTile/SensorTile_BlueNRG.o
                0x08007638                Disable_SPI_IRQ
 .text.Clear_SPI_EXTI_Flag
                0x08007640        0xc Drivers/BSP/SensorTile/SensorTile_BlueNRG.o
                0x08007640                Clear_SPI_EXTI_Flag
 .text.BSP_ACCELERO_Init
                0x0800764c      0x24c Drivers/BSP/SensorTile/SensorTile_accelero.o
                0x0800764c                BSP_ACCELERO_Init
 .text.BSP_ACCELERO_Sensor_Enable
                0x08007898       0x20 Drivers/BSP/SensorTile/SensorTile_accelero.o
                0x08007898                BSP_ACCELERO_Sensor_Enable
 .text.SystemInit
                0x080078b8       0x50 Drivers/CMSIS/system_stm32l4xx.o
                0x080078b8                SystemInit
 .text.HAL_MspInit
                0x08007908        0x4 Drivers/STM32L4xx_HAL_Driver/stm32l4xx_hal.o
                0x08007908                HAL_MspInit
 .text.HAL_InitTick
                0x0800790c       0x2c Drivers/STM32L4xx_HAL_Driver/stm32l4xx_hal.o
                0x0800790c                HAL_InitTick
 .text.HAL_Init
                0x08007938       0x18 Drivers/STM32L4xx_HAL_Driver/stm32l4xx_hal.o
                0x08007938                HAL_Init
 .text.HAL_IncTick
                0x08007950       0x10 Drivers/STM32L4xx_HAL_Driver/stm32l4xx_hal.o
                0x08007950                HAL_IncTick
 .text.HAL_GetTick
                0x08007960        0xc Drivers/STM32L4xx_HAL_Driver/stm32l4xx_hal.o
                0x08007960                HAL_GetTick
 .text.HAL_Delay
                0x0800796c       0x1c Drivers/STM32L4xx_HAL_Driver/stm32l4xx_hal.o
                0x0800796c                HAL_Delay
 .text.HAL_GetHalVersion
                0x08007988        0x8 Drivers/STM32L4xx_HAL_Driver/stm32l4xx_hal.o
                0x08007988                HAL_GetHalVersion
 .text.HAL_NVIC_SetPriorityGrouping
                0x08007990       0x24 Drivers/STM32L4xx_HAL_Driver/stm32l4xx_hal_cortex.o
                0x08007990                HAL_NVIC_SetPriorityGrouping
 .text.HAL_NVIC_SetPriority
                0x080079b4       0x6c Drivers/STM32L4xx_HAL_Driver/stm32l4xx_hal_cortex.o
                0x080079b4                HAL_NVIC_SetPriority
 .text.HAL_NVIC_EnableIRQ
                0x08007a20       0x1c Drivers/STM32L4xx_HAL_Driver/stm32l4xx_hal_cortex.o
                0x08007a20                HAL_NVIC_EnableIRQ
 .text.HAL_NVIC_DisableIRQ
                0x08007a3c       0x28 Drivers/STM32L4xx_HAL_Driver/stm32l4xx_hal_cortex.o
                0x08007a3c                HAL_NVIC_DisableIRQ
 .text.HAL_SYSTICK_Config
                0x08007a64       0x34 Drivers/STM32L4xx_HAL_Driver/stm32l4xx_hal_cortex.o
                0x08007a64                HAL_SYSTICK_Config
 .text.HAL_DMA_IRQHandler
                0x08007a98       0x9c Drivers/STM32L4xx_HAL_Driver/stm32l4xx_hal_dma.o
                0x08007a98                HAL_DMA_IRQHandler
 .text.HAL_GPIO_Init
                0x08007b34      0x228 Drivers/STM32L4xx_HAL_Driver/stm32l4xx_hal_gpio.o
                0x08007b34                HAL_GPIO_Init
 .text.HAL_GPIO_ReadPin
                0x08007d5c        0xc Drivers/STM32L4xx_HAL_Driver/stm32l4xx_hal_gpio.o
                0x08007d5c                HAL_GPIO_ReadPin
 .text.HAL_GPIO_WritePin
                0x08007d68        0xc Drivers/STM32L4xx_HAL_Driver/stm32l4xx_hal_gpio.o
                0x08007d68                HAL_GPIO_WritePin
 .text.HAL_GPIO_EXTI_IRQHandler
                0x08007d74       0x18 Drivers/STM32L4xx_HAL_Driver/stm32l4xx_hal_gpio.o
                0x08007d74                HAL_GPIO_EXTI_IRQHandler
 .text.I2C_WaitOnTXISFlagUntilTimeout
                0x08007d8c       0xc4 Drivers/STM32L4xx_HAL_Driver/stm32l4xx_hal_i2c.o
 .text.I2C_WaitOnSTOPFlagUntilTimeout
                0x08007e50       0xc8 Drivers/STM32L4xx_HAL_Driver/stm32l4xx_hal_i2c.o
 .text.HAL_I2C_MspInit
                0x08007f18        0x4 Drivers/STM32L4xx_HAL_Driver/stm32l4xx_hal_i2c.o
                0x08007f18                HAL_I2C_MspInit
 .text.HAL_I2C_Init
                0x08007f1c       0xa8 Drivers/STM32L4xx_HAL_Driver/stm32l4xx_hal_i2c.o
                0x08007f1c                HAL_I2C_Init
 .text.HAL_I2C_MspDeInit
                0x08007fc4        0x4 Drivers/STM32L4xx_HAL_Driver/stm32l4xx_hal_i2c.o
                0x08007fc4                HAL_I2C_MspDeInit
 .text.HAL_I2C_DeInit
                0x08007fc8       0x34 Drivers/STM32L4xx_HAL_Driver/stm32l4xx_hal_i2c.o
                0x08007fc8                HAL_I2C_DeInit
 .text.HAL_I2C_Mem_Write
                0x08007ffc      0x258 Drivers/STM32L4xx_HAL_Driver/stm32l4xx_hal_i2c.o
                0x08007ffc                HAL_I2C_Mem_Write
 .text.HAL_I2C_Mem_Read
                0x08008254      0x254 Drivers/STM32L4xx_HAL_Driver/stm32l4xx_hal_i2c.o
                0x08008254                HAL_I2C_Mem_Read
 .text.HAL_I2C_GetState
                0x080084a8        0x8 Drivers/STM32L4xx_HAL_Driver/stm32l4xx_hal_i2c.o
                0x080084a8                HAL_I2C_GetState
 .text.HAL_PCD_Init
                0x080084b0      0x440 Drivers/STM32L4xx_HAL_Driver/stm32l4xx_hal_pcd.o
                0x080084b0                HAL_PCD_Init
 .text.HAL_PCD_Start
                0x080088f0       0x2c Drivers/STM32L4xx_HAL_Driver/stm32l4xx_hal_pcd.o
                0x080088f0                HAL_PCD_Start
 .text.HAL_PCD_IRQHandler
                0x0800891c      0x6f4 Drivers/STM32L4xx_HAL_Driver/stm32l4xx_hal_pcd.o
                0x0800891c                HAL_PCD_IRQHandler
 .text.HAL_PCD_SetAddress
                0x08009010       0x28 Drivers/STM32L4xx_HAL_Driver/stm32l4xx_hal_pcd.o
                0x08009010                HAL_PCD_SetAddress
 .text.HAL_PCD_EP_Open
                0x08009038       0x4c Drivers/STM32L4xx_HAL_Driver/stm32l4xx_hal_pcd.o
                0x08009038                HAL_PCD_EP_Open
 .text.HAL_PCD_EP_Close
                0x08009084       0x54 Drivers/STM32L4xx_HAL_Driver/stm32l4xx_hal_pcd.o
                0x08009084                HAL_PCD_EP_Close
 .text.HAL_PCD_EP_Receive
                0x080090d8       0x44 Drivers/STM32L4xx_HAL_Driver/stm32l4xx_hal_pcd.o
                0x080090d8                HAL_PCD_EP_Receive
 .text.HAL_PCD_EP_GetRxCount
                0x0800911c       0x14 Drivers/STM32L4xx_HAL_Driver/stm32l4xx_hal_pcd.o
                0x0800911c                HAL_PCD_EP_GetRxCount
 .text.HAL_PCD_EP_Transmit
                0x08009130       0x40 Drivers/STM32L4xx_HAL_Driver/stm32l4xx_hal_pcd.o
                0x08009130                HAL_PCD_EP_Transmit
 .text.HAL_PCD_EP_SetStall
                0x08009170       0x60 Drivers/STM32L4xx_HAL_Driver/stm32l4xx_hal_pcd.o
                0x08009170                HAL_PCD_EP_SetStall
 .text.HAL_PCD_EP_ClrStall
                0x080091d0       0x4c Drivers/STM32L4xx_HAL_Driver/stm32l4xx_hal_pcd.o
                0x080091d0                HAL_PCD_EP_ClrStall
 .text.HAL_PCDEx_SetTxFiFo
                0x0800921c       0x48 Drivers/STM32L4xx_HAL_Driver/stm32l4xx_hal_pcd_ex.o
                0x0800921c                HAL_PCDEx_SetTxFiFo
 .text.HAL_PCDEx_SetRxFiFo
                0x08009264        0x8 Drivers/STM32L4xx_HAL_Driver/stm32l4xx_hal_pcd_ex.o
                0x08009264                HAL_PCDEx_SetRxFiFo
 .text.HAL_PCDEx_ActivateLPM
                0x0800926c       0x28 Drivers/STM32L4xx_HAL_Driver/stm32l4xx_hal_pcd_ex.o
                0x0800926c                HAL_PCDEx_ActivateLPM
 .text.HAL_PCDEx_ActivateBCD
                0x08009294       0x14 Drivers/STM32L4xx_HAL_Driver/stm32l4xx_hal_pcd_ex.o
                0x08009294                HAL_PCDEx_ActivateBCD
 .text.HAL_PCDEx_LPM_Callback
                0x080092a8        0x4 Drivers/STM32L4xx_HAL_Driver/stm32l4xx_hal_pcd_ex.o
                0x080092a8                HAL_PCDEx_LPM_Callback
 .text.HAL_PWR_EnableBkUpAccess
                0x080092ac       0x10 Drivers/STM32L4xx_HAL_Driver/stm32l4xx_hal_pwr.o
                0x080092ac                HAL_PWR_EnableBkUpAccess
 .text.HAL_PWREx_GetVoltageRange
                0x080092bc       0x10 Drivers/STM32L4xx_HAL_Driver/stm32l4xx_hal_pwr_ex.o
                0x080092bc                HAL_PWREx_GetVoltageRange
 .text.HAL_PWREx_EnableVddUSB
                0x080092cc       0x10 Drivers/STM32L4xx_HAL_Driver/stm32l4xx_hal_pwr_ex.o
                0x080092cc                HAL_PWREx_EnableVddUSB
 .text.HAL_PWREx_EnableVddIO2
                0x080092dc       0x10 Drivers/STM32L4xx_HAL_Driver/stm32l4xx_hal_pwr_ex.o
                0x080092dc                HAL_PWREx_EnableVddIO2
 .text.HAL_RCC_GetSysClockFreq
                0x080092ec      0x164 Drivers/STM32L4xx_HAL_Driver/stm32l4xx_hal_rcc.o
                0x080092ec                HAL_RCC_GetSysClockFreq
 .text.HAL_RCC_OscConfig
                0x08009450      0x620 Drivers/STM32L4xx_HAL_Driver/stm32l4xx_hal_rcc.o
                0x08009450                HAL_RCC_OscConfig
 .text.HAL_RCC_ClockConfig
                0x08009a70      0x180 Drivers/STM32L4xx_HAL_Driver/stm32l4xx_hal_rcc.o
                0x08009a70                HAL_RCC_ClockConfig
 .text.HAL_RCC_GetHCLKFreq
                0x08009bf0        0xc Drivers/STM32L4xx_HAL_Driver/stm32l4xx_hal_rcc.o
                0x08009bf0                HAL_RCC_GetHCLKFreq
 .text.RCCEx_PLLSAI1_Config
                0x08009bfc      0x188 Drivers/STM32L4xx_HAL_Driver/stm32l4xx_hal_rcc_ex.o
 .text.RCCEx_PLLSAI2_Config
                0x08009d84      0x14c Drivers/STM32L4xx_HAL_Driver/stm32l4xx_hal_rcc_ex.o
 .text.HAL_RCCEx_PeriphCLKConfig
                0x08009ed0      0x420 Drivers/STM32L4xx_HAL_Driver/stm32l4xx_hal_rcc_ex.o
                0x08009ed0                HAL_RCCEx_PeriphCLKConfig
 .text.HAL_RCCEx_DisableLSECSS
                0x0800a2f0       0x1c Drivers/STM32L4xx_HAL_Driver/stm32l4xx_hal_rcc_ex.o
                0x0800a2f0                HAL_RCCEx_DisableLSECSS
 .text.HAL_RCCEx_EnableMSIPLLMode
                0x0800a30c       0x10 Drivers/STM32L4xx_HAL_Driver/stm32l4xx_hal_rcc_ex.o
                0x0800a30c                HAL_RCCEx_EnableMSIPLLMode
 .text.unlikely.SPI_WaitFlagStateUntilTimeout
                0x0800a31c       0x8a Drivers/STM32L4xx_HAL_Driver/stm32l4xx_hal_spi.o
 *fill*         0x0800a3a6        0x2 
 .text.SPI_EndRxTxTransaction
                0x0800a3a8       0xe8 Drivers/STM32L4xx_HAL_Driver/stm32l4xx_hal_spi.o
 .text.HAL_SPI_Init
                0x0800a490       0xe4 Drivers/STM32L4xx_HAL_Driver/stm32l4xx_hal_spi.o
                0x0800a490                HAL_SPI_Init
 .text.HAL_SPI_TransmitReceive
                0x0800a574      0x430 Drivers/STM32L4xx_HAL_Driver/stm32l4xx_hal_spi.o
                0x0800a574                HAL_SPI_TransmitReceive
 .text.HAL_SPI_GetState
                0x0800a9a4        0x8 Drivers/STM32L4xx_HAL_Driver/stm32l4xx_hal_spi.o
                0x0800a9a4                HAL_SPI_GetState
 .text.HAL_TIM_Base_Init
                0x0800a9ac       0xfc Drivers/STM32L4xx_HAL_Driver/stm32l4xx_hal_tim.o
                0x0800a9ac                HAL_TIM_Base_Init
 .text.HAL_TIM_Base_Start_IT
                0x0800aaa8       0x18 Drivers/STM32L4xx_HAL_Driver/stm32l4xx_hal_tim.o
                0x0800aaa8                HAL_TIM_Base_Start_IT
 .text.HAL_TIM_OC_DelayElapsedCallback
                0x0800aac0        0x4 Drivers/STM32L4xx_HAL_Driver/stm32l4xx_hal_tim.o
                0x0800aac0                HAL_TIM_OC_DelayElapsedCallback
 .text.HAL_TIM_IC_CaptureCallback
                0x0800aac4        0x4 Drivers/STM32L4xx_HAL_Driver/stm32l4xx_hal_tim.o
                0x0800aac4                HAL_TIM_IC_CaptureCallback
 .text.HAL_TIM_PWM_PulseFinishedCallback
                0x0800aac8        0x4 Drivers/STM32L4xx_HAL_Driver/stm32l4xx_hal_tim.o
                0x0800aac8                HAL_TIM_PWM_PulseFinishedCallback
 .text.HAL_TIM_TriggerCallback
                0x0800aacc        0x4 Drivers/STM32L4xx_HAL_Driver/stm32l4xx_hal_tim.o
                0x0800aacc                HAL_TIM_TriggerCallback
 .text.HAL_TIM_IRQHandler
                0x0800aad0      0x154 Drivers/STM32L4xx_HAL_Driver/stm32l4xx_hal_tim.o
                0x0800aad0                HAL_TIM_IRQHandler
 .text.HAL_TIMEx_CommutationCallback
                0x0800ac24        0x4 Drivers/STM32L4xx_HAL_Driver/stm32l4xx_hal_tim_ex.o
                0x0800ac24                HAL_TIMEx_CommutationCallback
 .text.HAL_TIMEx_BreakCallback
                0x0800ac28        0x4 Drivers/STM32L4xx_HAL_Driver/stm32l4xx_hal_tim_ex.o
                0x0800ac28                HAL_TIMEx_BreakCallback
 .text.USB_CoreInit
                0x0800ac2c       0x28 Drivers/STM32L4xx_HAL_Driver/stm32l4xx_ll_usb.o
                0x0800ac2c                USB_CoreInit
 .text.USB_EnableGlobalInt
                0x0800ac54       0x10 Drivers/STM32L4xx_HAL_Driver/stm32l4xx_ll_usb.o
                0x0800ac54                USB_EnableGlobalInt
 .text.USB_DisableGlobalInt
                0x0800ac64       0x10 Drivers/STM32L4xx_HAL_Driver/stm32l4xx_ll_usb.o
                0x0800ac64                USB_DisableGlobalInt
 .text.USB_SetCurrentMode
                0x0800ac74       0x34 Drivers/STM32L4xx_HAL_Driver/stm32l4xx_ll_usb.o
                0x0800ac74                USB_SetCurrentMode
 .text.USB_DevInit
                0x0800aca8      0x15c Drivers/STM32L4xx_HAL_Driver/stm32l4xx_ll_usb.o
                0x0800aca8                USB_DevInit
 .text.USB_FlushTxFifo
                0x0800ae04       0x24 Drivers/STM32L4xx_HAL_Driver/stm32l4xx_ll_usb.o
                0x0800ae04                USB_FlushTxFifo
 .text.USB_ActivateEndpoint
                0x0800ae28       0x80 Drivers/STM32L4xx_HAL_Driver/stm32l4xx_ll_usb.o
                0x0800ae28                USB_ActivateEndpoint
 .text.USB_DeactivateEndpoint
                0x0800aea8       0x50 Drivers/STM32L4xx_HAL_Driver/stm32l4xx_ll_usb.o
                0x0800aea8                USB_DeactivateEndpoint
 .text.USB_EPStartXfer
                0x0800aef8      0x1a4 Drivers/STM32L4xx_HAL_Driver/stm32l4xx_ll_usb.o
                0x0800aef8                USB_EPStartXfer
 .text.USB_EP0StartXfer
                0x0800b09c       0xe4 Drivers/STM32L4xx_HAL_Driver/stm32l4xx_ll_usb.o
                0x0800b09c                USB_EP0StartXfer
 .text.USB_WritePacket
                0x0800b180       0x2c Drivers/STM32L4xx_HAL_Driver/stm32l4xx_ll_usb.o
                0x0800b180                USB_WritePacket
 .text.USB_ReadPacket
                0x0800b1ac       0x28 Drivers/STM32L4xx_HAL_Driver/stm32l4xx_ll_usb.o
                0x0800b1ac                USB_ReadPacket
 .text.USB_EPSetStall
                0x0800b1d4       0x38 Drivers/STM32L4xx_HAL_Driver/stm32l4xx_ll_usb.o
                0x0800b1d4                USB_EPSetStall
 .text.USB_EPClearStall
                0x0800b20c       0x30 Drivers/STM32L4xx_HAL_Driver/stm32l4xx_ll_usb.o
                0x0800b20c                USB_EPClearStall
 .text.USB_SetDevAddress
                0x0800b23c       0x20 Drivers/STM32L4xx_HAL_Driver/stm32l4xx_ll_usb.o
                0x0800b23c                USB_SetDevAddress
 .text.USB_DevConnect
                0x0800b25c       0x18 Drivers/STM32L4xx_HAL_Driver/stm32l4xx_ll_usb.o
                0x0800b25c                USB_DevConnect
 .text.USB_DevDisconnect
                0x0800b274       0x18 Drivers/STM32L4xx_HAL_Driver/stm32l4xx_ll_usb.o
                0x0800b274                USB_DevDisconnect
 .text.USB_ReadInterrupts
                0x0800b28c        0x8 Drivers/STM32L4xx_HAL_Driver/stm32l4xx_ll_usb.o
                0x0800b28c                USB_ReadInterrupts
 .text.USB_ReadDevAllOutEpInterrupt
                0x0800b294       0x10 Drivers/STM32L4xx_HAL_Driver/stm32l4xx_ll_usb.o
                0x0800b294                USB_ReadDevAllOutEpInterrupt
 .text.USB_ReadDevAllInEpInterrupt
                0x0800b2a4       0x10 Drivers/STM32L4xx_HAL_Driver/stm32l4xx_ll_usb.o
                0x0800b2a4                USB_ReadDevAllInEpInterrupt
 .text.USB_ReadDevOutEPInterrupt
                0x0800b2b4       0x14 Drivers/STM32L4xx_HAL_Driver/stm32l4xx_ll_usb.o
                0x0800b2b4                USB_ReadDevOutEPInterrupt
 .text.USB_ReadDevInEPInterrupt
                0x0800b2c8       0x24 Drivers/STM32L4xx_HAL_Driver/stm32l4xx_ll_usb.o
                0x0800b2c8                USB_ReadDevInEPInterrupt
 .text.USB_GetMode
                0x0800b2ec        0x8 Drivers/STM32L4xx_HAL_Driver/stm32l4xx_ll_usb.o
                0x0800b2ec                USB_GetMode
 .text.USB_ActivateSetup
                0x0800b2f4       0x38 Drivers/STM32L4xx_HAL_Driver/stm32l4xx_ll_usb.o
                0x0800b2f4                USB_ActivateSetup
 .text.USB_EP0_OutStart
                0x0800b32c       0x24 Drivers/STM32L4xx_HAL_Driver/stm32l4xx_ll_usb.o
                0x0800b32c                USB_EP0_OutStart
 .text.USB_CoreReset
                0x0800b350       0x68 Drivers/STM32L4xx_HAL_Driver/stm32l4xx_ll_usb.o
 .text.Reset_Handler
                0x0800b3b8       0x50 Example/SW4STM32/startup_stm32l476xx.o
                0x0800b3b8                Reset_Handler
 .text.Default_Handler
                0x0800b408        0x2 Example/SW4STM32/startup_stm32l476xx.o
                0x0800b408                RTC_Alarm_IRQHandler
                0x0800b408                TIM8_TRG_COM_IRQHandler
                0x0800b408                TIM8_CC_IRQHandler
                0x0800b408                TSC_IRQHandler
                0x0800b408                TAMP_STAMP_IRQHandler
                0x0800b408                EXTI3_IRQHandler
                0x0800b408                LPTIM2_IRQHandler
                0x0800b408                DFSDM1_FLT1_IRQHandler
                0x0800b408                I2C3_ER_IRQHandler
                0x0800b408                DFSDM1_FLT2_IRQHandler
                0x0800b408                EXTI0_IRQHandler
                0x0800b408                I2C2_EV_IRQHandler
                0x0800b408                CAN1_RX0_IRQHandler
                0x0800b408                FPU_IRQHandler
                0x0800b408                TIM1_UP_TIM16_IRQHandler
                0x0800b408                ADC1_2_IRQHandler
                0x0800b408                SPI1_IRQHandler
                0x0800b408                TIM6_DAC_IRQHandler
                0x0800b408                TIM8_UP_IRQHandler
                0x0800b408                DMA1_Channel4_IRQHandler
                0x0800b408                SAI2_IRQHandler
                0x0800b408                DFSDM1_FLT3_IRQHandler
                0x0800b408                USART3_IRQHandler
                0x0800b408                DMA1_Channel7_IRQHandler
                0x0800b408                CAN1_RX1_IRQHandler
                0x0800b408                LCD_IRQHandler
                0x0800b408                UART5_IRQHandler
                0x0800b408                ADC3_IRQHandler
                0x0800b408                TIM4_IRQHandler
                0x0800b408                DMA2_Channel1_IRQHandler
                0x0800b408                QUADSPI_IRQHandler
                0x0800b408                I2C1_EV_IRQHandler
                0x0800b408                DMA1_Channel6_IRQHandler
                0x0800b408                UART4_IRQHandler
                0x0800b408                DMA2_Channel4_IRQHandler
                0x0800b408                RCC_IRQHandler
                0x0800b408                DMA1_Channel1_IRQHandler
                0x0800b408                Default_Handler
                0x0800b408                DMA2_Channel7_IRQHandler
                0x0800b408                EXTI15_10_IRQHandler
                0x0800b408                TIM7_IRQHandler
                0x0800b408                SDMMC1_IRQHandler
                0x0800b408                TIM5_IRQHandler
                0x0800b408                I2C3_EV_IRQHandler
                0x0800b408                RTC_WKUP_IRQHandler
                0x0800b408                PVD_PVM_IRQHandler
                0x0800b408                SPI2_IRQHandler
                0x0800b408                CAN1_TX_IRQHandler
                0x0800b408                DMA2_Channel5_IRQHandler
                0x0800b408                DMA1_Channel5_IRQHandler
                0x0800b408                EXTI4_IRQHandler
                0x0800b408                RNG_IRQHandler
                0x0800b408                TIM1_TRG_COM_TIM17_IRQHandler
                0x0800b408                DMA1_Channel3_IRQHandler
                0x0800b408                COMP_IRQHandler
                0x0800b408                WWDG_IRQHandler
                0x0800b408                LPUART1_IRQHandler
                0x0800b408                DMA2_Channel6_IRQHandler
                0x0800b408                TIM2_IRQHandler
                0x0800b408                EXTI1_IRQHandler
                0x0800b408                USART2_IRQHandler
                0x0800b408                DFSDM1_FLT0_IRQHandler
                0x0800b408                I2C2_ER_IRQHandler
                0x0800b408                DMA1_Channel2_IRQHandler
                0x0800b408                TIM8_BRK_IRQHandler
                0x0800b408                CAN1_SCE_IRQHandler
                0x0800b408                FLASH_IRQHandler
                0x0800b408                USART1_IRQHandler
                0x0800b408                SPI3_IRQHandler
                0x0800b408                I2C1_ER_IRQHandler
                0x0800b408                FMC_IRQHandler
                0x0800b408                SWPMI1_IRQHandler
                0x0800b408                LPTIM1_IRQHandler
                0x0800b408                SAI1_IRQHandler
                0x0800b408                DMA2_Channel3_IRQHandler
                0x0800b408                TIM1_BRK_TIM15_IRQHandler
 *fill*         0x0800b40a        0x2 
 .text.osKernelStart
                0x0800b40c        0xc Middlewares/FreeRTOS/CMSIS_RTOS/cmsis_os.o
                0x0800b40c                osKernelStart
 .text.osKernelSysTick
                0x0800b418       0x10 Middlewares/FreeRTOS/CMSIS_RTOS/cmsis_os.o
                0x0800b418                osKernelSysTick
 .text.osThreadCreate
                0x0800b428       0x30 Middlewares/FreeRTOS/CMSIS_RTOS/cmsis_os.o
                0x0800b428                osThreadCreate
 .text.osDelay  0x0800b458       0x10 Middlewares/FreeRTOS/CMSIS_RTOS/cmsis_os.o
                0x0800b458                osDelay
 .text.osTimerCreate
                0x0800b468       0x28 Middlewares/FreeRTOS/CMSIS_RTOS/cmsis_os.o
                0x0800b468                osTimerCreate
 .text.osTimerStart
                0x0800b490       0x5c Middlewares/FreeRTOS/CMSIS_RTOS/cmsis_os.o
                0x0800b490                osTimerStart
 .text.osTimerStop
                0x0800b4ec       0x58 Middlewares/FreeRTOS/CMSIS_RTOS/cmsis_os.o
                0x0800b4ec                osTimerStop
 .text.osSemaphoreCreate
                0x0800b544       0x28 Middlewares/FreeRTOS/CMSIS_RTOS/cmsis_os.o
                0x0800b544                osSemaphoreCreate
 .text.osSemaphoreWait
                0x0800b56c       0x5c Middlewares/FreeRTOS/CMSIS_RTOS/cmsis_os.o
                0x0800b56c                osSemaphoreWait
 .text.osSemaphoreRelease
                0x0800b5c8       0x50 Middlewares/FreeRTOS/CMSIS_RTOS/cmsis_os.o
                0x0800b5c8                osSemaphoreRelease
 .text.osPoolCreate
                0x0800b618       0x74 Middlewares/FreeRTOS/CMSIS_RTOS/cmsis_os.o
                0x0800b618                osPoolCreate
 .text.osPoolAlloc
                0x0800b68c       0x90 Middlewares/FreeRTOS/CMSIS_RTOS/cmsis_os.o
                0x0800b68c                osPoolAlloc
 .text.osPoolFree
                0x0800b71c       0x2c Middlewares/FreeRTOS/CMSIS_RTOS/cmsis_os.o
                0x0800b71c                osPoolFree
 .text.osMessageCreate
                0x0800b748        0xc Middlewares/FreeRTOS/CMSIS_RTOS/cmsis_os.o
                0x0800b748                osMessageCreate
 .text.osMessagePut
                0x0800b754       0x58 Middlewares/FreeRTOS/CMSIS_RTOS/cmsis_os.o
                0x0800b754                osMessagePut
 .text.osMessageGet
                0x0800b7ac       0x8c Middlewares/FreeRTOS/CMSIS_RTOS/cmsis_os.o
                0x0800b7ac                osMessageGet
 .text.osSystickHandler
                0x0800b838       0x14 Middlewares/FreeRTOS/CMSIS_RTOS/cmsis_os.o
                0x0800b838                osSystickHandler
 .text.osThreadSuspend
                0x0800b84c        0xc Middlewares/FreeRTOS/CMSIS_RTOS/cmsis_os.o
                0x0800b84c                osThreadSuspend
 .text.osThreadResume
                0x0800b858       0x34 Middlewares/FreeRTOS/CMSIS_RTOS/cmsis_os.o
                0x0800b858                osThreadResume
 .text.vListInitialise
                0x0800b88c       0x18 Middlewares/FreeRTOS/list.o
                0x0800b88c                vListInitialise
 .text.vListInitialiseItem
                0x0800b8a4        0x8 Middlewares/FreeRTOS/list.o
                0x0800b8a4                vListInitialiseItem
 .text.vListInsertEnd
                0x0800b8ac       0x20 Middlewares/FreeRTOS/list.o
                0x0800b8ac                vListInsertEnd
 .text.vListInsert
                0x0800b8cc       0x34 Middlewares/FreeRTOS/list.o
                0x0800b8cc                vListInsert
 .text.uxListRemove
                0x0800b900       0x28 Middlewares/FreeRTOS/list.o
                0x0800b900                uxListRemove
 .text.xQueueGenericCreate
                0x0800b928       0x90 Middlewares/FreeRTOS/queue.o
                0x0800b928                xQueueGenericCreate
 .text.xQueueCreateCountingSemaphore
                0x0800b9b8       0x3c Middlewares/FreeRTOS/queue.o
                0x0800b9b8                xQueueCreateCountingSemaphore
 .text.xQueueGenericSend
                0x0800b9f4      0x37c Middlewares/FreeRTOS/queue.o
                0x0800b9f4                xQueueGenericSend
 .text.xQueueGenericSendFromISR
                0x0800bd70      0x12c Middlewares/FreeRTOS/queue.o
                0x0800bd70                xQueueGenericSendFromISR
 .text.xQueueGiveFromISR
                0x0800be9c       0xac Middlewares/FreeRTOS/queue.o
                0x0800be9c                xQueueGiveFromISR
 .text.xQueueGenericReceive
                0x0800bf48      0x310 Middlewares/FreeRTOS/queue.o
                0x0800bf48                xQueueGenericReceive
 .text.xQueueReceiveFromISR
                0x0800c258       0xb4 Middlewares/FreeRTOS/queue.o
                0x0800c258                xQueueReceiveFromISR
 .text.vQueueAddToRegistry
                0x0800c30c       0x28 Middlewares/FreeRTOS/queue.o
                0x0800c30c                vQueueAddToRegistry
 .text.vQueueWaitForMessageRestricted
                0x0800c334       0xcc Middlewares/FreeRTOS/queue.o
                0x0800c334                vQueueWaitForMessageRestricted
 .text.prvResetNextTaskUnblockTime.part.2
                0x0800c400       0x14 Middlewares/FreeRTOS/tasks.o
 .text.prvAddCurrentTaskToDelayedList
                0x0800c414       0x6c Middlewares/FreeRTOS/tasks.o
 .text.xTaskCreate
                0x0800c480      0x234 Middlewares/FreeRTOS/tasks.o
                0x0800c480                xTaskCreate
 .text.vTaskSuspend
                0x0800c6b4      0x134 Middlewares/FreeRTOS/tasks.o
                0x0800c6b4                vTaskSuspend
 .text.vTaskResume
                0x0800c7e8       0x90 Middlewares/FreeRTOS/tasks.o
                0x0800c7e8                vTaskResume
 .text.xTaskResumeFromISR
                0x0800c878       0xa4 Middlewares/FreeRTOS/tasks.o
                0x0800c878                xTaskResumeFromISR
 .text.vTaskStartScheduler
                0x0800c91c      0x1b0 Middlewares/FreeRTOS/tasks.o
                0x0800c91c                vTaskStartScheduler
 .text.vTaskSuspendAll
                0x0800cacc       0x14 Middlewares/FreeRTOS/tasks.o
                0x0800cacc                vTaskSuspendAll
 .text.xTaskGetTickCount
                0x0800cae0        0xc Middlewares/FreeRTOS/tasks.o
                0x0800cae0                xTaskGetTickCount
 .text.xTaskGetTickCountFromISR
                0x0800caec       0x10 Middlewares/FreeRTOS/tasks.o
                0x0800caec                xTaskGetTickCountFromISR
 .text.vTaskStepTick
                0x0800cafc       0x2c Middlewares/FreeRTOS/tasks.o
                0x0800cafc                vTaskStepTick
 .text.xTaskIncrementTick
                0x0800cb28      0x100 Middlewares/FreeRTOS/tasks.o
                0x0800cb28                xTaskIncrementTick
 .text.xTaskResumeAll
                0x0800cc28       0xe4 Middlewares/FreeRTOS/tasks.o
                0x0800cc28                xTaskResumeAll
 .text.vTaskDelay
                0x0800cd0c       0x4c Middlewares/FreeRTOS/tasks.o
                0x0800cd0c                vTaskDelay
 .text.prvIdleTask
                0x0800cd58       0xd8 Middlewares/FreeRTOS/tasks.o
 .text.vTaskSwitchContext
                0x0800ce30       0x68 Middlewares/FreeRTOS/tasks.o
                0x0800ce30                vTaskSwitchContext
 .text.vTaskPlaceOnEventList
                0x0800ce98       0x84 Middlewares/FreeRTOS/tasks.o
                0x0800ce98                vTaskPlaceOnEventList
 .text.vTaskPlaceOnEventListRestricted
                0x0800cf1c       0x9c Middlewares/FreeRTOS/tasks.o
                0x0800cf1c                vTaskPlaceOnEventListRestricted
 .text.xTaskRemoveFromEventList
                0x0800cfb8       0x8c Middlewares/FreeRTOS/tasks.o
                0x0800cfb8                xTaskRemoveFromEventList
 .text.vTaskSetTimeOutState
                0x0800d044       0x28 Middlewares/FreeRTOS/tasks.o
                0x0800d044                vTaskSetTimeOutState
 .text.xTaskCheckForTimeOut
                0x0800d06c       0x78 Middlewares/FreeRTOS/tasks.o
                0x0800d06c                xTaskCheckForTimeOut
 .text.vTaskMissedYield
                0x0800d0e4       0x10 Middlewares/FreeRTOS/tasks.o
                0x0800d0e4                vTaskMissedYield
 .text.eTaskConfirmSleepModeStatus
                0x0800d0f4       0x28 Middlewares/FreeRTOS/tasks.o
                0x0800d0f4                eTaskConfirmSleepModeStatus
 .text.xTaskGetSchedulerState
                0x0800d11c       0x20 Middlewares/FreeRTOS/tasks.o
                0x0800d11c                xTaskGetSchedulerState
 .text.vTaskPriorityInherit
                0x0800d13c       0x8c Middlewares/FreeRTOS/tasks.o
                0x0800d13c                vTaskPriorityInherit
 .text.xTaskPriorityDisinherit
                0x0800d1c8       0xa4 Middlewares/FreeRTOS/tasks.o
                0x0800d1c8                xTaskPriorityDisinherit
 .text.pvTaskIncrementMutexHeldCount
                0x0800d26c       0x18 Middlewares/FreeRTOS/tasks.o
                0x0800d26c                pvTaskIncrementMutexHeldCount
 .text.prvSwitchTimerLists
                0x0800d284       0x88 Middlewares/FreeRTOS/timers.o
 .text.prvTimerTask
                0x0800d30c      0x238 Middlewares/FreeRTOS/timers.o
 .text.xTimerCreateTimerTask
                0x0800d544       0x88 Middlewares/FreeRTOS/timers.o
                0x0800d544                xTimerCreateTimerTask
 .text.xTimerCreate
                0x0800d5cc       0x94 Middlewares/FreeRTOS/timers.o
                0x0800d5cc                xTimerCreate
 .text.xTimerGenericCommand
                0x0800d660       0x64 Middlewares/FreeRTOS/timers.o
                0x0800d660                xTimerGenericCommand
 .text.unlikely.prvInsertBlockIntoFreeList
                0x0800d6c4       0x4c Middlewares/FreeRTOS/portable/heap_4.o
 .text.pvPortMalloc
                0x0800d710       0xf8 Middlewares/FreeRTOS/portable/heap_4.o
                0x0800d710                pvPortMalloc
 .text.vPortFree
                0x0800d808       0x68 Middlewares/FreeRTOS/portable/heap_4.o
                0x0800d808                vPortFree
 .text.prvTaskExitError
                0x0800d870       0x30 Middlewares/FreeRTOS/portable/port.o
 .text.prvPortStartFirstTask
                0x0800d8a0       0x20 Middlewares/FreeRTOS/portable/port.o
 .text.vPortEnableVFP
                0x0800d8c0       0x14 Middlewares/FreeRTOS/portable/port.o
 .text.pxPortInitialiseStack
                0x0800d8d4       0x2c Middlewares/FreeRTOS/portable/port.o
                0x0800d8d4                pxPortInitialiseStack
 .text.SVC_Handler
                0x0800d900       0x24 Middlewares/FreeRTOS/portable/port.o
                0x0800d900                SVC_Handler
 .text.vPortEnterCritical
                0x0800d924       0x44 Middlewares/FreeRTOS/portable/port.o
                0x0800d924                vPortEnterCritical
 .text.vPortExitCritical
                0x0800d968       0x28 Middlewares/FreeRTOS/portable/port.o
                0x0800d968                vPortExitCritical
 .text.PendSV_Handler
                0x0800d990       0x64 Middlewares/FreeRTOS/portable/port.o
                0x0800d990                PendSV_Handler
 .text.xPortSysTickHandler
                0x0800d9f4       0x2c Middlewares/FreeRTOS/portable/port.o
                0x0800d9f4                xPortSysTickHandler
 .text.vPortSuppressTicksAndSleep
                0x0800da20      0x154 Middlewares/FreeRTOS/portable/port.o
                0x0800da20                vPortSuppressTicksAndSleep
 .text.vPortSetupTimerInterrupt
                0x0800db74       0x44 Middlewares/FreeRTOS/portable/port.o
                0x0800db74                vPortSetupTimerInterrupt
 .text.xPortStartScheduler
                0x0800dbb8       0xec Middlewares/FreeRTOS/portable/port.o
                0x0800dbb8                xPortStartScheduler
 .text.vPortValidateInterruptPriority
                0x0800dca4       0x58 Middlewares/FreeRTOS/portable/port.o
                0x0800dca4                vPortValidateInterruptPriority
 .text.aci_gap_init_IDB05A1
                0x0800dcfc       0x7c Middlewares/STM32_BlueNRG/HCI/Controller/bluenrg_gap_aci.o
                0x0800dcfc                aci_gap_init_IDB05A1
 .text.aci_gap_init_IDB04A1
                0x0800dd78       0x78 Middlewares/STM32_BlueNRG/HCI/Controller/bluenrg_gap_aci.o
                0x0800dd78                aci_gap_init_IDB04A1
 .text.aci_gap_set_discoverable
                0x0800ddf0       0xd4 Middlewares/STM32_BlueNRG/HCI/Controller/bluenrg_gap_aci.o
                0x0800ddf0                aci_gap_set_discoverable
 .text.aci_gap_set_auth_requirement
                0x0800dec4       0x7c Middlewares/STM32_BlueNRG/HCI/Controller/bluenrg_gap_aci.o
                0x0800dec4                aci_gap_set_auth_requirement
 .text.aci_gap_update_adv_data
                0x0800df40       0x5c Middlewares/STM32_BlueNRG/HCI/Controller/bluenrg_gap_aci.o
                0x0800df40                aci_gap_update_adv_data
 .text.aci_gatt_init
                0x0800df9c       0x38 Middlewares/STM32_BlueNRG/HCI/Controller/bluenrg_gatt_aci.o
                0x0800df9c                aci_gatt_init
 .text.aci_gatt_add_serv
                0x0800dfd4       0x94 Middlewares/STM32_BlueNRG/HCI/Controller/bluenrg_gatt_aci.o
                0x0800dfd4                aci_gatt_add_serv
 .text.aci_gatt_add_char
                0x0800e068      0x114 Middlewares/STM32_BlueNRG/HCI/Controller/bluenrg_gatt_aci.o
                0x0800e068                aci_gatt_add_char
 .text.aci_gatt_update_char_value
                0x0800e17c       0x88 Middlewares/STM32_BlueNRG/HCI/Controller/bluenrg_gatt_aci.o
                0x0800e17c                aci_gatt_update_char_value
 .text.aci_gatt_allow_read
                0x0800e204       0x44 Middlewares/STM32_BlueNRG/HCI/Controller/bluenrg_gatt_aci.o
                0x0800e204                aci_gatt_allow_read
 .text.aci_hal_set_tx_power_level
                0x0800e248       0x48 Middlewares/STM32_BlueNRG/HCI/Controller/bluenrg_hal_aci.o
                0x0800e248                aci_hal_set_tx_power_level
 .text.getBlueNRGVersion
                0x0800e290       0x44 Middlewares/STM32_BlueNRG/HCI/Controller/bluenrg_utils.o
                0x0800e290                getBlueNRGVersion
 .text.HCI_Init
                0x0800e2d4       0x34 Middlewares/STM32_BlueNRG/HCI/hci.o
                0x0800e2d4                HCI_Init
 .text.HCI_Isr  0x0800e308       0x78 Middlewares/STM32_BlueNRG/HCI/hci.o
                0x0800e308                HCI_Isr
 .text.HCI_Process
                0x0800e380       0x58 Middlewares/STM32_BlueNRG/HCI/hci.o
                0x0800e380                HCI_Process
 .text.hci_send_req
                0x0800e3d8      0x1f0 Middlewares/STM32_BlueNRG/HCI/hci.o
                0x0800e3d8                hci_send_req
 .text.hci_le_read_local_version
                0x0800e5c8       0x88 Middlewares/STM32_BlueNRG/HCI/hci_le.o
                0x0800e5c8                hci_le_read_local_version
 .text.hci_le_set_scan_resp_data
                0x0800e650       0x64 Middlewares/STM32_BlueNRG/HCI/hci_le.o
                0x0800e650                hci_le_set_scan_resp_data
 .text.hci_le_set_random_address
                0x0800e6b4       0x54 Middlewares/STM32_BlueNRG/HCI/hci_le.o
                0x0800e6b4                hci_le_set_random_address
 .text.list_init_head
                0x0800e708        0x8 Middlewares/STM32_BlueNRG/Utils/ble_list.o
                0x0800e708                list_init_head
 .text.list_is_empty
                0x0800e710       0x18 Middlewares/STM32_BlueNRG/Utils/ble_list.o
                0x0800e710                list_is_empty
 .text.list_insert_head
                0x0800e728       0x18 Middlewares/STM32_BlueNRG/Utils/ble_list.o
                0x0800e728                list_insert_head
 .text.list_insert_tail
                0x0800e740       0x18 Middlewares/STM32_BlueNRG/Utils/ble_list.o
                0x0800e740                list_insert_tail
 .text.list_remove_head
                0x0800e758       0x34 Middlewares/STM32_BlueNRG/Utils/ble_list.o
                0x0800e758                list_remove_head
 .text.list_remove_tail
                0x0800e78c       0x34 Middlewares/STM32_BlueNRG/Utils/ble_list.o
                0x0800e78c                list_remove_tail
 .text.list_get_size
                0x0800e7c0       0x24 Middlewares/STM32_BlueNRG/Utils/ble_list.o
                0x0800e7c0                list_get_size
 .text.Timer_Set
                0x0800e7e4       0x10 Middlewares/STM32_BlueNRG/Utils/gp_timer.o
                0x0800e7e4                Timer_Set
 .text.Timer_Expired
                0x0800e7f4       0x1c Middlewares/STM32_BlueNRG/Utils/gp_timer.o
                0x0800e7f4                Timer_Expired
 .text.Osal_MemCpy
                0x0800e810        0x4 Middlewares/STM32_BlueNRG/Utils/osal.o
                0x0800e810                Osal_MemCpy
 .text.Osal_MemSet
                0x0800e814        0x4 Middlewares/STM32_BlueNRG/Utils/osal.o
                0x0800e814                Osal_MemSet
 .text.USBD_CDC_DataIn
                0x0800e818       0x14 Middlewares/STM32_USBD_Library/Class/CDC/usbd_cdc.o
 .text.USBD_CDC_EP0_RxReady
                0x0800e82c       0x2c Middlewares/STM32_USBD_Library/Class/CDC/usbd_cdc.o
 .text.USBD_CDC_GetFSCfgDesc
                0x0800e858        0xc Middlewares/STM32_USBD_Library/Class/CDC/usbd_cdc.o
 .text.USBD_CDC_GetHSCfgDesc
                0x0800e864        0xc Middlewares/STM32_USBD_Library/Class/CDC/usbd_cdc.o
 .text.USBD_CDC_GetOtherSpeedCfgDesc
                0x0800e870        0xc Middlewares/STM32_USBD_Library/Class/CDC/usbd_cdc.o
 .text.USBD_CDC_GetDeviceQualifierDescriptor
                0x0800e87c        0xc Middlewares/STM32_USBD_Library/Class/CDC/usbd_cdc.o
                0x0800e87c                USBD_CDC_GetDeviceQualifierDescriptor
 .text.USBD_CDC_DataOut
                0x0800e888       0x30 Middlewares/STM32_USBD_Library/Class/CDC/usbd_cdc.o
 .text.USBD_CDC_Setup
                0x0800e8b8       0x6c Middlewares/STM32_USBD_Library/Class/CDC/usbd_cdc.o
 .text.USBD_CDC_DeInit
                0x0800e924       0x3c Middlewares/STM32_USBD_Library/Class/CDC/usbd_cdc.o
 .text.USBD_CDC_Init
                0x0800e960       0x90 Middlewares/STM32_USBD_Library/Class/CDC/usbd_cdc.o
 .text.USBD_CDC_RegisterInterface
                0x0800e9f0       0x10 Middlewares/STM32_USBD_Library/Class/CDC/usbd_cdc.o
                0x0800e9f0                USBD_CDC_RegisterInterface
 .text.USBD_CDC_SetTxBuffer
                0x0800ea00       0x10 Middlewares/STM32_USBD_Library/Class/CDC/usbd_cdc.o
                0x0800ea00                USBD_CDC_SetTxBuffer
 .text.USBD_CDC_SetRxBuffer
                0x0800ea10        0xc Middlewares/STM32_USBD_Library/Class/CDC/usbd_cdc.o
                0x0800ea10                USBD_CDC_SetRxBuffer
 .text.USBD_CDC_TransmitPacket
                0x0800ea1c       0x30 Middlewares/STM32_USBD_Library/Class/CDC/usbd_cdc.o
                0x0800ea1c                USBD_CDC_TransmitPacket
 .text.USBD_Init
                0x0800ea4c       0x2c Middlewares/STM32_USBD_Library/Core/usbd_core.o
                0x0800ea4c                USBD_Init
 .text.USBD_RegisterClass
                0x0800ea78       0x10 Middlewares/STM32_USBD_Library/Core/usbd_core.o
                0x0800ea78                USBD_RegisterClass
 .text.USBD_Start
                0x0800ea88        0xc Middlewares/STM32_USBD_Library/Core/usbd_core.o
                0x0800ea88                USBD_Start
 .text.USBD_SetClassConfig
                0x0800ea94       0x14 Middlewares/STM32_USBD_Library/Core/usbd_core.o
                0x0800ea94                USBD_SetClassConfig
 .text.USBD_ClrClassConfig
                0x0800eaa8       0x10 Middlewares/STM32_USBD_Library/Core/usbd_core.o
                0x0800eaa8                USBD_ClrClassConfig
 .text.USBD_LL_SetupStage
                0x0800eab8       0x60 Middlewares/STM32_USBD_Library/Core/usbd_core.o
                0x0800eab8                USBD_LL_SetupStage
 .text.USBD_LL_DataOutStage
                0x0800eb18       0x6c Middlewares/STM32_USBD_Library/Core/usbd_core.o
                0x0800eb18                USBD_LL_DataOutStage
 .text.USBD_LL_DataInStage
                0x0800eb84       0xac Middlewares/STM32_USBD_Library/Core/usbd_core.o
                0x0800eb84                USBD_LL_DataInStage
 .text.USBD_LL_Reset
                0x0800ec30       0x40 Middlewares/STM32_USBD_Library/Core/usbd_core.o
                0x0800ec30                USBD_LL_Reset
 .text.USBD_LL_SetSpeed
                0x0800ec70        0x8 Middlewares/STM32_USBD_Library/Core/usbd_core.o
                0x0800ec70                USBD_LL_SetSpeed
 .text.USBD_LL_Suspend
                0x0800ec78       0x14 Middlewares/STM32_USBD_Library/Core/usbd_core.o
                0x0800ec78                USBD_LL_Suspend
 .text.USBD_LL_Resume
                0x0800ec8c       0x10 Middlewares/STM32_USBD_Library/Core/usbd_core.o
                0x0800ec8c                USBD_LL_Resume
 .text.USBD_LL_SOF
                0x0800ec9c       0x1c Middlewares/STM32_USBD_Library/Core/usbd_core.o
                0x0800ec9c                USBD_LL_SOF
 .text.USBD_LL_IsoINIncomplete
                0x0800ecb8        0x4 Middlewares/STM32_USBD_Library/Core/usbd_core.o
                0x0800ecb8                USBD_LL_IsoINIncomplete
 .text.USBD_LL_IsoOUTIncomplete
                0x0800ecbc        0x4 Middlewares/STM32_USBD_Library/Core/usbd_core.o
                0x0800ecbc                USBD_LL_IsoOUTIncomplete
 .text.USBD_LL_DevConnected
                0x0800ecc0        0x4 Middlewares/STM32_USBD_Library/Core/usbd_core.o
                0x0800ecc0                USBD_LL_DevConnected
 .text.USBD_LL_DevDisconnected
                0x0800ecc4       0x18 Middlewares/STM32_USBD_Library/Core/usbd_core.o
                0x0800ecc4                USBD_LL_DevDisconnected
 .text.USBD_StdDevReq
                0x0800ecdc      0x298 Middlewares/STM32_USBD_Library/Core/usbd_ctlreq.o
                0x0800ecdc                USBD_StdDevReq
 .text.USBD_StdItfReq
                0x0800ef74       0x40 Middlewares/STM32_USBD_Library/Core/usbd_ctlreq.o
                0x0800ef74                USBD_StdItfReq
 .text.USBD_StdEPReq
                0x0800efb4       0xcc Middlewares/STM32_USBD_Library/Core/usbd_ctlreq.o
                0x0800efb4                USBD_StdEPReq
 .text.USBD_ParseSetupRequest
                0x0800f080       0x28 Middlewares/STM32_USBD_Library/Core/usbd_ctlreq.o
                0x0800f080                USBD_ParseSetupRequest
 .text.USBD_GetString
                0x0800f0a8       0x50 Middlewares/STM32_USBD_Library/Core/usbd_ctlreq.o
                0x0800f0a8                USBD_GetString
 .text.USBD_CtlSendData
                0x0800f0f8       0x1c Middlewares/STM32_USBD_Library/Core/usbd_ioreq.o
                0x0800f0f8                USBD_CtlSendData
 .text.USBD_CtlContinueSendData
                0x0800f114       0x10 Middlewares/STM32_USBD_Library/Core/usbd_ioreq.o
                0x0800f114                USBD_CtlContinueSendData
 .text.USBD_CtlPrepareRx
                0x0800f124       0x20 Middlewares/STM32_USBD_Library/Core/usbd_ioreq.o
                0x0800f124                USBD_CtlPrepareRx
 .text.USBD_CtlContinueRx
                0x0800f144       0x10 Middlewares/STM32_USBD_Library/Core/usbd_ioreq.o
                0x0800f144                USBD_CtlContinueRx
 .text.USBD_CtlSendStatus
                0x0800f154       0x18 Middlewares/STM32_USBD_Library/Core/usbd_ioreq.o
                0x0800f154                USBD_CtlSendStatus
 .text.USBD_CtlReceiveStatus
                0x0800f16c       0x18 Middlewares/STM32_USBD_Library/Core/usbd_ioreq.o
                0x0800f16c                USBD_CtlReceiveStatus
 .text.__libc_init_array
                0x0800f184       0x48 c:/ac6/systemworkbench/plugins/fr.ac6.mcu.externaltools.arm-none.win32_1.17.0.201812190825/tools/compiler/bin/../lib/gcc/arm-none-eabi/7.3.1/../../../../arm-none-eabi/lib/thumb/v7e-m/fpv4-sp/hard\libc_nano.a(lib_a-init.o)
                0x0800f184                __libc_init_array
 .text.malloc   0x0800f1cc       0x10 c:/ac6/systemworkbench/plugins/fr.ac6.mcu.externaltools.arm-none.win32_1.17.0.201812190825/tools/compiler/bin/../lib/gcc/arm-none-eabi/7.3.1/../../../../arm-none-eabi/lib/thumb/v7e-m/fpv4-sp/hard\libc_nano.a(lib_a-malloc.o)
                0x0800f1cc                malloc
 .text.free     0x0800f1dc       0x10 c:/ac6/systemworkbench/plugins/fr.ac6.mcu.externaltools.arm-none.win32_1.17.0.201812190825/tools/compiler/bin/../lib/gcc/arm-none-eabi/7.3.1/../../../../arm-none-eabi/lib/thumb/v7e-m/fpv4-sp/hard\libc_nano.a(lib_a-malloc.o)
                0x0800f1dc                free
 .text.memcpy   0x0800f1ec       0x16 c:/ac6/systemworkbench/plugins/fr.ac6.mcu.externaltools.arm-none.win32_1.17.0.201812190825/tools/compiler/bin/../lib/gcc/arm-none-eabi/7.3.1/../../../../arm-none-eabi/lib/thumb/v7e-m/fpv4-sp/hard\libc_nano.a(lib_a-memcpy-stub.o)
                0x0800f1ec                memcpy
 .text.memmove  0x0800f202       0x32 c:/ac6/systemworkbench/plugins/fr.ac6.mcu.externaltools.arm-none.win32_1.17.0.201812190825/tools/compiler/bin/../lib/gcc/arm-none-eabi/7.3.1/../../../../arm-none-eabi/lib/thumb/v7e-m/fpv4-sp/hard\libc_nano.a(lib_a-memmove.o)
                0x0800f202                memmove
 .text.memset   0x0800f234       0x10 c:/ac6/systemworkbench/plugins/fr.ac6.mcu.externaltools.arm-none.win32_1.17.0.201812190825/tools/compiler/bin/../lib/gcc/arm-none-eabi/7.3.1/../../../../arm-none-eabi/lib/thumb/v7e-m/fpv4-sp/hard\libc_nano.a(lib_a-memset.o)
                0x0800f234                memset
 .text._free_r  0x0800f244       0x9c c:/ac6/systemworkbench/plugins/fr.ac6.mcu.externaltools.arm-none.win32_1.17.0.201812190825/tools/compiler/bin/../lib/gcc/arm-none-eabi/7.3.1/../../../../arm-none-eabi/lib/thumb/v7e-m/fpv4-sp/hard\libc_nano.a(lib_a-nano-freer.o)
                0x0800f244                _free_r
 .text._malloc_r
                0x0800f2e0       0xb4 c:/ac6/systemworkbench/plugins/fr.ac6.mcu.externaltools.arm-none.win32_1.17.0.201812190825/tools/compiler/bin/../lib/gcc/arm-none-eabi/7.3.1/../../../../arm-none-eabi/lib/thumb/v7e-m/fpv4-sp/hard\libc_nano.a(lib_a-nano-mallocr.o)
                0x0800f2e0                _malloc_r
 .text.__cvt    0x0800f394       0xc2 c:/ac6/systemworkbench/plugins/fr.ac6.mcu.externaltools.arm-none.win32_1.17.0.201812190825/tools/compiler/bin/../lib/gcc/arm-none-eabi/7.3.1/../../../../arm-none-eabi/lib/thumb/v7e-m/fpv4-sp/hard\libc_nano.a(lib_a-nano-vfprintf_float.o)
                0x0800f394                __cvt
 .text.__exponent
                0x0800f456       0x66 c:/ac6/systemworkbench/plugins/fr.ac6.mcu.externaltools.arm-none.win32_1.17.0.201812190825/tools/compiler/bin/../lib/gcc/arm-none-eabi/7.3.1/../../../../arm-none-eabi/lib/thumb/v7e-m/fpv4-sp/hard\libc_nano.a(lib_a-nano-vfprintf_float.o)
                0x0800f456                __exponent
 .text._printf_float
                0x0800f4bc      0x480 c:/ac6/systemworkbench/plugins/fr.ac6.mcu.externaltools.arm-none.win32_1.17.0.201812190825/tools/compiler/bin/../lib/gcc/arm-none-eabi/7.3.1/../../../../arm-none-eabi/lib/thumb/v7e-m/fpv4-sp/hard\libc_nano.a(lib_a-nano-vfprintf_float.o)
                0x0800f4bc                _printf_float
 .text._printf_common
                0x0800f93c       0xea c:/ac6/systemworkbench/plugins/fr.ac6.mcu.externaltools.arm-none.win32_1.17.0.201812190825/tools/compiler/bin/../lib/gcc/arm-none-eabi/7.3.1/../../../../arm-none-eabi/lib/thumb/v7e-m/fpv4-sp/hard\libc_nano.a(lib_a-nano-vfprintf_i.o)
                0x0800f93c                _printf_common
 *fill*         0x0800fa26        0x2 
 .text._printf_i
                0x0800fa28      0x224 c:/ac6/systemworkbench/plugins/fr.ac6.mcu.externaltools.arm-none.win32_1.17.0.201812190825/tools/compiler/bin/../lib/gcc/arm-none-eabi/7.3.1/../../../../arm-none-eabi/lib/thumb/v7e-m/fpv4-sp/hard\libc_nano.a(lib_a-nano-vfprintf_i.o)
                0x0800fa28                _printf_i
 .text._sbrk_r  0x0800fc4c       0x20 c:/ac6/systemworkbench/plugins/fr.ac6.mcu.externaltools.arm-none.win32_1.17.0.201812190825/tools/compiler/bin/../lib/gcc/arm-none-eabi/7.3.1/../../../../arm-none-eabi/lib/thumb/v7e-m/fpv4-sp/hard\libc_nano.a(lib_a-sbrkr.o)
                0x0800fc4c                _sbrk_r
 .text.sprintf  0x0800fc6c       0x40 c:/ac6/systemworkbench/plugins/fr.ac6.mcu.externaltools.arm-none.win32_1.17.0.201812190825/tools/compiler/bin/../lib/gcc/arm-none-eabi/7.3.1/../../../../arm-none-eabi/lib/thumb/v7e-m/fpv4-sp/hard\libc_nano.a(lib_a-sprintf.o)
                0x0800fc6c                siprintf
                0x0800fc6c                sprintf
 .text.quorem   0x0800fcac      0x118 c:/ac6/systemworkbench/plugins/fr.ac6.mcu.externaltools.arm-none.win32_1.17.0.201812190825/tools/compiler/bin/../lib/gcc/arm-none-eabi/7.3.1/../../../../arm-none-eabi/lib/thumb/v7e-m/fpv4-sp/hard\libc_nano.a(lib_a-dtoa.o)
 *fill*         0x0800fdc4        0x4 
 .text._dtoa_r  0x0800fdc8      0xb70 c:/ac6/systemworkbench/plugins/fr.ac6.mcu.externaltools.arm-none.win32_1.17.0.201812190825/tools/compiler/bin/../lib/gcc/arm-none-eabi/7.3.1/../../../../arm-none-eabi/lib/thumb/v7e-m/fpv4-sp/hard\libc_nano.a(lib_a-dtoa.o)
                0x0800fdc8                _dtoa_r
 .text._localeconv_r
                0x08010938       0x1c c:/ac6/systemworkbench/plugins/fr.ac6.mcu.externaltools.arm-none.win32_1.17.0.201812190825/tools/compiler/bin/../lib/gcc/arm-none-eabi/7.3.1/../../../../arm-none-eabi/lib/thumb/v7e-m/fpv4-sp/hard\libc_nano.a(lib_a-localeconv.o)
                0x08010938                _localeconv_r
 .text.__malloc_lock
                0x08010954        0x2 c:/ac6/systemworkbench/plugins/fr.ac6.mcu.externaltools.arm-none.win32_1.17.0.201812190825/tools/compiler/bin/../lib/gcc/arm-none-eabi/7.3.1/../../../../arm-none-eabi/lib/thumb/v7e-m/fpv4-sp/hard\libc_nano.a(lib_a-mlock.o)
                0x08010954                __malloc_lock
 .text.__malloc_unlock
                0x08010956        0x2 c:/ac6/systemworkbench/plugins/fr.ac6.mcu.externaltools.arm-none.win32_1.17.0.201812190825/tools/compiler/bin/../lib/gcc/arm-none-eabi/7.3.1/../../../../arm-none-eabi/lib/thumb/v7e-m/fpv4-sp/hard\libc_nano.a(lib_a-mlock.o)
                0x08010956                __malloc_unlock
 .text._Balloc  0x08010958       0x68 c:/ac6/systemworkbench/plugins/fr.ac6.mcu.externaltools.arm-none.win32_1.17.0.201812190825/tools/compiler/bin/../lib/gcc/arm-none-eabi/7.3.1/../../../../arm-none-eabi/lib/thumb/v7e-m/fpv4-sp/hard\libc_nano.a(lib_a-mprec.o)
                0x08010958                _Balloc
 .text._Bfree   0x080109c0       0x2e c:/ac6/systemworkbench/plugins/fr.ac6.mcu.externaltools.arm-none.win32_1.17.0.201812190825/tools/compiler/bin/../lib/gcc/arm-none-eabi/7.3.1/../../../../arm-none-eabi/lib/thumb/v7e-m/fpv4-sp/hard\libc_nano.a(lib_a-mprec.o)
                0x080109c0                _Bfree
 .text.__multadd
                0x080109ee       0x76 c:/ac6/systemworkbench/plugins/fr.ac6.mcu.externaltools.arm-none.win32_1.17.0.201812190825/tools/compiler/bin/../lib/gcc/arm-none-eabi/7.3.1/../../../../arm-none-eabi/lib/thumb/v7e-m/fpv4-sp/hard\libc_nano.a(lib_a-mprec.o)
                0x080109ee                __multadd
 .text.__hi0bits
                0x08010a64       0x3e c:/ac6/systemworkbench/plugins/fr.ac6.mcu.externaltools.arm-none.win32_1.17.0.201812190825/tools/compiler/bin/../lib/gcc/arm-none-eabi/7.3.1/../../../../arm-none-eabi/lib/thumb/v7e-m/fpv4-sp/hard\libc_nano.a(lib_a-mprec.o)
                0x08010a64                __hi0bits
 .text.__lo0bits
                0x08010aa2       0x5e c:/ac6/systemworkbench/plugins/fr.ac6.mcu.externaltools.arm-none.win32_1.17.0.201812190825/tools/compiler/bin/../lib/gcc/arm-none-eabi/7.3.1/../../../../arm-none-eabi/lib/thumb/v7e-m/fpv4-sp/hard\libc_nano.a(lib_a-mprec.o)
                0x08010aa2                __lo0bits
 .text.__i2b    0x08010b00       0x12 c:/ac6/systemworkbench/plugins/fr.ac6.mcu.externaltools.arm-none.win32_1.17.0.201812190825/tools/compiler/bin/../lib/gcc/arm-none-eabi/7.3.1/../../../../arm-none-eabi/lib/thumb/v7e-m/fpv4-sp/hard\libc_nano.a(lib_a-mprec.o)
                0x08010b00                __i2b
 .text.__multiply
                0x08010b12      0x12c c:/ac6/systemworkbench/plugins/fr.ac6.mcu.externaltools.arm-none.win32_1.17.0.201812190825/tools/compiler/bin/../lib/gcc/arm-none-eabi/7.3.1/../../../../arm-none-eabi/lib/thumb/v7e-m/fpv4-sp/hard\libc_nano.a(lib_a-mprec.o)
                0x08010b12                __multiply
 *fill*         0x08010c3e        0x2 
 .text.__pow5mult
                0x08010c40       0x9c c:/ac6/systemworkbench/plugins/fr.ac6.mcu.externaltools.arm-none.win32_1.17.0.201812190825/tools/compiler/bin/../lib/gcc/arm-none-eabi/7.3.1/../../../../arm-none-eabi/lib/thumb/v7e-m/fpv4-sp/hard\libc_nano.a(lib_a-mprec.o)
                0x08010c40                __pow5mult
 .text.__lshift
                0x08010cdc       0xa8 c:/ac6/systemworkbench/plugins/fr.ac6.mcu.externaltools.arm-none.win32_1.17.0.201812190825/tools/compiler/bin/../lib/gcc/arm-none-eabi/7.3.1/../../../../arm-none-eabi/lib/thumb/v7e-m/fpv4-sp/hard\libc_nano.a(lib_a-mprec.o)
                0x08010cdc                __lshift
 .text.__mcmp   0x08010d84       0x34 c:/ac6/systemworkbench/plugins/fr.ac6.mcu.externaltools.arm-none.win32_1.17.0.201812190825/tools/compiler/bin/../lib/gcc/arm-none-eabi/7.3.1/../../../../arm-none-eabi/lib/thumb/v7e-m/fpv4-sp/hard\libc_nano.a(lib_a-mprec.o)
                0x08010d84                __mcmp
 .text.__mdiff  0x08010db8       0xba c:/ac6/systemworkbench/plugins/fr.ac6.mcu.externaltools.arm-none.win32_1.17.0.201812190825/tools/compiler/bin/../lib/gcc/arm-none-eabi/7.3.1/../../../../arm-none-eabi/lib/thumb/v7e-m/fpv4-sp/hard\libc_nano.a(lib_a-mprec.o)
                0x08010db8                __mdiff
 .text.__d2b    0x08010e72       0x9e c:/ac6/systemworkbench/plugins/fr.ac6.mcu.externaltools.arm-none.win32_1.17.0.201812190825/tools/compiler/bin/../lib/gcc/arm-none-eabi/7.3.1/../../../../arm-none-eabi/lib/thumb/v7e-m/fpv4-sp/hard\libc_nano.a(lib_a-mprec.o)
                0x08010e72                __d2b
 .text._calloc_r
                0x08010f10       0x1c c:/ac6/systemworkbench/plugins/fr.ac6.mcu.externaltools.arm-none.win32_1.17.0.201812190825/tools/compiler/bin/../lib/gcc/arm-none-eabi/7.3.1/../../../../arm-none-eabi/lib/thumb/v7e-m/fpv4-sp/hard\libc_nano.a(lib_a-nano-callocr.o)
                0x08010f10                _calloc_r
 .text.__ssputs_r
                0x08010f2c       0xb4 c:/ac6/systemworkbench/plugins/fr.ac6.mcu.externaltools.arm-none.win32_1.17.0.201812190825/tools/compiler/bin/../lib/gcc/arm-none-eabi/7.3.1/../../../../arm-none-eabi/lib/thumb/v7e-m/fpv4-sp/hard\libc_nano.a(lib_a-nano-svfprintf.o)
                0x08010f2c                __ssputs_r
 .text._svfprintf_r
                0x08010fe0      0x1f0 c:/ac6/systemworkbench/plugins/fr.ac6.mcu.externaltools.arm-none.win32_1.17.0.201812190825/tools/compiler/bin/../lib/gcc/arm-none-eabi/7.3.1/../../../../arm-none-eabi/lib/thumb/v7e-m/fpv4-sp/hard\libc_nano.a(lib_a-nano-svfprintf.o)
                0x08010fe0                _svfiprintf_r
                0x08010fe0                _svfprintf_r
 .text.__ascii_mbtowc
                0x080111d0       0x24 c:/ac6/systemworkbench/plugins/fr.ac6.mcu.externaltools.arm-none.win32_1.17.0.201812190825/tools/compiler/bin/../lib/gcc/arm-none-eabi/7.3.1/../../../../arm-none-eabi/lib/thumb/v7e-m/fpv4-sp/hard\libc_nano.a(lib_a-mbtowc_r.o)
                0x080111d0                __ascii_mbtowc
 .text._realloc_r
                0x080111f4       0x4c c:/ac6/systemworkbench/plugins/fr.ac6.mcu.externaltools.arm-none.win32_1.17.0.201812190825/tools/compiler/bin/../lib/gcc/arm-none-eabi/7.3.1/../../../../arm-none-eabi/lib/thumb/v7e-m/fpv4-sp/hard\libc_nano.a(lib_a-nano-reallocr.o)
                0x080111f4                _realloc_r
 .text.__ascii_wctomb
                0x08011240       0x1a c:/ac6/systemworkbench/plugins/fr.ac6.mcu.externaltools.arm-none.win32_1.17.0.201812190825/tools/compiler/bin/../lib/gcc/arm-none-eabi/7.3.1/../../../../arm-none-eabi/lib/thumb/v7e-m/fpv4-sp/hard\libc_nano.a(lib_a-wctomb_r.o)
                0x08011240                __ascii_wctomb
 .text._malloc_usable_size_r
                0x0801125a       0x10 c:/ac6/systemworkbench/plugins/fr.ac6.mcu.externaltools.arm-none.win32_1.17.0.201812190825/tools/compiler/bin/../lib/gcc/arm-none-eabi/7.3.1/../../../../arm-none-eabi/lib/thumb/v7e-m/fpv4-sp/hard\libc_nano.a(lib_a-nano-msizer.o)
                0x0801125a                _malloc_usable_size_r
 *fill*         0x0801126a        0x2 
 .text._sbrk    0x0801126c       0x1c c:/ac6/systemworkbench/plugins/fr.ac6.mcu.externaltools.arm-none.win32_1.17.0.201812190825/tools/compiler/bin/../lib/gcc/arm-none-eabi/7.3.1/../../../../arm-none-eabi/lib/thumb/v7e-m/fpv4-sp/hard\libnosys.a(sbrk.o)
                0x0801126c                _sbrk
 *(.glue_7)
 .glue_7        0x08011288        0x0 linker stubs
 *(.glue_7t)
 .glue_7t       0x08011288        0x0 linker stubs
 *(.eh_frame)
 .eh_frame      0x08011288        0x0 c:/ac6/systemworkbench/plugins/fr.ac6.mcu.externaltools.arm-none.win32_1.17.0.201812190825/tools/compiler/bin/../lib/gcc/arm-none-eabi/7.3.1/thumb/v7e-m/fpv4-sp/hard/crtbegin.o
 *(.init)
 .init          0x08011288        0x4 c:/ac6/systemworkbench/plugins/fr.ac6.mcu.externaltools.arm-none.win32_1.17.0.201812190825/tools/compiler/bin/../lib/gcc/arm-none-eabi/7.3.1/thumb/v7e-m/fpv4-sp/hard/crti.o
                0x08011288                _init
 .init          0x0801128c        0x8 c:/ac6/systemworkbench/plugins/fr.ac6.mcu.externaltools.arm-none.win32_1.17.0.201812190825/tools/compiler/bin/../lib/gcc/arm-none-eabi/7.3.1/thumb/v7e-m/fpv4-sp/hard/crtn.o
 *(.fini)
 .fini          0x08011294        0x4 c:/ac6/systemworkbench/plugins/fr.ac6.mcu.externaltools.arm-none.win32_1.17.0.201812190825/tools/compiler/bin/../lib/gcc/arm-none-eabi/7.3.1/thumb/v7e-m/fpv4-sp/hard/crti.o
                0x08011294                _fini
 .fini          0x08011298        0x8 c:/ac6/systemworkbench/plugins/fr.ac6.mcu.externaltools.arm-none.win32_1.17.0.201812190825/tools/compiler/bin/../lib/gcc/arm-none-eabi/7.3.1/thumb/v7e-m/fpv4-sp/hard/crtn.o
                0x080112a0                . = ALIGN (0x8)
                0x080112a0                _etext = .

.vfp11_veneer   0x080112a0        0x0
 .vfp11_veneer  0x080112a0        0x0 linker stubs

.v4_bx          0x080112a0        0x0
 .v4_bx         0x080112a0        0x0 linker stubs

.iplt           0x080112a0        0x0
 .iplt          0x080112a0        0x0 c:/ac6/systemworkbench/plugins/fr.ac6.mcu.externaltools.arm-none.win32_1.17.0.201812190825/tools/compiler/bin/../lib/gcc/arm-none-eabi/7.3.1/thumb/v7e-m/fpv4-sp/hard/crtbegin.o

.rodata         0x080112a0      0x9f8
                0x080112a0                . = ALIGN (0x8)
 *(.rodata)
 .rodata        0x080112a0      0x17c Application/User/main.o
 .rodata        0x0801141c       0x22 Application/User/sensor_service.o
 *fill*         0x0801143e        0x2 
 .rodata        0x08011440       0x60 Drivers/BSP/Components/LSM303AGR_ACC_driver.o
                0x08011440                LSM303AGR_ACC_Sensitivity_List
 .rodata        0x080114a0        0x8 Drivers/BSP/SensorTile/SensorTile.o
                0x080114a0                GPIO_PIN
 .rodata        0x080114a8       0x48 Drivers/CMSIS/system_stm32l4xx.o
                0x080114a8                MSIRangeTable
                0x080114d8                AHBPrescTable
                0x080114e8                APBPrescTable
 *(.rodata*)
 .rodata.str1.4
                0x080114f0      0x2fa Application/User/main.o
 *fill*         0x080117ea        0x2 
 .rodata.str1.4
                0x080117ec      0x18a Application/User/sensor_service.o
 *fill*         0x08011976        0x2 
 .rodata.str1.4
                0x08011978       0x52 Application/User/usbd_desc.o
 .rodata.str1.4
                0x080119ca       0x52 Middlewares/FreeRTOS/CMSIS_RTOS/cmsis_os.o
                                  0x1 (size before relaxing)
 *fill*         0x080119ca        0x2 
 .rodata.str1.4
                0x080119cc       0x10 Middlewares/FreeRTOS/timers.o
 .rodata._printf_float.str1.1
                0x080119dc       0x12 c:/ac6/systemworkbench/plugins/fr.ac6.mcu.externaltools.arm-none.win32_1.17.0.201812190825/tools/compiler/bin/../lib/gcc/arm-none-eabi/7.3.1/../../../../arm-none-eabi/lib/thumb/v7e-m/fpv4-sp/hard\libc_nano.a(lib_a-nano-vfprintf_float.o)
 .rodata._printf_i.str1.1
                0x080119ee       0x22 c:/ac6/systemworkbench/plugins/fr.ac6.mcu.externaltools.arm-none.win32_1.17.0.201812190825/tools/compiler/bin/../lib/gcc/arm-none-eabi/7.3.1/../../../../arm-none-eabi/lib/thumb/v7e-m/fpv4-sp/hard\libc_nano.a(lib_a-nano-vfprintf_i.o)
 .rodata._dtoa_r.str1.1
                0x08011a10        0xd c:/ac6/systemworkbench/plugins/fr.ac6.mcu.externaltools.arm-none.win32_1.17.0.201812190825/tools/compiler/bin/../lib/gcc/arm-none-eabi/7.3.1/../../../../arm-none-eabi/lib/thumb/v7e-m/fpv4-sp/hard\libc_nano.a(lib_a-dtoa.o)
                                  0xf (size before relaxing)
 *fill*         0x08011a1d        0x3 
 .rodata.__sf_fake_stderr
                0x08011a20       0x20 c:/ac6/systemworkbench/plugins/fr.ac6.mcu.externaltools.arm-none.win32_1.17.0.201812190825/tools/compiler/bin/../lib/gcc/arm-none-eabi/7.3.1/../../../../arm-none-eabi/lib/thumb/v7e-m/fpv4-sp/hard\libc_nano.a(lib_a-findfp.o)
                0x08011a20                __sf_fake_stderr
 .rodata.__sf_fake_stdin
                0x08011a40       0x20 c:/ac6/systemworkbench/plugins/fr.ac6.mcu.externaltools.arm-none.win32_1.17.0.201812190825/tools/compiler/bin/../lib/gcc/arm-none-eabi/7.3.1/../../../../arm-none-eabi/lib/thumb/v7e-m/fpv4-sp/hard\libc_nano.a(lib_a-findfp.o)
                0x08011a40                __sf_fake_stdin
 .rodata.__sf_fake_stdout
                0x08011a60       0x20 c:/ac6/systemworkbench/plugins/fr.ac6.mcu.externaltools.arm-none.win32_1.17.0.201812190825/tools/compiler/bin/../lib/gcc/arm-none-eabi/7.3.1/../../../../arm-none-eabi/lib/thumb/v7e-m/fpv4-sp/hard\libc_nano.a(lib_a-findfp.o)
                0x08011a60                __sf_fake_stdout
 .rodata.__mprec_bigtens
                0x08011a80       0x28 c:/ac6/systemworkbench/plugins/fr.ac6.mcu.externaltools.arm-none.win32_1.17.0.201812190825/tools/compiler/bin/../lib/gcc/arm-none-eabi/7.3.1/../../../../arm-none-eabi/lib/thumb/v7e-m/fpv4-sp/hard\libc_nano.a(lib_a-mprec.o)
                0x08011a80                __mprec_bigtens
 .rodata.__mprec_tens
                0x08011aa8       0xc8 c:/ac6/systemworkbench/plugins/fr.ac6.mcu.externaltools.arm-none.win32_1.17.0.201812190825/tools/compiler/bin/../lib/gcc/arm-none-eabi/7.3.1/../../../../arm-none-eabi/lib/thumb/v7e-m/fpv4-sp/hard\libc_nano.a(lib_a-mprec.o)
                0x08011aa8                __mprec_tens
 .rodata.p05.7359
                0x08011b70        0xc c:/ac6/systemworkbench/plugins/fr.ac6.mcu.externaltools.arm-none.win32_1.17.0.201812190825/tools/compiler/bin/../lib/gcc/arm-none-eabi/7.3.1/../../../../arm-none-eabi/lib/thumb/v7e-m/fpv4-sp/hard\libc_nano.a(lib_a-mprec.o)
 .rodata._svfprintf_r.str1.1
                0x08011b7c       0x11 c:/ac6/systemworkbench/plugins/fr.ac6.mcu.externaltools.arm-none.win32_1.17.0.201812190825/tools/compiler/bin/../lib/gcc/arm-none-eabi/7.3.1/../../../../arm-none-eabi/lib/thumb/v7e-m/fpv4-sp/hard\libc_nano.a(lib_a-nano-svfprintf.o)
 .rodata._setlocale_r.str1.1
                0x08011b8d        0x8 c:/ac6/systemworkbench/plugins/fr.ac6.mcu.externaltools.arm-none.win32_1.17.0.201812190825/tools/compiler/bin/../lib/gcc/arm-none-eabi/7.3.1/../../../../arm-none-eabi/lib/thumb/v7e-m/fpv4-sp/hard\libc_nano.a(lib_a-locale.o)
                                  0x9 (size before relaxing)
 .rodata.str1.1
                0x08011b95        0x2 c:/ac6/systemworkbench/plugins/fr.ac6.mcu.externaltools.arm-none.win32_1.17.0.201812190825/tools/compiler/bin/../lib/gcc/arm-none-eabi/7.3.1/../../../../arm-none-eabi/lib/thumb/v7e-m/fpv4-sp/hard\libc_nano.a(lib_a-locale.o)
 .rodata._ctype_
                0x08011b97      0x101 c:/ac6/systemworkbench/plugins/fr.ac6.mcu.externaltools.arm-none.win32_1.17.0.201812190825/tools/compiler/bin/../lib/gcc/arm-none-eabi/7.3.1/../../../../arm-none-eabi/lib/thumb/v7e-m/fpv4-sp/hard\libc_nano.a(lib_a-ctype_.o)
                0x08011b97                _ctype_
                0x08011c98                . = ALIGN (0x8)

.ARM.extab
 *(.ARM.extab* .gnu.linkonce.armextab.*)

.ARM            0x08011c98        0x8
                0x08011c98                __exidx_start = .
 *(.ARM.exidx*)
 .ARM.exidx     0x08011c98        0x8 c:/ac6/systemworkbench/plugins/fr.ac6.mcu.externaltools.arm-none.win32_1.17.0.201812190825/tools/compiler/bin/../lib/gcc/arm-none-eabi/7.3.1/thumb/v7e-m/fpv4-sp/hard\libgcc.a(_udivmoddi4.o)
                0x08011ca0                __exidx_end = .

.rel.dyn        0x08011ca0        0x0
 .rel.iplt      0x08011ca0        0x0 c:/ac6/systemworkbench/plugins/fr.ac6.mcu.externaltools.arm-none.win32_1.17.0.201812190825/tools/compiler/bin/../lib/gcc/arm-none-eabi/7.3.1/thumb/v7e-m/fpv4-sp/hard/crtbegin.o

.preinit_array  0x08011ca0        0x0
                0x08011ca0                PROVIDE (__preinit_array_start = .)
 *(.preinit_array*)
                0x08011ca0                PROVIDE (__preinit_array_end = .)

.init_array     0x08011ca0        0x8
                0x08011ca0                PROVIDE (__init_array_start = .)
 *(SORT_BY_NAME(.init_array.*))
 *(.init_array*)
 .init_array    0x08011ca0        0x4 c:/ac6/systemworkbench/plugins/fr.ac6.mcu.externaltools.arm-none.win32_1.17.0.201812190825/tools/compiler/bin/../lib/gcc/arm-none-eabi/7.3.1/thumb/v7e-m/fpv4-sp/hard/crtbegin.o
 .init_array    0x08011ca4        0x4 Application/User/main.o
                0x08011ca8                PROVIDE (__init_array_end = .)

.fini_array     0x08011ca8        0x4
                [!provide]                PROVIDE (__fini_array_start = .)
 *(SORT_BY_NAME(.fini_array.*))
 *(.fini_array*)
 .fini_array    0x08011ca8        0x4 c:/ac6/systemworkbench/plugins/fr.ac6.mcu.externaltools.arm-none.win32_1.17.0.201812190825/tools/compiler/bin/../lib/gcc/arm-none-eabi/7.3.1/thumb/v7e-m/fpv4-sp/hard/crtbegin.o
                [!provide]                PROVIDE (__fini_array_end = .)
                0x08011cac                _sidata = LOADADDR (.data)

.data           0x20000000     0x3418 load address 0x08011cac
                0x20000000                . = ALIGN (0x8)
